:020000040000FA
:040000006FD00400B9
:101000006F00907E00000000000000009020002093
:10101000AA220020A9BDF9F56C23002000000000E1
:10102000000000006C230020902000200000000041
:101030000000000090200020000000009020002010
:101040000000000090200020902000209020002030
:101050009020002090200020582F00209424002071
:101060000000000090200020902000201E2400207E
:1010700090200020D22300209020002090200020EB
:101080009020002090200020902000209020002020
:101090009020002001A04111B7170040985F3AC688
:1010A000945F3247E39CE6FE3245410182800111A4
:1010B00013078008F337078093F787083EC20100C3
:1010C0000100B7170040930570052380B70413068D
:1010D00080FA2380C7040100010083C6B70493F699
:1010E000F60DA385D704238007049246F3A6068055
:1010F0000100010093760502D5CEF336078093F602
:10110000860836C4010001002380B7042380C70489
:1011100001000100B70614007D89558D88C70100C4
:1011200001000100010023800704A246F3A6068007
:101130000100010073370780137787083AC6010062
:1011400001002380B7042380C704010001000100CF
:1011500001003727004093061005A303D7802380A2
:101160000704B247F3A70780010001009307800836
:10117000F3B7078093F787083ECE01000100B71749
:101180000040130770052380E704130780FA2380CB
:10119000E7040100010003C7B70413670708A3852C
:1011A000E70423800704F247F3A70780010001004A
:1011B0000561828093760504BDC6F336078093F6F9
:1011C000860836C8010001002380B7042380C704C5
:1011D00001000100B7061400938606047D89558D31
:1011E00088C7010001000100010023800704C246F6
:1011F000F3A6068001000100733707801377870884
:101200003ACA010001002380B7042380C70401000B
:1012100001003727004093062005A303D7802380D1
:101220000704D24781B773370780137787083ACC12
:10123000010001002380B7042380C70401000100DE
:1012400098471367070C98C723800704E24719BF24
:101250000111814601468145114506CE97000000E7
:10126000E780605893078008F3B7078093F78708F3
:101270003EC601000100B717004013077005238028
:10128000E704130780FA2380E7040100010003C785
:101290006704136717002383E70423800704B2471A
:1012A000F3A7078001000100F2400561828041112F
:1012B000814601468145114597000000E780A05214
:1012C00013078008F337078093F787083EC40100AF
:1012D0000100B7170040130670052380C70493066A
:1012E00080FA2380D70401000100FD552396B70240
:1012F00023800704A245F3A5058001000100733790
:101300000780137787083AC6010001002380C704CD
:101310002380D7040100010003C767041367170087
:101320002383E70423800704B247F3A70780010063
:10133000010001A0B1473305F50201007D1575FDDF
:101340008280411122C426C206C6AA8401446317C2
:101350009400B24022449244410182800504130566
:10136000803E420497000000E78000FD4180C5B741
:101370009305000273A04580824573901534924016
:101380002242B2424243D2436244F2440255925551
:101390002256B2564257D2576258F25806499649D9
:1013A000264AB64A464BD64B664CF64C065D965DD1
:1013B000265EB65E465FD65F09617300203041113C
:1013C000B7170040985F3AC6945F3247E39CE6FE49
:1013D000324541018280B71700401307000323887C
:1013E000E702854717170000232EF74673002030C9
:1013F000411122C42D6426C24AC006C637190040D6
:101400001304A4AAB704002023208900976000E0F9
:10141000E78080439C408297976000E0E780C0426D
:10142000E5B737370040834747009146BD8B639E41
:10143000D702B73600401306F00F973500009385AA
:10144000651F9737000083D7E72E03C7A6001377E1
:10145000F70F1DE3B7E70400BC4F09468945171590
:1014600000000345A5F7829731A099466394D70001
:10147000834757007300203003C786001377F70FA8
:10148000E365F6FC13851700AE97173800002313A9
:10149000A82A2380E70075B7B787004003C7670015
:1014A000098B6309071003C77700930600031377BE
:1014B0000703630DD70817380000034878771736FD
:1014C00000001306E6730547B30606012380E60015
:1014D00083C577001737000013078774429793F589
:1014E000F50F2300B70003C58700973500009385EB
:1014F0002572C2951375F50F2380A50003470700D9
:1015000089451377F703630CB70C63E7E50A6306B5
:10151000071A8545630CB7129737000083C75771C8
:101520003307F600034707001377F70F19CB85073A
:1015300093F7F70F3D476363F71A17370000A309C6
:10154000F76EB787004009472383E700B78700405D
:1015500083C77700E207E18763DE0704973700005F
:1015600083C7176D17370000130787693E978546B5
:101570002300D700173700001307876A3E979306AA
:1015800000032300D70017370000130767683E9752
:10159000A14685072300D70093F7F70F3D47636403
:1015A000F71417370000A305F768B787004009470D
:1015B0002383E70073002030930610026300D70EE8
:1015C000930620026305D70693060002E316D7F4BC
:1015D00003C727021377C70F13672700D5A803C7D0
:1015E00067001377070465CB03C7A702173800000D
:1015F00013088842173500001305C539134707083B
:101600002385E70203C7A7021377370F1367870005
:101610002385E702814713070004B305F5008C41D9
:10162000B306F80091078CC2E399E7FEF5B503C74E
:10163000A702134707042385E70203C7A70213770E
:10164000C70F136727002385E702F9B503C76700B3
:101650001377070449C303C767021738000013084C
:10166000682F173500001305A526134707082383A5
:10167000E70203C767021377370F136787002383D7
:10168000E702814713070004B305F5008C41B30658
:10169000F80091078CC2E399E7FEBDBD03C767025E
:1016A000134707042383E70203C767021377C70FB3
:1016B000136727002383E70285B503C76700137705
:1016C000070411CB03C727021377370F136787006F
:1016D0002381E70291B5238006003DBD97370000C6
:1016E000A3880754B9BD97370000A383075475BD7D
:1016F0002303048015472303E48001002302A48010
:10170000828083076480E3CE07FE23030480828007
:1017100083076480E3CE07FE03454480828083070D
:101720006480E3CE07FE2302A4808280411126C498
:101730004AC24EC006C61377F50BAD47AA892E895B
:101740009544630CF700194597000000E78080FA84
:1017500097000000E78020FB8D444E859700000035
:10176000E78040F9FD59FD1463983401B240A2446A
:101770001249824941018280135509011375F50F01
:1017800097000000E780E0F92209F1BF011126CCA3
:1017900006CEB704080097000000E780C0F61545A4
:1017A00097000000E78000F597000000E78080F6D2
:1017B00097000000E78000F62AC697000000E78047
:1017C00080F432459377150089EB13651500137586
:1017D000F50FF240E24405618280FD14E9F0014515
:1017E000CDBF397126DC4ADA4ED852D656D45AD2F9
:1017F0005ED006DE62CE66CCB7E700E07D5783AAF6
:10180000070022C603AA470023A0E71823A2E7186F
:10181000B7170040130770052380E704130780FA09
:101820002380E70483C74704930B75FFB684E20760
:1018300093FBFB0F8546AA892E8B32893724004003
:10184000E187015763FA76016308D50089461307DB
:1018500000026313D5000157D98F93F7F70FB71C18
:1018600000402382FC0411472303E4801305F00F9A
:1018700097000000E78000E8094C97000000E7802F
:1018800080E863657C15B7050700DA9537870700A0
:10189000795563FEE504B3879500636AF704370B57
:1018A0000800A94733EB65016395F90881E8814495
:1018B00097000000E78020E5268515A8DA85094510
:1018C00097000000E780C0E605090345F9FFFD1415
:1018D000050B97000000E780C0E481C49377FB0FFD
:1018E000E5F797000000E780A0EA69F17D55B7179A
:1018F0000040130770052380E704130780FA238054
:10190000E70403C74704418B2382E704F250B7E79B
:1019100000E023A0571123A24711E2543244525948
:10192000C259325AA25A125B825B724CE24C21615C
:101930008280A547639BF90685691309F00FB306FA
:101940009900B3742B01B6941349F9FFB37499004D
:10195000856B33796901416B9387F9FFB3F72701F1
:1019600099E363FC340193D94900C147E3E637FFAB
:101970003DBF0569C1697D19D9B71305800D63881D
:101980006901130500026384790113051008CA85F3
:1019900097000000E780C0D997000000E78040DF93
:1019A00031D54E99B38434416DBFDA852D4597000A
:1019B0000000E780E0D7CA94E30B99EE0509970091
:1019C0000000E78020D5A30FA9FEFDB79387F9FF9C
:1019D00093F7F70F636DFC0C83C71C0413073008E3
:1019E0006315F706370708006361EB06B3079B0032
:1019F000B706100063FBD704334BEB0089476399AC
:101A0000F9068980D549E38404EADA850945970017
:101A10000000E780E0D111090327C9FF9147232087
:101A2000E48003076480E34E07FE23033481FD173F
:101A3000EDFBFD14110B81C49377FB0FE9FF9700B9
:101A40000000E780E0D461F155B5B717004003C747
:101A50005704B70708001377070219E3B787070091
:101A60007955E376FBE833079B00E3F9E7F841B5E6
:101A70008547E380F9F0DA852D4597000000E7807F
:101A800020CB9389F4FFE38404E297000000E78011
:101A900060C893F7390091EB83260480032709007F
:101AA00093074900E396E6E03E89CE84D9BFB54767
:101AB0006399F9001305900B97000000E78080C33D
:101AC000FDB3B1471305B00AE388F9FE9947639760
:101AD000F904B7050800B365BB002D459700000069
:101AE000E78000C581448D4BA14997000000E78045
:101AF00060C263967401832704802320F900850463
:101B0000E39534FF8327048013172B0163550700E7
:101B10002312F90069BB2322F90051BB9D47639F43
:101B2000F90281451305B00497000000E78040C02A
:101B3000BD442320090023220900FD59970000001D
:101B4000E78040BD93F77400CA9703C70700FD14F0
:101B5000398D2380A700E39334FF91BBA14763979E
:101B6000F90697000000E780A0C28144630D0B00D6
:101B70008D479304C0036308FB00930400056304CE
:101B80008B01930440041375C507E30295D21945F0
:101B900097000000E78000B697000000E780A0B63D
:101BA000054597000000E780E0B426859700000017
:101BB000E78020B7094597000000E78080B69700CE
:101BC0000000E780E0BCE31405CE0DB39147639FAE
:101BD000F9001305600697000000E780A0B19700A8
:101BE0000000E78040B213059009F9B5E38109CC04
:101BF000F1547DB9BD660147173600001306C620B3
:101C0000938606A685458347060093F7F70F91C391
:101C100082800507E3F9E6FE973700002386B71EAA
:101C2000DDB77D166206618693178601E18763D46E
:101C3000070001458280931726003307F500AE9711
:101C400018439C4363E7E7007D16E37FF7FC7D556F
:101C5000828005458280FD15E205E18513978501A7
:101C6000618793F7F50F63480700FD15139725006B
:101C70002A97584365D713851700620561858280CE
:101C80003308B5021C4283A80600B335B502C297DB
:101C900033B50701AE98469585486367B5006394F0
:101CA000A50063E3070181480C43C6950CC388C2B5
:101CB0001CC2828081471397870161876343B70005
:101CC0008280139727002A97232007008507E5B70E
:101CD0008147014793968701E18663C5B6001335B6
:101CE0001700828093962700AA9694428507558F05
:101CF000D5B793D755408A07AA979C430545331516
:101D0000B5007D8D828017F3FFDFE702833D2A84D3
:101D100097000000E78060F405C5931725003E9406
:101D20000327C4FF814711EB7D1516053E9542053B
:101D3000418517F3FFDF6700033D05838507E5B79E
:101D40000145C5BF81471397870161876343C7007A
:101D5000828013972700B386E50094422A9785076F
:101D600014C3D5B77D1662066186014793178601B5
:101D7000E18763D50700133517008280931726008B
:101D8000B306F500AE9794429C437D16B58F5D8FE8
:101D9000F1BF8A05AA9501476363B500828083A6D7
:101DA000C5FFF11593D71600D98F9CC11397F60183
:101DB000E5B72A830148014701456343D700828084
:101DC000B387050183A80700B30706019C43C697A4
:101DD000AA976384F80033B517010507B308030118
:101DE000620723A0F80061871108C1BF2A83014759
:101DF0008147014563C3D70082803388E50083288B
:101E00000800330EE600032E0E003388A840330886
:101E1000C8416384080133B508018507B308E300AE
:101E2000E20723A00801E1871107E9B717F3FFDFF5
:101E3000E702232B0111B286B2842E86AA850A8579
:101E400097000000E780C0FA2A84A6850A859700DB
:101E50000000E78020E833348000060413351500C5
:101E6000018D056117F3FFDF6700E32917F3FFDF3B
:101E7000E702A3244111AA89AE8A328BB68402C23A
:101E800002C402C60144131C8401135C8C416349E3
:101E90009C02939B1400FD1B0549138CF4FFF15C1D
:101EA00033048901620461846340740792478E049D
:101EB000CE9423AEF4FE410117F3FFDF67006323E6
:101EC00013192400B30B2B01014A93172A00D6974C
:101ED00083A50B0088437800340050009700000071
:101EE000E78040DA050A93178A01E187F11BE35E78
:101EF000FCFC92474E9905042320F900A2473EC2FC
:101F0000B24702C63EC441B7131A8901135A8A4127
:101F1000131D240093178A01E18763CF970092472E
:101F20000A044E941CC0A24705091379F90F3EC25A
:101F3000B24702C63EC4ADB7B3079A0313152A00D1
:101F400056950841780034005000050AEA97DA9760
:101F50008C4397000000E780E0D26DBF197106C284
:101F600012C416C61AC81ECA22CC26CE2AD02ED219
:101F700032D436D63AD83EDA42DC46DECAC0CEC2C9
:101F8000D2C4D6C6DAC8DECAE2CCE6CEEAD0EED2F9
:101F9000F2D4F6D6FAD8FEDA971500009385058CB0
:101FA0008841E700050092402242B2424243D243B8
:101FB0006244F244025592552256B2564257D257C5
:101FC0006258F25806499649264AB64A464BD64BBD
:101FD000664CF64C065D965D265EB65E465FD65F45
:101FE0000961730020300000972100209381810156
:101FF000175100201301018117F5FFFF1305C500DC
:102000009705002093850500171600201306C6FDCE
:1020100063FAC5008322050023A055001105910530
:10202000E3EAC5FE17050200130505FF971500201A
:102030009385C5FB171600201306C66563FAC50015
:102040008322050023A0550011059105E3EAC5FE92
:1020500017150020130505649745002093858526F4
:102060006377B500232005001105E36DB5FEFD4241
:10207000739002BC8D4273904280B722000093821D
:10208000828873900230970200209382A2F793E235
:10209000320073905230975200009382C294739032
:1020A00012346FB0F47573002030397101436EC67D
:1020B00019A0397141536AC866CA62CC5ECE19A0B4
:1020C000397101535AD056D252D44ED64AD826DA54
:1020D00022DC06DE33016140828241114AC026C201
:1020E00022C406C68282B24D4101024D924C224C5E
:1020F000B24B4101024B924A224AB2494101024984
:1021000092442244B240410182803D432A87637356
:10211000C3029377F700BDEFADE5937606FF3D8AE6
:10212000BA960CC34CC30CC74CC74107E36BD7FE30
:1021300011E28280B306C3408A0697020000969699
:102140006780A6002307B700A306B7002306B700E1
:10215000A305B7002305B700A304B7002304B70005
:10216000A303B7002303B700A302B7002302B700FD
:10217000A301B7002301B700A300B7002300B700F5
:10218000828093F5F50F93968500D58D9396050182
:10219000D58D61B7939627009702000096968682A8
:1021A000E78086FA9680C1171D8F3E96E374C3F8C8
:1021B000A5B73367B500FD530D8B79E7B7877F7FF0
:1021C0009387F7F710419441B372F6003363F6003A
:1021D000BE92B3E262006397720C6318D606504158
:1021E000D441B372F6003363F600BE92B3E26200EC
:1021F0006398720A631BD60410459445B372F600C7
:102200003363F600BE92B3E262006391720A631E0A
:10221000D6025045D445B372F6003363F600BE9241
:10222000B3E26200639A72086311D60210499449BE
:10223000B372F6003363F600BE92B3E262006393BA
:1022400072085105D105E30FD6F6131706019397CF
:102250000601631CF7001357060193D706013305E7
:10226000F7409375F50F91E982804183C18333056F
:10227000F7409375F50F91E182801377F70F93F78D
:10228000F70F3305F74082800346050083C605003B
:10229000050585056313D60065FA3305D6408280AF
:1022A00011059105E312D6FE014582802105A105A5
:1022B000E31CD6FC014582803105B105E316D6FC4E
:1022C000014582804105C105E310D6FC01458280AD
:1022D000B717004003C777051377E70FA38BE70411
:1022E000130700F8A38DE7043D47238CE704130789
:1022F0005003A38CE70403C7A7051377D70F238DDB
:10230000E7048280B717004003C7E7020D89411137
:102310001377C70F498F93068008F3B6068093F6AC
:10232000860836C601000100930670052380D70495
:10233000930680FA2380D704010001002387E70277
:1023400023800704B247F3A7078001000100410181
:10235000828041112A83014E930E407E130F001993
:10236000930F400663E56E129308001913034006AD
:10237000B3781503854E0D4FA14F337365020D8958
:102380001335150063EFBE121308F6FF79467298F5
:102390004208135808013307C70213D61700BE07B7
:1023A00032976146B3F6C60213068070B386C60242
:1023B0003697A166F58F42075D8FB716004083C739
:1023C000F60293F70708A303F1000346710083C7E1
:1023D000F60293F70708E394C7FE83477100B71628
:1023E000004093F7F70F6388071293078008F3B74D
:1023F000078093F787083EC401000100B71700402B
:10240000930670052380D704930680FA2380D704AF
:102410000100010023AA070383C6170393E60608F9
:10242000A388D70223800704A247F3A707800100EF
:1024300001001166B71700407D16D45BC85F938515
:102440004703A98EF18EF5FA93068008F3B606804D
:1024500093F6860836C601000100930670052380B6
:10246000D704930680FA2380D7040100010098C1A5
:1024700003C7170313670704A388E7022380070431
:10248000B247F3A7078001000100410182807D135C
:102490003368E3039308E016630E08003368F30320
:1024A0009308D016630808009378330093B8180097
:1024B0009388D81633081E01131E0801135E0E01FF
:1024C00055B56393E5030548638608000148630337
:1024D00003002A8871087298FD15131E0801C205B1
:1024E000135E0E01C18179BD13F8150063F4BF00BE
:1024F0007908D5B713381800E5BF83C7F60293F7FC
:102500000708A303F1000346710083C7F60293F79F
:102510000708E394C7FE8347710093F7F70FF1DFD5
:10252000E9B531714AD966CB06DF22DD26DB4ED70D
:1025300052D556D35AD15ECF62CD6AC96EC7AA8C26
:1025400002D897100000E78020B12A8993078008FD
:10255000F3B7078093F787083EDA01000100B71749
:102560000040130770052380E704130780FA2380D7
:10257000E7040100010003C7F7021377770FA38771
:10258000E70203C7F70213678700A387E7022380E8
:102590000704D257F3A70780010001000545970003
:1025A0000000E78060D6130780C13347E902116A53
:1025B00093070AE893065002BD69930BA004814A71
:1025C000014B13048008930470057D1AB347F90288
:1025D0003307D7023EC0FD873ECC938709A69309F7
:1025E000803E3347F7023AC27D873AC43347390306
:1025F0008549B399990193D93940B306D702B30BF2
:102600007703B3C6F602B3CBFB0236C6FD8636C8E7
:1026100093D6FB4136CEB7460F0093860624334946
:10262000D9028566938606FAB3969601B389E902C4
:10263000130760553309D90293060010B389E902E4
:102640003349D902B3C9F9029316390036CA37198A
:102650000040FD8636D0930D090493D7F9413ED250
:10266000F336048093F6860836DC010001009307F8
:1026700070052380FD00930680FA2380DD000100B1
:1026800001008346390593F6860FA309D9048346D2
:10269000390593E61600A309D90423800D00E256FC
:1026A000F3A6068001000100130C80FA116DF336C9
:1026B000048093F6860836DE01000100930770055A
:1026C0002380FD0023808D01010001008346390530
:1026D000216693E60602A309D90483560905B3E6E9
:1026E000A6012318D90483560905D18E2318D904CD
:1026F00023800D00F256F3A60680010001008346F8
:10270000390593F606026381061A03463905218AC4
:102710006DDE081897100000E7800098733604807B
:1027200013768608B2C20100010023809D00238039
:102730008D0101000100B717004003C6370513766D
:10274000F60DA389C70403C6370513660602A389DD
:10275000C704835609052166B3E6A6012318D904E8
:1027600083560905D18E2318D90423800D0096467F
:10277000F3A60680010001008346390593F60602A0
:10278000638B061483463905A18AEDFE970000206D
:10279000E7806090AA8636D497000020E780A08F5B
:1027A000A256E30AD5FE835609054255B3E6A601B3
:1027B0002318D90497100000E780C08F834639059D
:1027C000A18AEDDE03560905834629058247337643
:1027D000CA00B306DA0293D5F641B296B388F64042
:1027E000E24733B8C6002E983308F840A247B3B684
:1027F00016013308D84063C70701631DF8009247EC
:1028000063FA1701C247634FF80E63950701B24799
:1028100063EAF80E894663E9660FF24693151800DD
:1028200013D3F8015E8613951800B365B30042D642
:1028300046D497C00100E78020E53258050B137B92
:10284000FB0F63470001631A0838A25863870838F2
:1028500013081500B336A800B69513D6F5013298C3
:10286000B336C800AE9613581800FE06B3E606014C
:102870007336048013768608B2C6010001002380F7
:102880009D0023808D01010001000356C902B2960C
:10289000C206C1822316D90223800D00B646F3A6D4
:1028A00006800100010021B5F336048093F6860806
:1028B000B6C00100010023809D0023808D0101002E
:1028C00001008346390593E60602A309D904238053
:1028D0000D0086460DB5F336048093F68608B6C41F
:1028E0000100010023809D0023808D010100010073
:1028F0008346390593E60602A309D90423800D0017
:10290000A646BDB5E30B0BF0F336048093F68608BC
:10291000B6C801000100930680FA23809D00238041
:10292000DD00010001008346390593F5FC0F93F6A5
:10293000860FA309D90483463905CD8EA309D9048E
:1029400023800D00C646F3A6068001000100130592
:1029500080FA03463905930639051D8A631C9629BA
:102960007336048013768608B2CC0100010013068A
:1029700080FA23809D002380CD000100010003C662
:1029800006001376F60D2380C60003C60600136604
:1029900006022380C600835609051166D18E2318CE
:1029A000D904835609052166D18E2318D9042380C2
:1029B0000D00E646F3A6068001000100130680FA2A
:1029C0008346390593F60602638006268346390559
:1029D000130C3905A18AFDDA081897000000E7807A
:1029E000A06BF336048093F68608B6D00100010090
:1029F000930680FA23809D002380DD000100010002
:102A000083460C00116693F6F60D2300DC00834626
:102A10000C0093E606022300DC0083560905D18EE4
:102A20002318D904835609052166D18E2318D904A9
:102A300023800D008656F3A60680010001001306D0
:102A400080FA8346390593F60602638A0620834698
:102A50003905A18AEDFE97F0FF1FE780C0632A8C3D
:102A600097F0FF1FE7802063E30C85FF835609057D
:102A700011664255D18E2318D90497000000E780D3
:102A800060638346390513063905A18AFDDAF336FA
:102A9000048093F68608B6D401000100930680FAFC
:102AA00023809D002380DD00010001008346060095
:102AB00093F6F60D2300D60023800D00A656F3A64C
:102AC0000680010001008356090503462905D24707
:102AD000B376DA003306CA021305800C9355F6412B
:102AE0003696330DF6408257333CD6002E9C333653
:102AF000A601330CFC40330CCC40330885039256BE
:102B00004E86B335A5033305A503C29597C00100D2
:102B1000E78080B763468001631E0C16630C0D16B8
:102B2000130615003335A6002E959356F5013696FB
:102B3000B335D600AA959396F50105828585D18E89
:102B40006346B000639D051A638B061A0356C902DB
:102B500015823305D6003336C500B2956348B00000
:102B6000639105241306F00F637DA622894663F363
:102B7000561593078008F3B7078093F78708BED6EA
:102B80000100010037170040930770052300F70488
:102B9000930780FA2300F704010001008356C7025F
:102BA00089678117D58FC207C1832316F7022300D7
:102BB0000704B657F3A7078001000100FA506A54D2
:102BC000DA544A59BA592A5A9A5A0A5BFA4B6A4C49
:102BD000DA4C4A4DBA4D296182801308F5FF33352E
:102BE000A800FD152E951356F5013298B336C8008E
:102BF000AA9695B9F336048093F68608B6CA010002
:102C0000010023809D002380AD0001000100834668
:102C10003905CD8EA309D90423800D00D646F3A62D
:102C200006800100010035B3F336048093F6860870
:102C3000B6CE0100010023809D002380CD0001005D
:102C400001008346390593E60602A309D9042380CF
:102C50000D00F646F3A606800100010095B3F33699
:102C6000048093F68608B6D20100010023809D00FF
:102C70002380CD00010001008346390593E606025A
:102C8000A309D90423800D009656F3A606800100FF
:102C9000010045BB9306F5FF33B5A600FD152E9543
:102CA0009355F501AE96B3B5B600AA951396F50106
:102CB000858269B5F336048093F68608B6D801009C
:102CC0000100930680FA23809D002380DD0001002F
:102CD00001008356C9020566011693F6F60FD18EE0
:102CE000C206C1822316D90223800D00C656F3A660
:102CF000068001000100850A93FAFA0F95B233E6C7
:102D0000B60045C20356C9023305D0403338A0008F
:102D1000B305B040B385054115826345B000D1E1EC
:102D20006371A608894663F0560593078008F3B7D8
:102D3000078093F78708BEDA01000100B71700404B
:102D4000130770052380E704130780FA2380E70444
:102D50000100010003D7C7027D8B2396E702238081
:102D60000704D65781BDF336048093F68608B6DC97
:102D700001000100930680FA23809D002380DD007E
:102D8000010001008356C9020566011693F6F60F8D
:102D9000D18EC206C1822316D90223800D00E656C9
:102DA000B9B793078008F3B7078093F78708BEDEAB
:102DB0000100010037170040930770052300F70456
:102DC000930780FA2300F704010001000356C702AD
:102DD00093975600B297C207C1832316F7022300C8
:102DE0000704F657C1BB914763EEB70217D701003E
:102DF0001307C7268A05BA959C41BA978287B717E9
:102E0000004003A7470B1345F5FF698F23AAE70A84
:102E100003A7070B698F23A8E70A03A7070A798D81
:102E200023A0A70A8280B717004083A6470B134749
:102E3000F5FFF98E23AAD70A83A6070B558D23A881
:102E4000A70A83A6070A758F23A0E70A8280B7170F
:102E5000004003A7470B498F23AAE70A03A7070BE4
:102E60001345F5FF45BFB717004083A6470B13472F
:102E7000F5FF758F23AAE70A03A7070A598D4DB7F7
:102E8000B717004003A7470B498FEDB7914763EE93
:102E9000B70217D701001307A71D8A05BA959C41F1
:102EA000BA978287B717004003A7470D1345F5FF70
:102EB000698F23AAE70C03A7070D698F23A8E70CE6
:102EC00003A7070C798D23A0A70C8280B7170040B9
:102ED00083A6470D1347F5FFF98E23AAD70C83A6C7
:102EE000070D558D23A8A70C83A6070C758F23A06B
:102EF000E70C8280B717004003A7470D498F23AA2C
:102F0000E70C03A7070D1345F5FF45BFB7170040B2
:102F100083A6470D1347F5FF758F23AAE70C03A778
:102F2000070C598D4DB7B717004003A7470D498FC0
:102F3000EDB7797122D43714004026D24AD0035914
:102F400024028354040206D64209C2044ECE52CC57
:102F500056CA13590901C1802DE11379F9F793F489
:102F6000F49F4209C20413590901C18093078008E4
:102F7000F3B7078093F787083EC401000100930769
:102F800070052300F404930780FA2300F404010081
:102F90000100231124032310940223000404A247F8
:102FA000F3A7078001000100B25022549254025945
:102FB000F249624AD24A45618280B7F507008146EC
:102FC0003000B105194597000020E7808081A247B5
:102FD00013972701E34A07FC1369090893E40440A7
:102FE00093098008F3B7098093F787083EC0010072
:102FF0000100930A700523005405130A80FA230088
:10300000440501000100231124032310940223002E
:1030100004048247F3A7078001000100294597F0C7
:10302000FF1FE7802031F3B9098093F989084EC268
:1030300001000100230054052300440501000100A4
:103040008357040293E707202310F40223000404AB
:103050009247B9B7B7170040884742054181937737
:10306000050491EB9377F5013755E80113050580C9
:103070003345F50282809377050C130700046397AC
:10308000E7009377F50137459C1CCDB72165130503
:1030900005D0828037E700E01C435443A183E20659
:1030A000D58F1CC1FD572320F7182322F7188280E3
:1030B00013178500B7E700E023A0E710618123A282
:1030C000A7108280B7F700E08847CC47828081470D
:1030D00037370040A14663C4C7003285828003456C
:1030E000B740E38EA6FE3385F5000345050085074E
:1030F0002304A740CDB797070020938727EF9C4371
:10310000173700201307071C3E95636EE50017373D
:1031100000201307274F6368A70017070020232705
:10312000A7EC3E858280FD57EDBF8280411122C40D
:1031300006C62A8497000000E78000F22947B307FB
:10314000E502B2408D83B3D7870222449507B3D7F7
:10315000E70237370040C207C1832316F700410159
:103160008280411137150E0006C697000000E780E7
:1031700020FCB7370040130770F82381E7000D47A4
:10318000A381E70013070004A380E7000547238716
:10319000E700B24041018280373700408347270073
:1031A0001A0593F7F703C98F93F7F70F2301F70079
:1031B0008280B737004003C7170019C9D98DA38093
:1031C000B70003C70700136787002380E7008280EA
:1031D00093C5F5FFF98DA380B7008280AE872A875B
:1031E000B736004021463738004089E71703000012
:1031F0006700E3F383C8B600E30916FF05078348B9
:10320000F7FFFD17C20723041801C183F9BF41115D
:1032100022C406C62A8497000000E780E0E329471D
:10322000B307E502B2408D83B3D7870222449507E6
:10323000B3D7E70237370040C207C1832316F740F0
:1032400041018280716541111305052006C6970072
:103250000000E78000FCB7370040130770F82381B7
:10326000E7400D47A381E74013070004A380E74030
:1032700005472387E740B24041018280CC4141119C
:1032800006C6328503C6150083C5050022064D8E8D
:1032900042068D654186138875A2630C0611634B47
:1032A000C804138845A26300060D634AC8009385CD
:1032B00035A26301B6082390060029464DA0138865
:1032C00055A26305060D938565A2E316B6FE8D45EE
:1032D0001D4663E6E5081146198E63F3C7003E8676
:1032E000B7E704002390C600FC4797D501009385FB
:1032F00065DA9DA0138895A263030611634E060D3F
:103300001388A5A263000613938505A5E315B6FAF5
:1033100099451D4663E5E504198E63F3C7003E86B3
:10332000B7E704002390C600FC479705002093856B
:1033300025D61DA09D451D4663E3E5022146198E55
:1033400063F3C7003E86B7E70400FC472390C6003E
:103350009705002093858534BA9582970146B2403F
:10336000328541018280AD451D46E3EAE5FE3146E6
:10337000198E63F3C7003E86B7E704002390C600AA
:10338000FC4797D50100938565D3F9B7B1451D4634
:10339000E3E7E5FC3546198E63F3C7003E86B7E7E1
:1033A00004002390C600FC4797D50100938505D201
:1033B00065B78D451D46E3E4E5FA1146198E63F3C2
:1033C000C7003E86B7E704002390C600FC4797D5A8
:1033D00001009385E5CC49B78D451D46E3E1E5F84D
:1033E0001146198E63F3C7003E86B7E704002390A9
:1033F000C600FC4797D50100938505CFB1BFA54511
:103400001D46E3EEE5F42946198E63F3C7003E86B8
:10341000B7E704002390C600FC4797D501009385C9
:10342000E5C81DBFB5451D46E3EBE5F23946198EEB
:1034300063F3C7003E86B7E704002390C600FC474D
:1034400097D50100938505C401BFB7E7040003A326
:103450000713970600209386A6C24146A545170587
:1034600000201305E5B802832D455DE703C505007F
:103470000947631FE50803A84500411106C6034735
:10348000180032850346080022074168518F9308CF
:1034900028FE6307170563E9E800051863030703BF
:1034A00023900600294591A8130648FE630AC70425
:1034B0001518E31707FF15463E87637BF60015478F
:1034C00001A8130600023E876374F600130700028A
:1034D000B7E704002390E600FC471316070111A884
:1034E0003E8691C30546B7E70400FC472390C6001B
:1034F0004206CC45418282970145B240410182801B
:10350000130600083E87E375F6FC13070008C9B7E9
:103510002390060005458280828041677917630405
:10352000E504411122C406C685472A84639FF5003D
:10353000B7E7040022852244B24003A3871397050E
:1035400000209385E52F4101028389476399F500A7
:10355000B7E7040083A7070B8545829771D9B2406E
:103560002244410182808280797126D252CCAE847D
:103570002A8A97D50100938525B917D5010013052F
:1035800025BB06D63AC622D44AD0368432894ECEDE
:1035900097B00100E780805AA28517D50100130576
:1035A00025BA97B00100E7806059294597B001001E
:1035B000E780A05D83C7840093F70702F9E383C91E
:1035C00004008947054532476396F908D44083C70C
:1035D000160083C60600A207D58FC166138616FEA5
:1035E000638CC7028D16638FD7068D6693862690EF
:1035F00029456391D706B7E70400A286225403A3A6
:103600004714B250F2494A86A6850259925452850F
:10361000624A8547456102832D450DEF93070002FD
:10362000354563E98702B7E70400FC47C844130641
:103630000002CA8582978149970700209387072156
:103640009C43014581CB9C4391C74E852286CA8508
:1036500082970145B250225492540259F249624A6B
:10366000456182802D457DF79307700F3545E3E373
:1036700087FEB7E70400FC47C8442286CA858297C4
:1036800065BF2145C1BF411122C437E4040083272F
:10369000841326C2AA84416506C697050020938537
:1036A000251A7D1582978327C40A17050000130584
:1036B00005E78588829795C0032304132244B2400E
:1036C000924497060020938626AE4146C5451705CD
:1036D00000201305659C41010283B24022449244BC
:1036E00001454101828019C59707002023A0A71634
:1036F00001458280454582801147636AA70A97D6B3
:1037000001009386269F0A0536951841411106C689
:103710003697AE87B2850287130700026145639D25
:10372000E700B7E70400FC47130600021705002076
:10373000130545F782970145B24041018280054754
:103740006145E39BE7FEB7E70400FC470546170524
:103750000020130525F7F9BF1307700F6145E39D9E
:10376000E7FCB7E70400FC471306700F17050020BD
:10377000130585F5C1B7130700086145E39EE7FA15
:10378000B7E70400FC4713060008170500201305DF
:1037900025034DB715476145E390E7FAB7E7040005
:1037A000FC471546170500201305C50961B70945F3
:1037B0008280411126C2B7E4040083A7C41322C447
:1037C0004AC006C62E8497050020938565072A897E
:1037D0008297058905C5970700209387E78B83D7D4
:1037E000A70BA28503A3440D2310F4002244B2408A
:1037F00092444A850249014641010283B240224473
:103800009244024949454101828097070020238163
:1038100007049707002023AF0702B717004003A74C
:10382000070CB706C0FFFD16758F23A0E70C03A792
:10383000070DB7064000558F23A8E70C03A7070C18
:103840003D9B23A0E70C03A7070D1367070123A8DF
:10385000E70C8280B717004003A5470C83A7470CED
:10386000598113451500C18B058999E3136525001E
:103870009707002083C7C7FD6380A7029707002032
:103880002388A7FC11C9970700209387A7FC03A3EF
:1038900007006303030002838280114517F3FFFFD3
:1038A000670063C8411193962500AA852D4506C679
:1038B00097F0FF1FE780E0F2B240014541018280AE
:1038C000011122CC06CE3714004026CA4AC84EC683
:1038D00052C483447405034AB405834984050349EB
:1038E000940597F0FFFFE780E09E8347A40593F4DB
:1038F000F40F137AFA0F93E71700230DF40493F9EA
:10390000F90F1379F90FB717004003C7A705058B07
:103910006DFF03D5C705A38D4705238C3705A38C01
:103920002705A38B9704F2406244D2444249B2492E
:10393000224A0561828041119397050122C406C67F
:1039400026C2C1872E8463DC0700B7E40400FC5460
:10395000829719C1BC5482972165218D15A893F7D0
:10396000150013C515008DE793F725009DC7970037
:103970000000E78060EEB7E70400BC4F1306000AC2
:10398000894517050020034565ED829713452400FE
:10399000B24022449244410182809397250163D82A
:1039A0000702B7E4040083A7C41E829797000000B3
:1039B000E780E0EEBC4C37560700130606308965F9
:1039C00017050020034585E98297096579B7939724
:1039D00015010145E3DE07FA17C501001305457E11
:1039E00097B00100E780602DB7E70400BC4F1306D5
:1039F0000064916517050020034545E6829711652F
:103A0000A9BF2D71232A9110FD74E98C232C8110FC
:103A100023282111232631112A84AE893289930665
:103A200000100A86A6852D45232E111097F0FF1F42
:103A3000E78020DB13154401B7E70400FC47518100
:103A40000A0513962900CA850A958297A685856678
:103A50000146254597F0FF1FE780A0D80A86A68576
:103A600093060010294597F0FF1FE78080D7832039
:103A7000C1110324811183244111032901118329D8
:103A8000C11015618280B7F7070003C70701411114
:103A900006C622C426C24AC0A547631DF700970088
:103AA0000000E78040F6B2402244924402490145BA
:103AB0004101828013942500AA843289A286AA85B6
:103AC0000146254597F0FF1FE780A0D1A2864A86D0
:103AD000A685294597F0FF1FE780A0D0E9B71D71A3
:103AE000A2CC37E404005C5C485886CE494697C5B2
:103AF000010093856568829711E917C501001305D8
:103B0000E56897B00100E780401B01A0B7F600E030
:103B1000795798CAFD57DCCA0567B7E700E023A0CC
:103B2000E7101306F00290C223A0E718010001007D
:103B30003707002018471306000481459706002028
:103B400023ACE6D04157A38AE7403C44080882975B
:103B5000970700209387876D3EC8856713870740C6
:103B6000231AE1001D673ACC370701051307071038
:103B70003ACE938757D11307B00F2310E1022312D7
:103B8000F102054797F7FFFF938707542301E102EE
:103B90003ED817070000130727D197070000938727
:103BA00067D2B7F50700BAC23EDC1707000013075B
:103BB000C7ED97070000938787CE81463000E10567
:103BC0001945BAC43EDE97F0FF1FE78080C1180890
:103BD0008147994630003E96034606008507050753
:103BE000A30BC700E398D7FEC24791C70357410113
:103BF00085676373F70001A0B7E7040083A7470A4E
:103C000008088297AA8511C917C5010013054559EF
:103C100097B00100E78080F201A0F640664425617C
:103C20008280411126C2B7E4040083A7040806C6B7
:103C300022C417050000130545D082971704002001
:103C40001304C4C12300A40097000000E780800291
:103C500097000000E780A0BB03450400224403A3B3
:103C60008405B24092441306003289654101028303
:103C7000797106D622D413078008F337078093F7AB
:103C800087083EC201000100B71700409305700588
:103C90002380B704130680FA2380C70401000100C3
:103CA00083C6F70293F6A60FA387D70223800704E3
:103CB0009246F3A606800100010073370780137750
:103CC00087083AC4010001002380B7042380C70499
:103CD0000100010003C7F70213672700A387E7026B
:103CE00023800704A247F3A70780010001000545D0
:103CF00097E0FFFFE780406197000000E78020BA6F
:103D0000014781468147054685451305407E97E07A
:103D1000FFFFE780406437E404003C4468005146FC
:103D200081458297B707C0A83EC8B787E803938745
:103D300007D03ECA97E7FF1F938767683EC67C5847
:103D400068008297B250225445618280411197D514
:103D50000100938525AD17C501001305653D06C615
:103D600097B00100E78080DD17D50100130545C439
:103D700097B00100E78080DCB2402945410117B3CC
:103D80000100670083E0411197D501009385C5AA22
:103D900017C501001305C53906C697B00100E780B5
:103DA000E0D917D50100130565BF97B00100E78082
:103DB000E0D8B2402945410117B301006700E3DCB8
:103DC000411122C406C6834705002A849DC797D5A2
:103DD0000100938525AC17C501001305653597B023
:103DE0000100E780A0D54C4017D50100130585CA16
:103DF00097B00100E78080D43DA058410DEF97D5E2
:103E00000100938525A917C501001305653297B0F8
:103E10000100E780A0D217D50100130525C997B08E
:103E20000100E780A0D12244B2402945410117B3E7
:103E30000100670083D5A1679386D7036313D70278
:103E400097D50100938505A517C501001305452EDB
:103E500097B00100E78080CE17D50100130505C695
:103E60007DBFED0797D501009385C5A217C5010059
:103E70001305052C631BF70097B00100E78000CC09
:103E800017D501001305C5C459BF97B00100E780DD
:103E9000E0CA4C4017D50100130585C591BF4111FB
:103EA00097D501009385859A17C50100130545280C
:103EB00006C697B00100E78060C8B24029454101BD
:103EC00017B30100670063CC797122D426D24AD09F
:103ED0002E842A898145B2844800714606D697E02F
:103EE000FFFFE780C02297F7FF1F9387E74CDC476F
:103EF00083D70700231421012313F10097500000FA
:103F0000E78040E29547A305F1009307401F3EC6B6
:103F1000FD572305A100230AF10097500000E78018
:103F2000A0F42686A285480097500000E78060E252
:103F3000B250225492540259456182809717002052
:103F40002399077E971700202382076EB7E70400A6
:103F5000BC47411106C6414681451705002013059F
:103F6000651B8297170700200347C71C9307F00AB9
:103F70006315F7029307F0F889451705002013052C
:103F8000651B170700202307F71A97070020A38354
:103F9000071A97600000E780409B97600000E78069
:103FA000A0C68145370504009707002023A2071605
:103FB00097070020239C07149707002023890714E4
:103FC000970700202398070C970700202396070ADD
:103FD00097070020239B07129707002023940714BC
:103FE00097300000E7804027014597600000E78098
:103FF000C09E97D501009385E58717C5010013057D
:10400000251397B00100E78060B317D501001305B1
:1040100065B497B00100E78060B2B2402945410124
:1040200017B30100670063B6411122C497D50100A0
:10403000938585872A8417C501001305650F06C679
:1040400097B00100E78080AF4C4017D50100130501
:10405000E5A197B00100E78060AE294597B0010067
:10406000E780A0B2034704009307F00F631FF70235
:1040700097D501009385458317C501001305450BAE
:1040800097B00100E78080AB4C4017D501001305C5
:10409000E59E97B00100E78060AA2244B24029451E
:1040A000410117B30100670043AEB2402244410111
:1040B0008280411122C426C22A84AE8417C5010021
:1040C0001305050797C501009385C57906C697B006
:1040D0000100E780A0A617D50100130525A697B01B
:1040E0000100E780A0A5294597B00100E780E0A97D
:1040F00097C501009385057797070020239C87F6D5
:1041000017C501001305C502054497070020239138
:1041100097F697070020239E87F497170020239A8D
:10412000976097B00100E78060A19715002083D5C4
:10413000456017D501001305E5A097B00100E780A1
:10414000E09F294597B00100E78020A49717002041
:10415000238E874C97F7FF1F93870726DC4703D7EB
:104160000700C167FD176312F7022244B7E7040096
:10417000B240924403A3870517F5FF1F0345856EE0
:104180001306000A854541010283B240224492444D
:1041900041018280B1C1411122C417C5010013053C
:1041A00025F92E8497C501009385056B06C697B047
:1041B0000100E780A098A28517D501001305459757
:1041C00097B00100E78080972244B2402945410121
:1041D00017B301006700639B8280011122CC06CED9
:1041E00026CA4AC84EC693F715002E84638A071262
:1041F000814617F6FF1F130666198545170500202F
:10420000035545E797C00000E780000515C997C52D
:1042100001009385E56617C50100130565F197B0A8
:104220000100E780A09117C501001305250897B08C
:104230000100E780A090294597B00100E780E09455
:1042400097C501009385C56317C50100130545EEA9
:1042500097B00100E780808E17C501001305450661
:1042600097B00100E780808D294597B00100E78075
:10427000C09197F7FF1F93872714DC47054797C521
:1042800001009385E55F2390E70017C50100130542
:1042900025EA97B00100E780608A17C50100130581
:1042A000650397B00100E7806089294597B0010058
:1042B000E780A08D930710F817070020230CF7E67E
:1042C0009707002083D7C7DA17070020A304F7E673
:1042D0009145A183170500201305C5E517070020A8
:1042E000230BF7E497070020A38707E4975000000B
:1042F000E780A065B7E70400BC4F0D6613060620F3
:104300009305001017F5FF1F0345C5558297134508
:104310001400F2406244D2444249B24905618280AD
:1043200093F705108DC7054597500000E780E06AB8
:10433000171500200355E53F97500000E7804036F1
:1043400097200000E780400713450410D9B793F782
:104350002500E9CF17070020035747DB69C7AD6485
:10436000B71900409384A4AA23A0990097060020BF
:10437000938606DA944297C701009387A77F1706B2
:1043800000200346C6D8814517050020130585D8AF
:1043900097700000E780A00B23A0990097F7FF1FFC
:1043A0002390A7F22A8941C197C50100938505543E
:1043B00017C501001305C5D797A00100E780007855
:1043C000CA8517C50100130565F297A00100E780B3
:1043D000E076294597A00100E780207B9707002021
:1043E000239607D2930710F8170700202304F7D469
:1043F0009707002083D7C7C717070020A30CF7D261
:10440000A183170700202308F7D291458D47170590
:104410000020130525D217070020A30EF7D09750D0
:104420000000E780805213452400E5B593F745006E
:10443000D1C397C501009385654B17C501001305CE
:1044400025CF97A00100E780606F17C50100130515
:10445000A5EB97A00100E780606E294597A00100B9
:10446000E780A072930720F8170700202304F7CCF9
:104470009707002083D707C217070020A30CF7CAAD
:10448000A183170700202308F7CA854717070020D4
:10449000A303F7CA97500000E780009D170500208E
:1044A000130545C9914597500000E780004A134520
:1044B000440085B593F78500A9C797C5010093858A
:1044C000E54217C501001305A5C697A00100E780C6
:1044D000E06617C50100130565E497A00100E780B9
:1044E000E065294597A00100E780206A9707002032
:1044F000239E07C097700000E780400513458400A5
:1045000009BD93F70501D1C3854517050020035563
:1045100065B897600100E78060B797C50100938593
:10452000E53C17C501001305A5C097A00100E78071
:10453000E06017C501001305A5DF97A00100E78023
:10454000E05F294597A00100E7802064930730F8D9
:10455000170700202300F7BE9707002083D787B3F3
:1045600017070020A308F7BC17050020130585BC1A
:10457000A1838D4517070020230FF7BA975000003D
:10458000E780A03C1345040169B393F70502D1C746
:1045900097C501009385853517C50100130545B9F9
:1045A00097A00100E780805917C50100130585DA3F
:1045B00097A00100E7808058294597A00100E78077
:1045C000C05C930740F8170700202305F7B697074C
:1045D000002083D767AA17070020A30DF7B4A18393
:1045E000170700202309F7B4854717070020A30405
:1045F000F7B497070020239107A897500000E780A1
:10460000A086170500201305E5B2914597500000DC
:10461000E780A03313450402EDB993F70504FDC309
:1046200097C501009385852C17C50100130545B07A
:1046300097A00100E780805017C50100130505D33E
:1046400097A00100E780804F294597A00100E780EF
:10465000C0539707002083C7E7AD1307700A63862E
:10466000E7061307800A638CE7081307600A639361
:10467000E704930760F817070020230DF7AA9707B0
:10468000002083D787A817070020A305F7AAA183D6
:10469000170700202301F7AA854717070020A3006A
:1046A000F7AAB145170500201305C5A897500000CB
:1046B000E780A02997400000E780007B13450404B1
:1046C00097070020239307A4A9B1930770F8170751
:1046D00000202301F7A69707002083D707A3170719
:1046E0000020A309F7A4A183170700202305F7A43E
:1046F000854717070020A301F7A4994565B79307DD
:1047000080F8F1B793F705080145E38407C097C522
:1047100001009385A51D17C50100130565A197A08C
:104720000100E780A04117C501001305A5C597A0AA
:104730000100E780A040294597A00100E780E04400
:104740009307A0F8170700202306F79E970700207D
:1047500083D7479D17070020A30EF79CA183170757
:104760000020230AF79C854717070020A305F79C24
:10477000970700202398079A97400000E780C06EB3
:10478000170500201305059B914597500000E78011
:10479000C01B13450408B5BE011122CC37E4040048
:1047A0005C5C06CE354697C501009385A52117D5DB
:1047B0000100130525EC829711E917C501001305C7
:1047C000E59C97A00100E780404F01A097F7FF1FED
:1047D0009387070A3EC4B7F507008567938707806C
:1047E000814617F6FF1F13062608E10519453EC648
:1047F00097E0FF1FE780E0FE7C44194697F5FF1F16
:1048000093858506170500201305058982973400D6
:1048100017F6FF1F1306460597C501009385056827
:1048200017C501001305056997700000E780209700
:104830002A841DCD97C501009385450A17C501003F
:104840001305058F97A00100E780402FA28517C5AB
:1048500001001305251897A00100E780202E2945A7
:1048600097A00100E7806032F240624405618280D7
:1048700097E00000E78080F917C501001305850C5B
:1048800097600000E780608B97A00000E780C04D34
:1048900097600100E78040B217F5FF1F130545AE92
:1048A00097600100E780E09A17C501001305850AAB
:1048B00097600100E780C0B22A8497600000E7801B
:1048C000A0F197100100E780208A97800100E7801F
:1048D000402397700000E780E04997600000E78080
:1048E000A06797300100E780804B97C50100938552
:1048F000E5FE17C501001305A58319C897A001009F
:10490000E780C023A28517C501001305E50EA1B7F6
:1049100097A00100E780802217C50100130505104C
:1049200097A00100E7808021294597A00100E7803A
:10493000C02597300100E780602797F00000E780EE
:10494000204655C985453705040097300000E780AB
:10495000A09097C50100938565F817B50100130570
:10496000257D97A00100E780601D17C50100130594
:10497000650C97A00100E780601C294597A0010005
:10498000E780A02097F7FF1F9387879283D70700C0
:1049900017170020231FF7D8854717170020230774
:1049A000F7C897200000E780E0B497200000E78078
:1049B000A0A0171500200355C5D797500000E78029
:1049C00020CE054597500000E780200197C50100E3
:1049D0009385C5F017B501001305857597A00100F3
:1049E000E780C01517C501001305050797A0010052
:1049F000E780C014ADB597C50100938525EE17B5C6
:104A000001001305E57297A00100E780201317C588
:104A100001001305251497A00100E7802012294505
:104A200097A00100E7806016014569BF411122C4CB
:104A300037E404008327041A06C6829797500000C3
:104A4000E780C0C98327040817F5FFFF1305257900
:104A5000829797F7FF1F2387A7E017F5FF1F13051E
:104A6000A59597400000E780C0722244B240410102
:104A700017030000670083D2B7E70400FC471171F9
:104A8000A2DDCAD986DFA6DBCED72E8432892E8658
:104A9000AA8517F5FF1F1305E569829717F7FF1F12
:104AA0001307476983470700930680029387E70748
:104AB00093F7F70FE3ECF610BA898A0717B70100EE
:104AC00013074770BA979C43BA9782878D4797C55B
:104AD00001009385E5E217B5010013056565630FD5
:104AE000F40097A00100E780600517C501001305D9
:104AF000E59F97A00100E7806004BDA497A0010096
:104B0000E780C00317C501001305C59F97A00100EA
:104B1000E780C002294597A00100E78000079307BE
:104B200020F8114697F5FF1F9385C5604A8517F752
:104B3000FF1F2301F76097F7FF1FA38E075E97F013
:104B4000FFFFE780A0382A841DC997C5010093851F
:104B500025DB17B501001305A55D97A00100E780CF
:104B6000E0FDA28517C501001305859D97A00100F2
:104B7000E780C0FC294597A00100E780000197C5A8
:104B800001009385E5D717B501001305655A97A075
:104B90000100E780A0FA17C501001305A59B97A0A7
:104BA0000100E780A0F9294597A00100E780E0FD1A
:104BB0004165930730FA054697F5FF1F93858557A2
:104BC0007D1517F7FF1F2307F75697F0FFFFE780C4
:104BD000E02F2A841DC997C50100938565D217B5BA
:104BE00001001305E55497A00100E78020F5A28598
:104BF00017C501001305C59497A00100E78000F4D4
:104C0000294597A00100E78040F8B7E70400BC4FB2
:104C10000566130606C8A14517F5FF1F034585C4A1
:104C20008297FE506E54DE544E59BE5911618280F7
:104C300091476303F40297C50100938565CC17B5CE
:104C400001001305E54E97A00100E78020EF17C58E
:104C500001001305659371BDB7E70400FC4F914552
:104C600017F5FF1F034505C0829797C5010093857F
:104C700025C917B501001305A54B97A00100E780D2
:104C8000E0EB17C501001305E59197A00100E7804F
:104C9000E0EA294597A00100E78020EF9740000057
:104CA000E780801C914535A485476303F40297C5CE
:104CB00001009385E5C417B501001305654797A06A
:104CC0000100E780A0E717C501001305258F15B582
:104CD00097F7FF1F2390273DB7E704000566BC4FF9
:104CE000130606C8C1450DBF8D476303F40297C57F
:104CF00001009385E5C017B501001305654397A032
:104D00000100E780A0E317C501001305E58CD5B3CA
:104D1000930740F8114697F5FF1F9385A5414A85F3
:104D200017F7FF1F2308F74097F7FF1FA3850740DA
:104D300097F0FFFFE78080192A84E30405EE97C50A
:104D400001009385E5BB17B501001305653E97A0EB
:104D50000100E780A0DEA28517B501001305457E9E
:104D600097A00100E78080DD294597A00100E7803A
:104D7000C0E145BD9147E31CF4F6B7E70400FC4FE2
:104D80009305000217F5FF1F0345C5AD829797C530
:104D900001009385E5B617B501001305653997A0A5
:104DA0000100E780A0D917C5010013056584F1BD96
:104DB000894763E3870297C50100938565B417B5FA
:104DC00001001305E53697A00100E78020D717C53D
:104DD00001001305258331BB97F4FF1F83C4A4355D
:104DE00097F7FF1F83C7173597C50100938545B116
:104DF000A20417B501001305A533DD8C97A00100AF
:104E0000E780C0D3A28517C501001305E58097A0F0
:104E10000100E780A0D2C204294597A00100E780E5
:104E2000C0D6C1849305D4FF93960401C1824A86FB
:104E300093F5F50F17F5FF1F1305F52F97200000C9
:104E4000E7804045E35F90DC930750F817F7FF1FBA
:104E50002302F72E83C73900228697F5FF1F93851B
:104E6000652D85074A8517F7FF1FA306F72C97F0D6
:104E7000FFFFE780A0052A84E30505DA97C5010056
:104E8000938505A817B501001305852A97A0010091
:104E9000E780C0CAA28517C50100130565C8C9B55A
:104EA000894763E3870297C50100938565A517B518
:104EB00001001305E52797A00100E78020C817B57A
:104EC00001001305257735B197400000E780C0F950
:104ED000A28517F5FF1F1305E52597500000E78011
:104EE000C0A681B38D476303F40297C50100938583
:104EF00025A117B501001305A52397A00100E780A0
:104F0000E0C317B501001305A574E5B6B766020046
:104F10000146B7750200054597E0FF1FE780608CEA
:104F2000930760F817F7FF1F2306F72097F7FF1F77
:104F3000A38307209307000617F7FF1F230EF71E12
:104F4000894717F7FF1FA309F71E97F7FF1F23864F
:104F5000071E97F7FF1FA382071EC14717F7FF1F02
:104F6000230EF71C930720F917F7FF1FA308F71C60
:104F7000314697F7FF1FA384A71C97F5FF1F938562
:104F8000651B4A8597F7FF1F238B071A97F0FFFFD2
:104F9000E780C0F32A84E30605C897C5010093851E
:104FA000259617B501001305A51897A00100E78005
:104FB000E0B8A28517B501001305056B55B3B147DD
:104FC0006303F40297C501009385859317B501002B
:104FD0001305051697A00100E78040B617B501003C
:104FE0001305456A39B6B7E70400FC4F9305000482
:104FF00017F5FF1F03450587829797400000E7805C
:10500000A0E6B145F9B5914763E3870297C5010072
:105010009385058F17B501001305851197A0010031
:10502000E780C0B117B5010013058567D9B497F4BF
:10503000FF1F83C4641097F7FF1F83C7D70FA20415
:10504000DD8C8E04B77702006D14BE942286A6858F
:1050500017B501001305056697A00100E78000AEB3
:10506000B7E70400FC47228697F5FF1F9385D50C10
:105070002800829793160401C1823000A685094555
:1050800097D0FF1FE780E0752A8409C917B5010092
:105090001305056497A00100E78020C2930770F80C
:1050A000194697F5FF1F9385E5084A8517F7FF1FF7
:1050B0002302F70897F7FF1FA380870897F0FFFFE9
:1050C000E780C0E02A84E30E05B497C5010093850C
:1050D000258317B501001305A50597A00100E780FA
:1050E000E0A5A28517B501001305855F95B999471D
:1050F000630BF41297C501009385858017B50100F5
:105100001305050397A00100E78040A317B5010030
:105110001305855EF9BA914763E3870297B50100ED
:105120009385057E17B501001305850097A0010042
:10513000E780C0A017B501001305855D5DBA97F43F
:10514000FF1F83C464FF97F7FF1F83C7D7FEA20426
:10515000DD8C8E04B77702006D14BE942286A6857E
:1051600017B501001305055C97A00100E780009DBD
:10517000B7E70400FC47228697F5FF1F9385D5FB10
:105180002800829793160401C1823000A6850D4540
:1051900097D0FF1FE780E0642A8409C917B5010092
:1051A0001305055A97A00100E78020B1930780F806
:1051B000194697F5FF1F9385E5F74A8517F7FF1FF7
:1051C000230AF7F697F7FF1FA38887F697F0FFFFEC
:1051D000E780C0CF2A84E30605A497B50100938534
:1051E000257217B501001305A5F497A00100E7800B
:1051F000E094A28517B501001305C55595B69947EA
:105200006303F40297B501009385856F17B501001C
:10521000130505F297A00100E780409217B5010041
:105220001305C554F9B0B7E70400FC4F930500041B
:1052300017E5FF1F03450563829797400000E7804D
:10524000A0C2994579B18D476303F40297B5010077
:105250009385056B17B50100130585ED97A0010037
:10526000E780C08D17B501001305C55159B017B5BA
:1052700001001305255297A00100E78000A4130543
:10528000C01297D0FF1FE780C00B014597E0FFFFDA
:10529000E78080E00D4597100000E780E09F2945FA
:1052A00097D0FF1FE780E00997D0FF1FE78040FA03
:1052B0008DBA99476303F40297B50100938545645D
:1052C00017B501001305C5E697A00100E780008728
:1052D00017B501001305C54C29B817F7FF1F034781
:1052E000B7E597F7FF1F83C727E522075D8F916614
:1052F000BA96C2061166C1821306F6EF8D47636542
:10530000D60297E7FF1F9387270B9C4B17F6FF1FCB
:10531000034676E29386C7002DC203D6070069CA0A
:105320008907E39CD7FE89471307A0F8114697F534
:10533000FF1F938525E04A8597F6FF1F238CE6DE45
:1053400017F7FF1FA309F7DE97F0FFFFE78000B80C
:105350002A84E308058C97B501009385655A17B533
:1053600001001305E5DC97900100E780207DA28510
:1053700017B5010013050544E5B203D60700630E17
:10538000E60A8907E39BF6FE8D4779BF91476304E0
:10539000F40297B501009385A55617B501001305D2
:1053A00025D997900100E780607917B501001305B2
:1053B000E5416FF00FF4B7E70400FC4F93050008D8
:1053C00017E5FF1F0345054A8297C9B897B5010045
:1053D0009385055317B50100130585D597900100F6
:1053E000E780C07517B501001305C53F6FF06FF07A
:1053F0002390E70017E5FF1F130505FC9730010018
:10540000E78040A097B501009385854F17B501004F
:10541000130505D297900100E780407217B501008F
:105420001305453D97900100E7804071294597900D
:105430000100E78080758147C5BD2390070017E50F
:10544000FF1F130565F797300100E780A09B97B514
:1054500001009385E54A17B50100130565CD9790C6
:105460000100E780A06D17B501001305253A5DBF67
:10547000411122C406C6834705002A849DC797B5FB
:1054800001009385A54317B50100130565CA9790E0
:105490000100E780A06A4C4017B501001305856E36
:1054A00097900100E7808069E1A05841B707CF00DD
:1054B0009387777D631DF70697B5010093850540B7
:1054C00017B501001305C5C697900100E780006776
:1054D0001C448356E4008355C40003C6070017B577
:1054E00001001305A56B97900100E7802065294511
:1054F00097900100E78060690357E4009707002058
:1055000083D727236309F7008355C400084497E035
:10551000FFFFE780E0CC0356E4008355C400084455
:105520002244B240410117F3FFFF67002355B7073C
:10553000CC009387777D6315F70497B501009385B9
:10554000E53717B501001305A5BE97900100E78068
:10555000E05E1C448356E4008355C40003C6070084
:1055600017B501001305856397900100E780005D82
:105570002244B24029454101179301006700E360CE
:10558000B707CE009387777D6304F70297B50100D4
:105590009385C53217B50100130585B997900100B1
:1055A000E780C0594C4017B5010013056554CDBDC7
:1055B000B240224441018280B7E70400FC47411118
:1055C0002E8606C622C426C24AC02E842A89AA85EF
:1055D00017F5FF1F130505B6829797B50100938550
:1055E000E53317B501001305A5B497900100E780D6
:1055F000E05497F5FF1F83C5E5B317B50100130508
:10560000E5D997900100E780605329459790010004
:10561000E780A05797F4FF1F9384C4B183C70400A9
:1056200041479387070693F7F70F636EF75A17B74B
:105630000100130767C38A07BA979C43BA9782870A
:105640009D476307F40297B501009385252D17B593
:1056500001001305E5AD97900100E780204E17B5D6
:105660000100130525D497900100E780204D8DA4FB
:1056700097F7FF1F83C717ACDDCB17F7FF1F034753
:1056800097AB97F7FF1F83C707AB22075D8F97F78D
:10569000FF1F83C767AAC2075D8F97F7FF1F83C7E6
:1056A000B7A9E207D98F17F7FF1F2323F7A683C7F0
:1056B000640097B501009385652617B501001305B1
:1056C00025A717F7FF1F2304F7A497900100E78091
:1056D000E04697F7FF1F9387A7A38C4317F6FF1F9A
:1056E0000346E6A217B50100130585CD979001008A
:1056F000E780C044294597900100E780004997F76B
:10570000FF1FA38907A22244B24092440249930793
:1057100000F817F7FF1F230FF7A09D4517F5FF1F90
:10572000130545A14101174300006700032297605C
:105730000000E78020F197F7FF1F238EA79E935765
:10574000850017F7FF1FA308F79E935705012A84CA
:1057500017F7FF1F2302F79E93578501014517F79F
:10576000FF1FA30BF79C97600000E78060EE97F7A0
:10577000FF1F2384A79C97B501009385251A17B5B1
:1057800001001305E59A97900100E780203B17F68A
:10579000FF1F0346869AA28517B501001305C5C3EE
:1057A000B1B7CD476303F40297B5010093850517A0
:1057B00017B501001305C59797900100E7800038E1
:1057C00017B501001305C5C279BD37E404007C4458
:1057D000414697F5FF1F9385F59517F5FF1F1305B4
:1057E0006593829797F7FF1F83C7E79517F7FF1F0A
:1057F00003475795A20703238405D98F17F7FF1F87
:105800002316F7901306000A89452244B2409244B9
:10581000024917E5FF1F0345E504410102838D4757
:105820006303F40297B501009385450F17B5010096
:105830001305059097900100E780403017B50100EF
:105840001305C5CA0DB517F4FF1F0344C48E97F79F
:10585000FF1F83C7378E97B501009385250C22045F
:1058600017B501001305C58C5D8C97900100E7808A
:10587000E02CA28517B50100130505B9979001002A
:10588000E780C02B294597900100E78000300D4646
:1058900097F5FF1F9385058A228597E0FFFFE78034
:1058A000E062AA8421C197B501009385250717B549
:1058B00001001305E58797900100E7802028A68561
:1058C00017B50100130585B597900100E780002703
:1058D0002244B240924402492945410117930100F4
:1058E0006700A32A97E7FF1F2396877AB7E704008C
:1058F000116603A38705130606E8914539B78D475E
:105900006303F40297B501009385450117B50100C3
:105910001305058297900100E780402217B501002A
:10592000130585CB89B317F4FF1F0344C48097F791
:10593000FF1F83C7378097B50100938525FE22049A
:1059400017A501001305C57E5D8C97900100E780C7
:10595000E01EA28517B50100130585AD97900100E3
:10596000E780C01D294597900100E78000220D4681
:1059700097E5FF1F9385057C228597E0FFFFE78071
:10598000E054AA841DC197B50100938525F917A598
:1059900001001305E57997900100E780201AA6859C
:1059A00017B50100130505AA05B797E7FF1F239553
:1059B000876CB7E70400116603A38705130606E8A2
:1059C0009305000299B5894763E3870297B5010003
:1059D0009385C5F417A501001305857597900100FF
:1059E000E780C01517B501001305C5C1ADB997E42F
:1059F000FF1F83C4447497E7FF1F83C7B77397B52E
:105A000001009385A5F1A20417A5010013054572B5
:105A1000DD8C97900100E7806012A68517B5010024
:105A20001305C5A397900100E78040112945979081
:105A30000100E7808015228697E5FF1F9385856F1B
:105A4000268597E0FFFFE78060482A84630E051AE9
:105A500097B50100938585EC17A501001305456DE9
:105A600097900100E780800DA28517B5010013050E
:105A700025A099BD854763F98718834519002244FD
:105A8000B24092440249B335B00097E7FF1F238D1F
:105A9000B76017B501001305E59E4101179301009A
:105AA0006700C309A2852244B24092444A85024954
:105AB0004101170300006700632499476303F40260
:105AC00097B50100938585E517A501001305456687
:105AD00097900100E780800617B50100130545CCBB
:105AE00059B617E4FF1F0344046597E7FF1F83C7F8
:105AF000776497B50100938565E2220417A501003C
:105B0000130505635D8C97900100E7802003A28553
:105B100017B501001305859897900100E7800002F2
:105B2000294597900100E7804006194697E5FF1F39
:105B300093854560228597E0FFFFE7802039AA849E
:105B40001DC197B50100938565DD17A501001305FB
:105B5000255E97900100E78060FEA68517B50100DD
:105B60001305C59495B397E7FF1F239D875AB7E7A1
:105B70000400116603A38705130606E893050008D1
:105B800069B1854797B50100938545D917A50100EF
:105B90001305055A630BF40097900100E78000FAA3
:105BA00017B501001305C5917DBC97900100E780F2
:105BB000E0F817B501001305259297900100E780E2
:105BC000E0F7294597900100E78020FC2244B2408D
:105BD0009244024997E7FF1F239A07524101176336
:105BE00000006700A39697B50100938525D317A5FC
:105BF00001001305E55397900100E78020F417B5E5
:105C00000100130525BE85B4B240224492440249E6
:105C100041018280411106C622C497E0FFFFE78060
:105C2000E02A21CD97E7FF1F83D7274885072A84DD
:105C300017E7FF1F231BF74697B50100938585CF14
:105C400097E7FF1F2394A74617A501001305454EAC
:105C500097900100E78080EEA28517B5010013053B
:105C600025EC97900100E78060ED2244B240294581
:105C7000410117930100670043F197E7FF1F83D7A6
:105C80000743B2402244850717E7FF1F2311F7425D
:105C900041018280411122C491462A8417E6FF1FE8
:105CA000130646579D652D4506C697D0FF1FE78012
:105CB00040B3B7F7070003C70701A5476313F70011
:105CC00001A09306001001469D65254597D0FF1F52
:105CD000E78020B197E7FF1F238E87522244B2400E
:105CE000914617E6FF1F1306E6529D6529454101BF
:105CF00017D3FF1F6700E3AE1171CED7B7E90400D9
:105D000083A7C904CAD917E9FF1F1309A942A2DD55
:105D10002E8686DFA6DB2E84AA854A85829797E7A2
:105D2000FF1F83C727411307700A6385E710636D60
:105D3000F7001307600A6385E704FE506E54DE54D3
:105D40004E59BE59116182801307800A6385E71698
:105D50001307900AE393E7FE8D476306F41C97B59B
:105D60000100938525EF17A501001305653C979069
:105D70000100E780A0DC17B501001305E5EA25A0C6
:105D80008D47630CF40297B501009385A5EC17A528
:105D900001001305E53997900100E78020DA17B577
:105DA00001001305A5E197900100E78020D929455E
:105DB00097900100E78060DD49B7854717B501007E
:105DC000130585E117E7FF1F2300F72E97900100C9
:105DD000E780A0EEB7750200B766020001460545F0
:105DE00097D0FF1FE780E09F930760F817E7FF1F3A
:105DF0002302F73497E7FF1FA38F0732930700268C
:105E000017E7FF1F232AF732E5779387072117E764
:105E1000FF1F2315F732B14597E7FF1F2381073294
:105E200097E7FF1FA38DA7304A8597000000E78002
:105E3000E01621B7914763E3870297B50100938588
:105E400065E117A501001305A52E97900100E780D5
:105E5000E0CE17B50100130525DAB1B797E4FF1FAF
:105E600083C4842D97E7FF1F83C7F72CA204DD8C22
:105E700083A7C9046D14228697E5FF1F9385D52B50
:105E8000280082978E0493160401B7750200C18220
:105E90003000A695094597D0FF1FE78080949307AF
:105EA00070F817E7FF1F2307F728994597E7FF1FAB
:105EB000A384A72895BF914763E3870297B50100A4
:105EC000938545D917A501001305852697900100F4
:105ED000E780C0C617B50100130585D3E9B597E47F
:105EE000FF1F83C4642597E7FF1F83C7D724A2043D
:105EF000DD8C83A7C9046D14228697E5FF1F938567
:105F0000B523280082978E0493160401B77502000A
:105F1000C1823000A6950D4597D0FF1FE780608CA9
:105F2000930780F8BDBF17B50100130525D19790E1
:105F30000100E78080D8930790F82304F10083479D
:105F400019008D452800A304F1008347290023058B
:105F5000F10097000000E78060041305C01297C0AD
:105F6000FF1FE780003E014597D0FFFFE780C0128A
:105F70000D4597000000E78020D2294597C0FF1FFC
:105F8000E780203C97C0FF1FE780802C7DB397E718
:105F9000FF1F23A9A728828097E7FF1F93878728E1
:105FA00003A3070063030300028317430000670095
:105FB000C39941114AC097F6FF1F83D6867732896D
:105FC00017D6FF1F0356664122C426C206C62A847E
:105FD000AE8497000000E780205D35C12DC0994751
:105FE00063FF97048347140003470400A207D98F77
:105FF00013978700A183D98FC2073167C183130725
:10600000C755639EE70297D7FF1F83D7073DA301BC
:10601000F400A1832302F40097F7FF1F83D7677171
:1060200091C7A302F400A1832303F400A68517B54A
:106030000100130525C697900100E78020B097F76F
:10604000FF1F83C7A75EB9CF97D5FF1F83D5E5385C
:1060500017B501001305C5C597900100E78000AE94
:106060002686A28517D5FF1F035525379700000008
:10607000E78080BA6301090497E7FF1F83C7C71A47
:106080009DCB95C897E7FF1F83C707028DE7228541
:106090002244B2400249A6859244410117430000C0
:1060A0006700A38A17B50100130585C19790010009
:1060B000E780A0C0C1B7B2402244924402494101E6
:1060C0008280834755008345450017B501001305BD
:1060D00025BBA207DD8D17930100670023A617B526
:1060E00001001305E5B817930100670003BD8D4754
:1060F00063FBB70A011126CA06CE22CC0344350041
:1061000097E4FF1F83C4541297B50100938505BC23
:10611000B337800017E7FF1FA308F71009C497B52E
:106120000100938565BB17B50100130565BB97900A
:106130000100E780A0A097E7FF1F83C7F70E6386E3
:10614000970097000000E780E02E97E7FF1F83C7C6
:10615000B70D8DC785472306F100B7E7040083A775
:1061600047177000854513055030829717B5010019
:10617000130505B897900100E78020B499679387CD
:1061800057EE2316F100680085479145A30781006B
:106190002307F10097000000E78040E0F2406244EE
:1061A000D244056182808280894763F7B708011174
:1061B00022CC06CE26CA8344250085472A84639DC7
:1061C000F404914763F5B704034545008347340061
:1061D00022055D8D97D7FF1F2391A7209700000010
:1061E000E78060459967938767EE2314F100834742
:1061F000340023059100A305F10083474400954531
:1062000028002306F10097000000E78020D9F24023
:106210006244D24405618280FDF89967938767EEF6
:106220002314F10097D7FF1F83D7271BA305F10085
:1062300023050100A183E1B782800111996722CC77
:10624000D51717F4FF1F1304643E2314F10083478E
:10625000040026CA97F4FF1F9384A44D2305F10080
:1062600083D7040028009545A305F100A18306CE3D
:106270002306F10097000000E78040D203D6040017
:106280008345040017B50100130505A89790010088
:10629000E780C08AF2406244D244056182809D67F3
:1062A0007971D9172316F10097F7FF1F83C70738B5
:1062B00006D62307F100A9C3B7E70400FC4741460F
:1062C00097E5FF1F938505E51305F10082976800A8
:1062D000CD4597000000E78060CC97F5FF1F83C590
:1062E000E53417B50100130525A597900100E78057
:1062F000E084B25045618280B7E70400BC47414664
:1063000081451305F1008297D9B745C5411106C6ED
:1063100022C4930750FA2300F5009307A005A300B9
:10632000F50089472301F5009147A301F500930784
:106330006003A302F50097F7FF1F9387272F83C7FA
:106340000700230205002A842303F50097E7FF1FB7
:10635000938797ED83C70700414697E5FF1F938515
:1063600065DBA303F50097F7FF1F83D7873C230462
:10637000F500A183A304F50097D7FF1F83D7E70596
:106380002305F500A183A305F500B7E70400FC474A
:10639000310582972285F14597000000E780C01CF7
:1063A000230EA4002181A30EA400B2402244410187
:1063B000828082805D710A8586C6A2C49700000033
:1063C000E780E0F437E404007C448A8508107946CD
:1063D00082973C441305E1030946814582971010DA
:1063E00093050002014597D0FFFFE7802031B640BA
:1063F000264461618280411122C426C24AC02A8497
:10640000AE843289AA8585660146254506C697C0B1
:10641000FF1FE780003DA2852244B240CA8626863F
:10642000024992442945410117C3FF1F6700633B9E
:106430000111B7C7A55A22CC9387C73317E4FF1FB2
:10644000130494DE3EC4834704002C0021461965E2
:1064500006CE3EC697000000E78020FA8345040080
:1064600017B501001305459C97800100E780006D7A
:10647000F2406244056182800111A14630009965B5
:106480002D4522CC06CE97C0FF1FE7808035A2475E
:1064900037C4A55A1304C43363958702B24517B5B0
:1064A00001001305A58BB335B00097E7FF1FA38D3F
:1064B000B7D697800100E7806068F24062440561CA
:1064C00082809165A1463000938505F02D4597C0E7
:1064D000FF1FE7800031A247E38287FC97E7FF1F99
:1064E000A38407D4814517B5010013056589D1B789
:1064F0007971D146700091652D4522D406D697C09A
:10650000FF1FE780002EB24737C4A55A1304F435A5
:1065100063988702B7E70400FC4717E5FF1F1305E0
:1065200065BF41460C08829717B501001305458BDE
:1065300097800100E7806078B250225445618280E4
:106540009165D1467000938505E82D4597C0FF1FE2
:10655000E7802029B247E38F87FA17B501001305BA
:10656000258AF9B7C16769768146FD170506139735
:10657000060141836364B7003E8582803307D500FE
:1065800003470700B98F214713F817008583630578
:106590000800B18FC207C1837D171377F70F6DF71E
:1065A0008506F1B741C5A547054763F2B70883479C
:1065B0001500034705003168A207D98F139787009C
:1065C000A183D98FC207C1831308C85505476390BB
:1065D0000707411106C622C426C20344250091477D
:1065E00063F087049307540063ECF502A301C50030
:1065F00021822302C5009304340091C6A302D50072
:10660000A1822303D5002A84A68597000000E78095
:10661000A0F526942300A4002181A300A400014733
:10662000B240224492443A854101828005473A852E
:1066300082800111B7C7A55A22CC9387E7342A84F8
:106640002AC621462C00156506CE3EC497000000E0
:10665000E780A0DAA28517A501001305E57E9780E3
:106660000100E780A04D97000000E780E0D4F240F1
:106670006244056182800111A146300095652D4577
:1066800022CC06CE97C0FF1FE780A015A24737C4D3
:10669000A55A1304E43463958702B24517A5010097
:1066A0001305057097D7FF1F2399B7D2C205C18183
:1066B00097800100E7808048F24062440561828053
:1066C0009165A1463000938505EE2D4597C0FF1FCB
:1066D000E7802011A247E38287FCD14717D7FF1F2D
:1066E000231DF7CED14517A501001305656DC9B768
:1066F00021C1411126C206C622C4AE848DC52A849A
:1067000097000000E780806697E7FF1F83C7C7B147
:1067100099CB22852244B240A68592444101173389
:10672000000067008322B2402244924441018280EB
:10673000828001114AC806CE22CC26CA4EC693F7E3
:1067400015002E899DCBAD67371700409387A7AA08
:106750001CC3B7E70400BC4F13060019854517D5C5
:10676000FF1F034565C7829713451900F240624435
:10677000D2444249B2490561828093F72500638A79
:10678000071C17F7FF1F0357A7FA954763F9E70C94
:10679000014417F6FF1F1306A6E9930630051305FB
:1067A0005004130810049308B004130390059307D2
:1067B00064006374F7043A84FD5997F4FF1F83C49F
:1067C00024E797F7FF1F83C7B7E6A204DD8CAD6708
:1067D0009387B755638BF41463E3970AA96793878C
:1067E000A755638EF414A28517F5FF1F130545E422
:1067F00097000000E78000F031A2B307860083C550
:106800000700639AD50483C517006396A50483C562
:1068100027006392050583C53700639ED50283C5B3
:106820004700639A150383C7570063966702A289DE
:106830000DE897F5FF1F83D5A5EFB3853541C20558
:1068400017F5FF1F1305C5DEC1814E9597000000A7
:10685000E78040EAE1A005044204418089BF3A8410
:10686000FD598547E3EB87F45DC4854517F5FF1FA8
:10687000130505DC97000000E780C0E769A8B16751
:106880009387C7556380F404B5679387D755E39C16
:10689000F4F4A28517F5FF1F130585D99730000082
:1068A000E780A00A8947630FF4049305E4FFC2055B
:1068B000C18117F5FF1F1305C5D797000000E780BA
:1068C000E04A89A097200000E780C0F79700000009
:1068D000E780204911C9A28517F5FF1F130545D58B
:1068E00097000000E78080480546A28517F5FF1F46
:1068F000130505D497F0FFFFE780E06B97200000B9
:10690000E78040F4A68517A501001305A5559780DB
:106910000100E780A022FD57E39DF9F097F7FF1FE4
:10692000239807E01345290091B5A28517F5FF1FAD
:10693000130505D097F0FFFFE780E078E1B7A28567
:1069400017F5FF1F1305C5CE97F0FFFFE7806079AD
:1069500055BF93F745000145E38A07E017A50100FD
:106960001305855197800100E7802035973000009E
:10697000E780402B13454900D5BB411122C437E4C1
:1069800004005C5C06C6354697A501009385850327
:1069900017B50100130505CE829711E917A501006F
:1069A0001305454E97800100E780203101A0832721
:1069B000041C82972A84054597C00000E78060E4A4
:1069C00097600100E780806997600100E780803E62
:1069D00097B00000E780E0F52285B24022444101F3
:1069E00082804111054506C622C426C297C0FFFF1A
:1069F000E78060541305A00497B0FF1FE780206B69
:106A0000757585457D1597C0FFFFE780003E7D7554
:106A100085451305F53697C0FFFFE78060473714BB
:106A200000408327840A8D451305002093E7072043
:106A30002324F40A97C0FFFFE780203BB7E404005B
:106A400097D0FFFFE7804080C85897800100E7801B
:106A5000C02617B501001305E5C197800100E78046
:106A6000C0258327840C8545414593E707082324E7
:106A7000F40C97C0FFFFE780A0418D451305000887
:106A800097C0FFFFE780C04097C0FFFFE780A06D81
:106A900037A507001305051297C0FFFFE78040697F
:106AA000014597C0FFFFE780606F95450545894721
:106AB00017F7FF1F2300F7C897C0FFFFE780A06FFD
:106AC000B7E700E013070006238DE740370700040F
:106AD00023A0E71097D0FFFFE780A00097D0FFFF2B
:106AE000E780601497000000E78060E997000000ED
:106AF000E780C09897000000E78020B897E0FFFF8C
:106B0000E78000F397000000E780802797000000EF
:106B1000E780801083A70408170500001305A5C1AE
:106B2000829797D7FF1F2389A78ABC4C130600645E
:106B30008545829797C0FF1FE780808B0145828043
:106B4000AD67371700409387A7AA1CC3B7E700E0DB
:106B50003707400023A0E71801000100B7F707003E
:106B600003C70701A5476316F7009397450191C333
:106B700001A04111AE860146AA85254506C697C0EB
:106B8000FF1FE78000C6B240B7E700E037074000CC
:106B900023A0E710410182804111B2862E86AA858A
:106BA0002D4506C697C0FF1FE780A0C3B240014530
:106BB000410182809307000463ECC7041D71A2CCDD
:106BC0002A840808A6CACAC886CE32C697800100A1
:106BD000E78060EBAD67371700409387A7AA1CC317
:106BE000B7E400E03709400023A0241901000100A8
:106BF000B2461008A285294597C0FF1FE78060BEF6
:106C0000F640664423A02411D6444649256182807B
:106C10003955828041110D658D4506C697C0FFFF2D
:106C2000E780A01CB71700408D6623A6D70A17F58A
:106C3000FF1F130565B01387C70A9387870A1CC116
:106C40005CC5856689675CC958C114C518C9B7E7B2
:106C50000400B24003A3871E410102838145B307AC
:106C6000B5008387070089E717230000670023C466
:106C70008505C205C181E5B797A701009387873ACB
:106C80001357C5003E9703470700011106CE2304A2
:106C9000E100135785003D8B3E970347070023060D
:106CA0000100A304E100135745003D8B3D893E9749
:106CB000AA970347070083C7070028002305E100C0
:106CC000A305F10097000000E78080F9F24005611C
:106CD0008280411126C2E97797F4FF1F938444B65E
:106CE00022C49387A7552E842381B4002E86AA85BB
:106CF00017F5FF1F130505B506C62390F400A38101
:106D0000040097800100E78000D893052400C205A5
:106D1000C18117F5FF1F1305C5B297000000E7807A
:106D2000A084B38784002382A7002181A382A700C7
:106D3000930564002244B24026859244C205C18175
:106D4000410117230000670083B609C99307800239
:106D500063E6B700170300006700E3F7828017F5CA
:106D6000FF1F0345E59E828097F7FF1F83C707AD8E
:106D700089E717230000670083B3828097F7FF1F1E
:106D800083C7E7AE99EF411106C697200000E78060
:106D9000E0A9B240854717F7FF1F230AF7AC41016E
:106DA000828082806307054A6385054A5D71CAC097
:106DB0004EDE86C6A2C4A6C252DC56DA5AD85ED6C9
:106DC00062D466D26AD0B9472A89AE8963F9B70618
:106DD000394697A501009385A51297800100E780A9
:106DE00020C831ED8347E900130710036394E702DD
:106DF000854717F7FF1F2303F7A417A50100130505
:106E0000251197F7FF1F239A07A297000000E7803C
:106E100020E571A01307000317A501001305451213
:106E2000E395E7FE97F7FF1F238A07A097F7FF1F59
:106E3000239507A017A501001305050FF9B797F7CC
:106E4000FF1F83C7A79F63870722BD6AB96B938C17
:106E5000FA55014A17FBFF1F130BCB8F138CEB6501
:106E6000938AFA6605A8B307490183C6070097F716
:106E7000FF1F83D7879CB1E39307A005639BF600B0
:106E8000854717F7FF1F231AF79A97F7FF1F2383EA
:106E9000D78C050A93170A01C183E3E637FDB64094
:106EA000264496440649F259625AD25A425BB25B72
:106EB000225C925C025D61618280054D639BA70349
:106EC0009307500A639EF600894717F7FF1F2316A2
:106ED000F796930750FA17F7FF1FA30DF78655BFD4
:106EE0009307A005E387F6FA97F7FF1F2397079408
:106EF0004DB7138717004207DA9741832380D700E5
:106F000017F6FF1F231BE6928D47E3F4E7F817F40B
:106F1000FF1F0344548497F7FF1F83C7C7832204CE
:106F20005D8C9307F4FFC207C1839306F00DE3ED78
:106F3000F6FA93076400C207C183E31CF7F49305D4
:106F40002400C205C18117F5FF1F1305C58097F006
:106F5000FFFFE780606133078B00834757000347DB
:106F60004700A207D98F17F7FF1F2318078C631854
:106F7000F50E8144630CA40197E4FF1F83C4C47D14
:106F8000A20497E7FF1F83C7377DDD8C170500003C
:106F90001305E5DB97F0FFFFE780A0FF6387840719
:106FA000636D9C029387EB556382F40497E7FF1FA0
:106FB00083C7877A05476389E70681CB1387A705CF
:106FC0001377F70F8D4663F2E6081307F0072300E7
:106FD000E100A300F10089459DA063829405E39739
:106FE00054FD97F0FFFFE780C02B11A8A28517E59D
:106FF000FF1F1305657697F0FFFFE780800F0145BF
:1070000097F0FFFFE780E0F869B5A28517E5FF1F5D
:107010001305857497F0FFFFE7804019CDB797F00F
:10702000FFFFE780C021E1BF930710F813051100AF
:107030002300F10097F0FFFFE780602DFD450A85F2
:1070400097000000E78020C95DBFA28517E5FF1FFC
:107050001305857097F0FFFFE78040CA4DB793078F
:10706000F00789450A852310F10097000000E780AA
:1070700080C605B5BD4763F83717414697A501009F
:10708000938545EE4A8597800100E780609D631CEB
:10709000051417A50100130525EE97000000E780F1
:1070A00020BC17E5FF1F0355C56897000000E78067
:1070B000E0BC97E7FF1F83C7675717A501001305BB
:1070C00025E389E717A50100130505E397000000F4
:1070D000E78000B917A50100130585EB97000000B4
:1070E000E78000B817C5FF1F0355C52C97000000A7
:1070F000E780C0B817A501001305C5E99700000097
:10710000E78000B617C5FF1F0355252D9700000027
:10711000E780C0B617A50100130545E897000000F9
:10712000E78000B417D5FF1F035565F897000000EE
:10713000E780C0B417A501001305C5E6970000005D
:10714000E78000B217D5FF1F035525F69700000012
:10715000E780C0B217A50100130545E597000000C0
:10716000E78000B017D5FF1F035545F497000000D6
:10717000E780C0B017A50100130585E39700000064
:10718000E78000AE17C5FF1F035585139700000069
:10719000E780C0AE17A50100130505E297000000C7
:1071A000E78000AC97D7FF1F83C7C7F6A20717D5A4
:1071B000FF1F034535F65D8D97000000E78000ACAA
:1071C00097D7FF1F83C727F5A20717D5FF1F0345D2
:1071D00095F45D8D97000000E78040AA17950100A7
:1071E0001305C5551DB1C14763FE3705414697A537
:1071F00001009385A5DC4A8597800100E7804086E1
:1072000031E18347090113071003639CE7008547B9
:1072100017E7FF1F230EF75217A50100130545DBE3
:10722000EDB61307000317A50100130565DDE39E06
:10723000E7BC97E7FF1F238D075017A50100130533
:10724000A5DAE1B6CE854A8597C0FFFFE78040F911
:10725000B9B18280411126C2AE848D4522C406C6D2
:107260002A8497C0FFFFE780A0C2B717004099C8E3
:1072700003A5C70C418D23A6A70CB240224492441B
:107280004101828003A5870C418D23A4A70CF5B78B
:107290008347050003471500A207D98FC20761770E
:1072A000C18713072720639AE70083452500370528
:1072B000040017030000670023FA828017E6FF1F0F
:1072C0001306465B8147B2861303F00FA9483308C3
:1072D000F6000348080013F7F70F6307A80C6306CE
:1072E00068008507E39517FF2947B387E6002380E9
:1072F000A70097E7FF1F9387A7585DA8411113D7F1
:1073000065001347170006C693F63500058B9547B1
:1073100091CA054699476387C60009469D4763831E
:10732000C600A14713F645003336C00093F6850327
:10733000050685C2A145638BB604E145638AB604A0
:10734000930580026388B604930580036393B600B7
:10735000914697E5FF1F238AF57897E5FF1F238560
:10736000C57897E5FF1FA381D578BE8517A50100D5
:10737000130545CF97700100E780407CB2408547F8
:1073800017E7FF1FA303F776410182808546D1B737
:107390008946C1B78D4675BF17A50100130505CFF6
:1073A000177301006700837917E7FF1F1307474D25
:1073B000BA972380B700E147E302F5F49307700220
:1073C000E30CF5FC82802A8723800500814717E5BE
:1073D000FF1F1305254A1308F00F2946B306F500D1
:1073E00083C606006396E60297E6FF1F938646492A
:1073F000B69783C7070005452380F5009947636E5C
:10740000F7029D4763FDE700E147630DF7008280C7
:10741000638506018507E393C7FC0145C5B7238053
:1074200005008280B737004003C7370083C70500D7
:1074300093F70704D98F2380F50082805D7152DCB9
:1074400056DA5ED6716A97EBFF1F938B2B7B8D6AA2
:10745000A6C24EDE62D486C6A2C4CAC05AD866D2BC
:107460006AD06ECEC1495E8C97E4FF1F93840442BC
:10747000130A0A20938A7ADC17E9FF1F0349097B64
:10748000B3872B0183C7070093F7F70FC9EFB787BF
:10749000004003C76700058BE310077C03C7670044
:1074A000118BE30D077E83C75700918B99E36F1013
:1074B000200317E7FF1F0347877785476304F7001B
:1074C0006F10400197E7FF1FA381E76297E7FF1F57
:1074D000238E074697E7FF1F238C075297E7FF1F6E
:1074E000238A075E97E7FF1F2387075E97E7FF1F43
:1074F000A38E074497E7FF1FA38C075097E7FF1F52
:10750000A38A075C97E7FF1FA387075C97E7FF1F26
:10751000A38E075C97E7FF1FA38B0770B787004018
:1075200011476F0070779307190093F7F70F3D47E6
:107530006364F70617E7FF1F230AF76E97E7FF1F3D
:107540009387C76DCA9783C707001307100293F785
:10755000F703638EE71E6366F70405446385871CA3
:10756000E38C07620947638EE71013070002E38488
:10757000E74EB7E700E03707400023A0E718010017
:107580000100629923000900FD1923A0E71093F977
:10759000F90FE39309EEE5BD97E7FF1F238807681E
:1075A00071BF130730026388E70C63E8E71613071F
:1075B0004002638CE70A13070003E39CE7FA97E7AE
:1075C000FF1F9387A764CA9703C70700A1471377D4
:1075D000F70FE31BF71483C7640097E6FF1F238DA3
:1075E000F64E97E7FF1F83C7D72A91C7FD5797E647
:1075F000FF1F2383F64E97E5FF1F83C5352997E7C5
:10760000FF1FA38BB74C97E7FF1F83C7272813FBE8
:1076100007089306000493F70706639FD74C930768
:10762000A009638DF51663EAB7129307F005638628
:10763000F54A930750096384F52A014497E7FF1F31
:1076400083C797491547E392E736B7E700E0370766
:10765000400023A0E71801000100B7860040238006
:107660008602130680FC6F00500EFD5717E7FF1FC0
:107670002303F746FDBDFD5717E7FF1F230CF74413
:10768000CDBD17A501001305E5B197700100E78096
:10769000C06297E7FF1F93876757CA9703C4070025
:1076A000014B97ECFF1F938CEC361374F40F17AD5E
:1076B0000100130DADAF63478B042945977001009E
:1076C000E780A04C854717E7FF1FA303F73417E7B0
:1076D000FF1F2300873417E7FF1F2309F74037E711
:1076E00000E0B70640002320D718010001003786CC
:1076F00000408347A60293F7370F2305F6022320A5
:10770000D71085BDB3876C0183C507006A85050B5B
:1077100097700100E780804279BF854717E7FF1F18
:107720002308F72EB9B517E7FF1F1307274E4A970F
:107730000347070097E6FF1FA38AF62097E6FF1F7F
:107740002387E62017E7FF1F2302F73A1DB5854779
:1077500017E7FF1F230CF71E29BD9307400A638913
:10776000F5349307200B6384F5369307100AE396EC
:10777000F5EC838724000144E3D207EC97E7FF1F71
:1077800083C7F71093F63700638A061A0546638AA3
:10779000C62209466395C61A1D4755A217E5FF1F65
:1077A0000345E50EC94797ECFF1F83CC5C0E97E5B8
:1077B000FF1F83C5E50D17E4FF1F0344740D631518
:1077C000F510CD476392FC1093077008639CF50297
:1077D0001307300FB7170E006308E4001307900D6E
:1077E000B7B704006314E40817E7FF1F232CF72E34
:1077F000BE8517A501001305E59B97700100E78082
:10780000E03325BD93078008639DF500B3078040F2
:1078100013F4F70FB7774600938787CDB3D7870266
:10782000E1B793079008639AF500B307804013F41B
:10783000F70F91679387C766D5B79307A008639B37
:10784000F500B307804013F4F70FB7173D00938797
:107850000790E9B79307B008639AF500B307804033
:1078600013F4F70F9167938797D04DBF93F5F50702
:107870008D47639BF500B307804013F4F70FB7976C
:107880005B00938707D859BF8947639BF500B3070F
:10789000804013F4F70FB7770B009387071BBDBF2A
:1078A0008547639AF500B307804013F4F70FDD674F
:1078B000938767E3A5B7D28785F9B307804093F72D
:1078C000F70FB3D7FA020DB797000000E780409F8B
:1078D000A285668597000000E780809EB9BB93056E
:1078E000610017E5FF1F034585FA17E4FF1F0344F6
:1078F00014FA97000000E78040AD930571002285DF
:1079000097000000E78060AC3C0017E7FF1F2325CD
:10791000F72E834761002304F10083477100A3041D
:10792000F100894717E7FF1F2308F71A83578100E3
:1079300017E7FF1F231CF7F4094409B3154793F613
:107940004700B336D00093F78703850685C32146E9
:10795000638BC7066146638AC70613068002638885
:10796000C706130680036393C700914717E6FF1FFE
:10797000230CD61697E6FF1FA388F61697E7FF1F7E
:107980002385E71617E7FF1F034787F09376070461
:1079900097E7FF1F83C7D7EF8DEE1377770C93061A
:1079A0007008630CD7021377F7078D466312D70C64
:1079B000B307F040B7955B0093F7F70F938505D8B1
:1079C00049A81947ADBF854755B7894745B78D4782
:1079D00071BF930670086311D7021307300FB715F4
:1079E0000E006389E7021307900DB7B504006383A7
:1079F000E7021307700845BF9306800C6311D70296
:107A0000B307F040B775460013F7F70F938785CD9E
:107A1000B3D5E70297E7FF1F23A6B70CD9BB9306A0
:107A2000900C631CD700B307F04093F5F70F9167F4
:107A30009387C766B3D5B702F1BF9306A00C631D49
:107A4000D700B307F040B7153D0093F7F70F9385C4
:107A50000590B3D5F5027DBF9306B00CE315D7F4BE
:107A6000B307F04093F5F70F9167938797D0D9B795
:107A70008946631BD700B307F040B7750B0093F737
:107A8000F70F9385051BF1B78546631AD700B30737
:107A9000F040DD6593F7F70F938565E35DBFD28511
:107AA00035FBB305F04093F5F50FB3D5BA029DB79A
:107AB00083C72400C18B99C7854717E7FF1F2300A1
:107AC000F702A5BE97E7FF1F238B0700BDB68547CA
:107AD00017E7FF1FA30BF7008DB63C0017E7FF1F4A
:107AE000232CF7100947930700032314F10097E6AE
:107AF000FF1F2383E6FE2DBD63940756A94763E568
:107B0000B74217970100130727538A05BA959C417E
:107B1000BA97828717E4FF1F034474D7894C630622
:107B2000940D63E68C0685476303F4089307F00F12
:107B300017E7FF1F034747FA63F6E70017E7FF1F42
:107B4000230CF7F897ECFF1F83CC0CF99307000484
:107B500013F4FC0F63F497011304000497E7FF1F6D
:107B60009387870903AD070022862685EA85B38CB3
:107B70008C40229D97700100E780E0F097E7FF1F9F
:107B8000238C97F597E7FF1F23A8A70745BC8D47D0
:107B9000630CF40A9947E31BF4F897970100938765
:107BA000275017E7FF1F2329F704A94751B717E705
:107BB000FF1F0347C70797E7FF1F9387E7F3494670
:107BC000979501009385C556630687009795010038
:107BD000938505523E8597700100E780C0EA17E75C
:107BE000FF1F232BA700C947A1B797E6FF1F83C636
:107BF0000604054797E7FF1F938707F06394E602A3
:107C00003E8513067002979501009385E54F9770A6
:107C10000100E78040E717E7FF1F232FA7FC93072A
:107C2000700239B73E85130630049795010093859D
:107C3000E54797700100E78000E517E7FF1F232D58
:107C4000A7FA93073004EDB597E5FF1F83C525C458
:107C5000179501001305455797700100E78000EE66
:107C6000054D97EDFF1F83CD8DFC97E5FF1F83C565
:107C700005C217950100130525556398AD0B977044
:107C80000100E780A0EB97E7FF1F83C747C0B5CB94
:107C9000E36EF4E8179401001304C44D638CB7013C
:107CA000179401001304844D638697011794010013
:107CB0001304444E228597700100E780400113753C
:107CC000F50F93071500860717E7FF1F2306F7E256
:107CD0008D4717E7FF1FA301F7E297E7FF1F938781
:107CE000A7E10147BE861376F70F89076365A602F1
:107CF00097E7FF1F23A2D7F097E7FF1F83C7C7DFD0
:107D000005BD979701009387E73F17E7FF1F2325DE
:107D1000F7EE914731BD3306E40003460600A38029
:107D2000070005072380C7007DBF97700100E7802B
:107D3000E0E097E7FF1F83C787B5E1D7E368F4DE8C
:107D40001794010013040440638CA70117940100E9
:107D50001304C43F63869701179401001304844001
:107D6000228597700100E78080F61375F50F930761
:107D70001500860717E7FF1F2300F7D88D4717E781
:107D8000FF1FA30BF7D697E7FF1F9387E7D601479F
:107D9000BE861376F70F8907E37CA6F43306E4006A
:107DA00003460600A380070005072380C700D5B758
:107DB00097E5FF1F83C5A5AD179501001305854104
:107DC00097700100E78080D797E7FF1F83C797D29E
:107DD00093E7470017E7FF1FA30EF7D083C72400E0
:107DE00017E7FF1FA306F7D089B817950100130501
:107DF000A53F97700100E78040EC97E7FF1F93874E
:107E000027CF83C7070017E7FF1F2301F7A817E451
:107E1000FF1F034464CC333480000DB0179501007C
:107E20001305C53D97700100E78020E997E7FF1F24
:107E300083C757CC93E7070117E7FF1FA30CF7CAC7
:107E400083C7240017E7FF1F2304F7CA6FF0EFFE74
:107E5000179501001305C53B97700100E780E0E529
:107E600003C704007D8B51EFB787004003C767024B
:107E70001377C70B136727002383E70203C7A70203
:107E80001377C70B136727002385E70203C7E702B1
:107E90001377C70B136727002387E70203C727035E
:107EA0001377C70B136727002389E702854717E776
:107EB000FF1F230DF7A817E7FF1F230BF7B417E7E2
:107EC000FF1F2309F7C017E7FF1F2306F7C097E737
:107ED000FF1FA38D07A697E7FF1FA38B07B297E7A6
:107EE000FF1FA38907BE97E7FF1FA38607BE97E77B
:107EF000FF1FA38D07BE97E7FF1FA38A07D26FF06E
:107F0000CFF389476312F70297E7FF1F83C74798AC
:107F10009146638CD70863E0F604638EE70C6369CF
:107F2000F70A05476380E70EFD5717E7FF1FA30514
:107F3000F7BA37074000B7E700E023A0E7180100D1
:107F40000100B78600401306F0FC2381C60223A07F
:107F5000E7106FF00FE2130720086382E7086362FF
:107F6000F70213071008E391E7FC378700408347C7
:107F7000670293F7C70B93E727002303F7026FF01D
:107F8000CFEB130730086389E70213074008E39D2E
:107F9000E7F8378700408347270393F7C70B93E73A
:107FA00027002309F7026FF04FE937870040834726
:107FB000270393F73707F5B7378700408347E70272
:107FC00093F7C70B93E727002307F7026FF0EFE65D
:107FD000378700408347E70293F73707F5B73787BE
:107FE00000408347A70293F7C70B93E727002305B9
:107FF000F7026FF08FE4378700408347A70293F7BB
:108000003707F5B7378700408347670293F737078D
:10801000ADB7179501001305A52097700100E78003
:10802000C0C997E7FF1F23830786D5B317950100C3
:108030001305052097700100E78020C897E7FF1F10
:108040002396078497E7FF1F938707A903C40700B8
:10805000894763F3870009441374F40F6FF00FDE50
:1080600013070002E392E7EC631B0B0A638FF50032
:10807000930720026383F508179501001305C51EB9
:1080800097700100E78080AB45B517950100130597
:10809000E51A97700100E78040C20144179D010076
:1080A000130D0D1BA14CB387840083C507006A859F
:1080B000050497700100E78060A8E31694FF178518
:1080C00001001305A56D97700100E78000BF17D46C
:1080D000FF1F0344E47B01E897D7FF1F238A07783B
:1080E000014B6FF0AFD58947E310F4E4854717D70C
:1080F000FF1F230FF7766FF04FD417D6FF1F0346ED
:10810000167997D5FF1F83C585781795010013054C
:10811000A51497700100E78060A26FF00FD2638012
:10812000F50693071002E399F5F497D5FF1F83C571
:108130002576179501001305251497700100E78037
:10814000E09F97E7FF1F23A997AA97E7FF1F938751
:108150006799944383D7470017E7FF1F0347E798C2
:1081600017D6FF1F2324D6721D4497D6FF1F2391D5
:10817000F67297D7FF1F238EE7706FF02FCC97D53D
:10818000FF1F83C5E57017950100130565109770F3
:108190000100E780A09A97D7FF1F238B076C97D722
:1081A000FF1F2395076E6FF02FF92547638FE7C8F0
:1081B0009946378700406394D70223008702B7E7C8
:1081C00000E0B706400023A0D71801000100130605
:1081D00000FC2301C70223A0D7106FF08FB99306CC
:1081E000100A639FD70023008702B7E700E0B706B5
:1081F000400023A0D71801000100130680FCD1BF66
:108200009306A009E381D7FE9306400AE38DD7FCCD
:1082100093062002639DD700B7E700E0B706400051
:1082200023A0D7180100010023008702F9B7854673
:10823000E384D7FE93070008E300FBFEB7E700E006
:10824000B706400023A0D71801000100130620FC48
:1082500023008702BDBF17E7FF1F0347F7876302AD
:10826000F71E63E7E70295476300F7109947630A33
:10827000F704B786004023800602B7E700E037071F
:10828000400023A0E718010001001306A0FC75B907
:108290009307F005630AF700930750096306F70098
:1082A00093071002E317F7FCB7E700E03707400039
:1082B00023A0E71801000100B7860040130620FC48
:1082C00069B117EBFF1F034B2B81930700045A8DF5
:1082D00063F46701130D000497E7FF1F9387C791AD
:1082E00083AC07001374FD0F2286E6852685976010
:1082F0000100E7804079B3078B40669417D7FF1FD2
:10830000230CF77C97E7FF1F23A8878EB7870040D1
:10831000630C0B022380A703B7E600E0370640009A
:1083200023A0C6180100010003C727021347070452
:108330002381E70203C727021377C70F2381E702D0
:1083400023A0C6106FF0EFA22380070237E700E0FA
:10835000B70640002320D71801000100130620FCB7
:108360002381C7026FF0AFB93787004083473700DA
:1083700097D6FF1F83C6D67793F70708D58FA3013B
:10838000F700B7064000B7E700E023A0D7180100C8
:1083900001001306A0FC35BD97E7FF1F93870787F1
:1083A000CA9783C7070093F7F70FC1CF97E7FF1F5F
:1083B00083C7E787D9E717D7FF1F0347F7719307ED
:1083C00000026310F70883AD040017DDFF1F034DA3
:1083D0002D4C97DCFF1F83CCBC4B17DBFF1F034BDF
:1083E0004B4BE6876A87DA866E8697D5FF1F83C573
:1083F000254817950100130525EB97600100E780DC
:10840000E07397D7FF1F23AFB76D97D7FF1F238D5B
:10841000A76D97D7FF1FA389976D97D7FF1F238657
:10842000676D97D7FF1FA3848744B7E700E037073E
:10843000400023A0E71801000100B78600406FF05C
:108440004FA2B7E700E03707400023A0E71801007C
:108450000100B786004015BD97D6FF1F83C6267D55
:108460000547639CE60429472381E70209472383E4
:10847000E7022385E70297D7FF1FA389076697D7EF
:10848000FF1FA386077AB7870040A381070017D78D
:10849000FF1FA30F076405472383E700B640264468
:1084A00096440649F259625AD25A425BB25B225C48
:1084B000925C025DF24D6161828029472381E7026F
:1084C00009472383E7022385E7022387E7022389FD
:1084D000E70255B717D7FF1FA30BF7386FE01FFF51
:1084E000854717D7FF1F2303F74617D7FF1F230121
:1084F000F75217D7FF1F230FF75C17D7FF1F230C67
:10850000F75C6FE0BFFE854717D7FF1F2300F744D6
:1085100017D7FF1F230EF74E17D7FF1F230CF75A4D
:1085200017D7FF1F2309F75A17D7FF1FA3000742CA
:1085300017D7FF1FA30E074C17D7FF1FA30C075811
:1085400097D7FF1FA38907588280411106C697005D
:108550000000E78080FBB7870040238007001307F7
:1085600040FC2386E7001307C004A386E70017D763
:10857000FF1F1307A7312398E70017D7FF1F130723
:10858000E734239AE70017D7FF1F13076740239CA0
:10859000E70017D7FF1F1307E74B239EE700294784
:1085A0002381E70209472383E7022385E702238724
:1085B000E7022389E702A3810700930600F8A3805E
:1085C000D700930690022380D700FD562383D7005F
:1085D0002381E7009306000537E700E0230BD7402F
:1085E000B70640002320D71003C7170013671700F2
:1085F000A380E700B24097D7FF1F239B074E41019E
:108600008280411106C697000000E78000F0B7871E
:10861000004023800700130700FC2386E700314752
:10862000A386E70017D7FF1F130747262398E70005
:1086300017D7FF1F13078729239AE70017D7FF1FB4
:1086400013070735239CE70029472381E7020947E1
:108650002383E7022385E702A3810700930600F83E
:10866000A380D700930690022380D700FD56238372
:10867000D7002381E7009306000537E700E0230BCE
:10868000D740B70640002320D71003C71700136751
:108690001700A380E700B24097D7FF1F239A074433
:1086A00041018280F1679387072017D7FF1F232B93
:1086B000F742854717D7FF1F2318F742A14717D75F
:1086C000FF1F2304F74297D7FF1FA380074297D7C6
:1086D000FF1F238D074097D7FF1F238B071897D7BE
:1086E000FF1FA3860718814717D5FF1F130585189D
:1086F000FD5517D6FF1F1306A6182947B306F50028
:108700002380B600B306F600238006008507E397B2
:10871000E7FE97D7FF1FA382073C97D7FF1FA380D1
:10872000073C97D7FF1F238B073A97D7FF1F238656
:10873000073A97D7FF1F2385073A97D7FF1FA38FC5
:10874000073897D7FF1F238C0738814717D6FF1F9D
:108750001306C64A4147B306F60023800600850784
:10876000E39BE7FE828017D7FF1F0347474C8547EF
:108770006316F700170300006700E3E81703000023
:108780006700E3DC411122C406C617D7FF1F034769
:10879000074A85472E8613F4F50FAA856317F70459
:1087A00017D5FF1F1305C52297600100E780A02D94
:1087B00097D7FF1F238E0724B787004023848702A3
:1087C000B7E600E03706400023A0C618010001000C
:1087D00003C7A7021377C70F2385E702B2402244DD
:1087E00023A0C61001454101828017D5FF1F130544
:1087F000E51197600100E780002997D7FF1F2387C5
:108800000714B787004023828702B7E600E03706E7
:10881000400023A0C6180100010003C767021377B8
:10882000C70F2383E7025DBF411106C69700000012
:10883000E78080E7B2404101170300006700E3F2E0
:10884000411106C697F0FFFFE78080BF97D7FF1F53
:1088500083C7D70FA1CB97D5FF1F83C5450F89C904
:1088600017D5FF1F1305C50E97E0FFFFE780C05324
:1088700097D7FF1FA38C070C97D7FF1F23880726C6
:1088800037E700E0B70640002320D71801000100B9
:10889000378600408347660293F7370F2303F602BB
:1088A0002320D710B2404101828041C9D9C597D752
:1088B000FF1F83C7E723D1C3011122CC4AC84EC68C
:1088C00056C25AC006CE26CA52C42E89AA8901446D
:1088D000930A0004371B030063772403B30789401E
:1088E000C207C183BE8463F4FA0093040004C20487
:1088F000C180130A1BD497D7FF1F83C727059DE3A9
:108900007D1A631C0A00F2406244D2444249B249D3
:10891000224A924A024B0561828097F0FFFFE7806E
:1089200020B2D1BF338589002694A68542049700E2
:108930000000E78060E5418045B7828097D7FF1F40
:108940009387873218429C4383D64500034507002E
:1089500083C5C700035646006396A50083D5E7008C
:10896000638DD502011106CE2386A7002397D70079
:10897000B705CF00DC4B9385757D05077D162EC2AC
:10898000230001003AC42316C1002317D10099C364
:108990000A858297F240056182808280DC4DDC4B43
:1089A00081CFB7E70400904503A38705914517D50C
:1089B000FF1F0345A52B028382806D713C083EC6D4
:1089C000B707E500232291103EC8AA843C083285EF
:1089D000232611103ECA23248110232021112E8921
:1089E00097300000E780E05F2A8497950100938527
:1089F000258F177501001305A57397600100E780A7
:108A0000E013A285179501001305059E97600100EC
:108A1000E780C012294597600100E7800017B7057D
:108A2000CB009385757D680097100000E780006992
:108A3000A285680097300000E780004D014781461D
:108A40007000CA85268597200000E780808C05CDC0
:108A50002A84979501009385A58817750100130551
:108A6000256D97600100E780600DA28517950100D4
:108A70001305459897600100E780400C29459760F1
:108A80000100E78080108320C1100324811083241B
:108A90004110032901105161828097D7FF1F9387EE
:108AA000A71C18429C43797122D406D603480700BC
:108AB00083C807012A8483D6450003554600639680
:108AC000080183D82701638DD80223880701050791
:108AD0002399D7003708CC00DC4B1308787D3ACCBB
:108AE0001307F5FF42CA23080100231EE100231FDC
:108AF000D10099C7080832C62EC482973246A245D3
:108B0000228597000000E78080EBB2502254456137
:108B100082806D713C083EC0B707E5003EC23C084C
:108B20003EC42326111023248110232291102317E1
:108B300001002318010023190100231A0100231B3F
:108B4000010097B7FF1F83D7A78B99E3C167FD1774
:108B50002316F10097B7FF1F83D7A78A91EB97D70A
:108B6000FF1F938767109C439C43DC4783D7070014
:108B700017B4FF1F1304C488584C2317F100835700
:108B80004400484B2318F10031E19785010093859B
:108B9000257C177501001305A55997600100E78032
:108BA000E0F9178501001305E57B97600100E78078
:108BB000E0F8294597600100E78020FD8320C1107F
:108BC00003248110832441105161828097B7FF1FD5
:108BD00083C7778389EBB7E70400BC5782975C4C67
:108BE00023AA0700E1BFFD1797B6FF1FA38DF680EC
:108BF00003560701834704014C470A85230BF10004
:108C000097300000E780602D97D7FF1F9387C70537
:108C10009C430147814688430A866C0097100000F8
:108C2000E780206FAA8429C197850100938545724A
:108C3000177501001305C54F97600100E78000F02C
:108C4000A685178501001305A57297600100E780CE
:108C5000E0EE294597600100E78020F3584CB7E724
:108C60000400BC57484B9DBF97A7FF1F83C7B77928
:108C7000F5D7B7E70400BC4F1044854517D5FF1F53
:108C80000345C5FE82971DBF5C4EDC4BB9CFB1CD0D
:108C9000411122C417750100130585492E8497855B
:108CA00001009385256906C697600100E78000E909
:108CB000A285178501001305656E97600100E780A6
:108CC000E0E7294597600100E78020ECB7E7040062
:108CD0002244B24003A3870517D5FF1F034505F9BA
:108CE000130640069145410102838280411122C44E
:108CF00017A4FF1F1304846E1C4C06C689C7DC43EF
:108D000099C34C488297584CB7E70400BC57484B6E
:108D100082975C4CB240224423AA07004101828022
:108D200017A7FF1F1307876D834707009306F00BF4
:108D3000850793F7F70F63E9F60097A6FF1F238FC8
:108D4000F66A034507008280930700F8FDB7835752
:108D500045006386071001114AC817A9FF1F1309B0
:108D6000296A52C4032AC90106CE22CC03274A012C
:108D700026CA4EC656C2F15735E31307D00DFD572C
:108D8000636EC704B7E9040083A709072A841305A3
:108D9000860042054181B284AE8A8297232AAA00C6
:108DA0000325C9015C49A9E797850100938585568C
:108DB000177501001305C53797600100E78000D8DB
:108DC000178501001305C56597600100E78000D78E
:108DD000294597600100E78040DBDD57F24062449F
:108DE000D2444249B249224A924A3E850561828074
:108DF00093874400B705CF002319F5009385757D4F
:108E0000310597100000E780602B0325C9018345D9
:108E10006400310597300000E780000F0325C90189
:108E20002686D685310597300000E780000B714615
:108E3000A2854A8597600100E780E0C4504419CAC2
:108E400083A78905854517D5FF1F034525E282972E
:108E5000814769B797000000E780E0CBD5BFFD5799
:108E60003E858280411126C297A4FF1F93844459F6
:108E7000D84C22C437E404003C54484B06C68297C1
:108E8000DC4C0323C4052244B240924423AA0700C9
:108E900017D5FF1F034585DD85454101028341113B
:108EA00026C297D4FF1F938424DC9C4006C622C4AC
:108EB0004AC0D5C3DC43C5C35CC12300B5002A84C6
:108EC00097850100938545401775010013054526D8
:108ED00097600100E78080C6294597600100E78020
:108EE000C0CA9C4023A4070023A2070097A7FF1F26
:108EF0009387C74EDC4FDC4B91C729559700000084
:108F0000E78000DF97A7FF1F9387874FDC4FDC4B7D
:108F100089C797000000E78020F537E90400832720
:108F2000C905894517D5FF1F034545D48297832777
:108F3000C905914517D5FF1F034545D382979C402E
:108F400003A347016309030022852244B2409244EF
:108F5000024941010283B240224492440249410144
:108F600082800111328506CE22CC26CA2E8497300B
:108F70000000E7800007AA849785010093850538E3
:108F8000177501001305C51A97600100E78000BB43
:108F9000030784000356640083554400A6861785A2
:108FA00001001305A54197600100E78020B929451C
:108FB00097600100E78060BD97A7FF1F83C76742E6
:108FC000639D9700014597000000E78060D28145CE
:108FD0000A8597000000E780C0ECF2406244D2446A
:108FE000056182806D7123248110232611102322B4
:108FF000911093F745002E84638707143C083EC008
:10900000B707E5003EC23C083EC423170100231801
:10901000010023190100231A0100231B010097A757
:10902000FF1F83D7A73B99E3C167FD172316F10004
:1090300097A7FF1F83D7A73A91EB97D7FF1F938777
:10904000A7C29C439C43DC4783D7070017A7FF1F99
:109050001307C7382317F100544F835747002318CD
:10906000F100DC4AA1E7978501009385652D17750E
:1090700001001305E50B97600100E78020AC178520
:1090800001001305252E97600100E78020AB2945DC
:1090900097600100E78060AF134544008320C11052
:1090A00003248110832441105161828097A7FF1F00
:1090B00083C737332555D9C3FD1717A6FF1FA30252
:1090C000F63203D6060183470701CC460A85230BF7
:1090D000F10097300000E78040E097D7FF1F9387AB
:1090E000A7B89C4317A7FF1F1307472F97860100B8
:1090F0009386462A88430A866C0097100000E78012
:109100004021AA8451D9978501009385652317755D
:1091100001001305E50197600100E78020A2A68504
:10912000178501001305C52497600100E78000A1A1
:10913000294597600100E78040A52685970000003B
:10914000E78000BB91BF93F725009DC7B7E70400F8
:10915000BC47414681452808829725559700000065
:10916000E78000B928089305F00F97000000E7801A
:1091700040D3134524001DB793F71500014599DF2F
:1091800097000000E78020991345140001BF5C4D53
:10919000411106C688C317D7FF1F2327F7ACB7E7CF
:1091A000040083A70708170500001305E5E382976D
:1091B000B24097D7FF1F238BA7AA014541018280A8
:1091C00001113335A000A307A100B7E7040083A76E
:1091D000471706CE1306F1008545130550308297D8
:1091E000F240056182808280411122C406C697D771
:1091F000FF1F83C727A9014489EF97B7FF1F83C7C4
:10920000B702054499E717C4FF1F034424421344DF
:109210001400228597000000E780C0FA178501003E
:109220001305052B09E4178501001305652B22445E
:10923000B24041011763010067004390797122D465
:10924000A30F010037E404008327841726D24AD0F5
:1092500006D6AA842E89130550309305F10132C633
:10926000829732468347F10193150601C18185CB70
:1092700001452EC697000000E780C0F483274417FD
:10928000B2454A8626858297054597000000E7800B
:1092900060F3B25022549254025945618280832770
:1092A00044174A8626858297EDB7411193970501A9
:1092B00022C406C626C2C1872E8463D40702B7E43F
:1092C0000400FC5417A5FF1F03458516829719C19A
:1092D000BC5482972165218DB240224492444101C1
:1092E000828093F715008DC7B7E7040083A7471A5C
:1092F00017A6FF1F1306C61297D5FF1F9385C597A4
:1093000017A5FF1F0345C512829713451400E9B73F
:1093100093F7250099CFB7E70400BC4F130600640C
:10932000894517A5FF1F0345A51082971345240003
:1093300065B793F7850085CF97D7FF1F83C74795FC
:1093400085E7B7E7040003A8871A1307401F97A70C
:10935000FF1F83C7E70D814613064006994517D5C1
:10936000FF1F03556592029813458400B5B793F724
:1093700045000145B5D3B7E4040083A7041817D509
:10938000FF1F035565908297BC4C130600649145FE
:1093900017A5FF1F0345C5098297134544002DBF3C
:1093A00097D7FF1F83D7478E6398A70217D7FF1F52
:1093B000231DB78C17D7FF1F231AC78C17D7FF1F82
:1093C0002317D78C2E86178501001305E517BE8558
:1093D00017530100670083761785010013054518B0
:1093E000176301006700638D0357450097D7FF1F80
:1093F00083D78789631EF704C1674111F91722C417
:1094000017D7FF1F2322F78837E4040097D7FF1FE1
:1094100023AE078697D7FF1FA386078697D7FF1F20
:10942000238807867C4C06C6894517A5FF1F034580
:10943000250082977C4C914517A5FF1F034545FFEA
:1094400082972244B240410117030000670003DA0B
:10945000178501001305C510176301006700E38538
:109460007D15954763E2A71C178701001307C70402
:109470000A053A951C41011122CC06CEBA972E84DA
:109480008287178501001305250E97600100E7808C
:10949000C082A1A203C7250099476311F7022E8558
:1094A00097000000E78080F4834564001785010081
:1094B0001305850C97500100E780406897B7FF1FA0
:1094C000238407D6178501001305C50C7DBF03C78C
:1094D000250095476319F702C16717C7FF1F035798
:1094E000A77AF91703D5A5006309F702B7E70400C7
:1094F00083A7C7178297178501001305A50A975000
:109500000100E780807B854717B7FF1F230EF7D048
:10951000178501001305850B8DBF97C7FF1F239586
:10952000A77683D7E50097C6FF1F2390F67683D7EB
:10953000050197C6FF1F239BF67483D7250197C6A5
:10954000FF1F2396F67497C7FF1FA38D0772631B37
:10955000E502B7E70400BC4F096613060690A14573
:1095600017A5FF1F0345C5EC82970356E4008355FA
:10957000A400178501001305250497500100E7801A
:10958000E05B51B79307700F2316F100B7E70400B3
:1095900083A7870D17A6FF1F034686E96C008297F5
:1095A0004DF9854717C7FF1FA30EF76C5DB71785E9
:1095B000010013056502D1BD83C525009147639263
:1095C000F502178501001305A50297500100E780F9
:1095D000C06E97000000E78060C1F2406244056100
:1095E000828099476392F502228597000000E78008
:1095F000E0DF83456400178501001305E5F7975008
:109600000100E780A053D1BF9547639AF5008347D7
:109610001400E1F3178501001305C5FFBDB51785DB
:1096200001001305A5FFE1BF82803757315F97A77F
:10963000FF1F938727E1130777D598C39356C5007B
:1096400017870100130707EDBA9683C506009356E6
:109650008500BD8ABA9603C6060093564500BD8AAA
:109660003D89BA962A9783C60600034707002384DC
:1096700007002383D700A383E7002382B700A382D8
:10968000C70097A7FF1F9387E7DC2383B700A38357
:10969000C7002384D700A384E7008280411106C657
:1096A00097000000E780A0F8B7E7040083A78714BD
:1096B00017A6FF1F130606D9D54501458297B2406C
:1096C0004D4697A5FF1F9385E5D8130570304101DE
:1096D000170300006700C3B661712324811A37E4C1
:1096E0000400832704082326111A2322911A232019
:1096F000211B232E311917050000130545BB829746
:1097000017A9FF1F1309C9D2994785442300A9004F
:10971000231CF100978501009385C5DE9307400661
:10972000177501001305C5A0231CF108230891003B
:1097300097C9FF1F9389E9FF97500100E780004018
:1097400083D50900178501001305C5DA975001007C
:10975000E780C03E294597500100E780004303D5CC
:109760000900896997000000E78060EC83274417AF
:10977000100885451305503082978327441717A694
:10978000FF1F130626CDCD45130570308297832722
:10979000441717A6FF1F1306E6C9B5451305603029
:1097A0008297832744173008894513051031829723
:1097B0008327441730098945130520318297832771
:1097C0004415938509900D45829783274415938509
:1097D000099011458297A305910023069100230863
:1097E000910002CD230C0100832784163009914596
:1097F000130570408297832784161306B1008545B0
:109800001305004082978327841670008545130551
:109810001040829783278416300885451305204021
:109820008297832784161008854513055040829738
:10983000832704157D558297832744137D5582978E
:109840007D5597A0FFFFE78040E48327440C829773
:1098500097A0FFFFE780A0BF8327841417A6FF1FF0
:10986000130646BED5450145829789471306700FFA
:10987000814528092306F1009790FFFFE7802089A2
:109880008D471306000881452808230CF10897909E
:10989000FFFFE780C0879147230CF1009767010025
:1098A0009387877A984383C747003AC8230AF10011
:1098B00097D0FFFFE78040B070008545054597A031
:1098C000FFFFE780A0E330099305700F094597A0DB
:1098D000FFFFE780A0E23008930500080D4597A040
:1098E000FFFFE780A0E110089545114597A0FFFF15
:1098F000E780C0E0C16717C7FF1F1307E738F917F4
:109900001CC32322070017A5FF1F130525B297A02C
:10991000FFFFE78080DD8327C41D17C5FF1F1305E8
:10992000253582973C480345090085458297832069
:10993000C11A0324811A8324411A0329011A832995
:10994000C1195D618280C16717C8FF1F0358C83302
:10995000F9176301F8083DCDB5CD011126CAB7E46A
:10996000040083A7841222CC2E862315B10006CED4
:109970002A8401478146ED45428582972AC611ED2A
:1099800017850100130545BA97500100E780E032C2
:10999000F2406244D24405618280FC440356A10037
:1099A000A28582972C0017C5FF1F0355E52D97A0B0
:1099B000FFFFE78040E069DD17850100130505B86A
:1099C00097500100E780602F83A7C412ED4528005F
:1099D00082977DBF82800DC5854717A7FF1FA30013
:1099E000F7A697A7FF1F238D07A4354697A5FF1F4E
:1099F000938545A413056030170300006700438476
:109A000097A7FF1FA38D07A2E9BF97C7FF1F83C7B3
:109A10002728A9EFC16717C7FF1F0357E726F917C4
:109A20006306F7044111854722C417C7FF1F2301AE
:109A3000F72637E404007C4C06C6A14517A5FF1F96
:109A40000345059F82970323841A2244B24097A7B7
:109A5000FF1F83C7E79D17C5FF1F0355E5221307A7
:109A6000401F8146314699454101028382806D71D4
:109A7000232481102326111023229110328401CD3A
:109A80008947630AF5028320C110032481108324CF
:109A9000411051618280178501001305E5B8AE843D
:109AA00097500100E7806021A285268597C0FFFFBF
:109AB000E780C0B0C9BFB7E70400FC472800829721
:109AC00017850100130505B797500100E780E01ED8
:109AD0008347810039C41307000B6380E7021387B3
:109AE000A7051377F70F8D4663EDE602A2852800E0
:109AF00097C0FFFFE780802079B78547E3F587F8B7
:109B000083459100177501001305C597B335B00063
:109B100097A7FF1F238AB75897500100E7800002DC
:109B20009DB703479100A207D98F35671307D75513
:109B30006385E7086368F7022D671307B7556387E6
:109B4000E70631671307C755638AE70429671307D8
:109B5000A7556394E702A285280097C0FFFFE7801E
:109B6000405815B739679306E7656381D70863E9FD
:109B7000F6001307E7556384E706A28528003DB782
:109B80003D679306F755638AD7061307F766E39692
:109B9000E7FE97C0FFFFE780C070F5B50146A285DC
:109BA000280097C0FFFFE7800041F1BDA285280093
:109BB00097C0FFFFE7802051F9B58947E3F587ECAF
:109BC00097000000E780A0E49305E4FFC205C1818F
:109BD0001305A1009790FFFFE78080606DB5A28517
:109BE000280097C0FFFFE780C05071BDA285280004
:109BF00097C0FFFFE780805B79B597C0FFFFE780E4
:109C0000006451B5C16717C5FF1F0355E507F91774
:109C10006307F500B7E7040003A3C7170283828038
:109C2000854717C7FF1F230FF704014517F3FFFFF1
:109C3000670043591783FFFFE702C3482A8408459A
:109C40002E89B28919C900C1971500009385A58690
:109C5000610597300100E780800181447D5A9710AB
:109C60000000E780E03963C7A40481449710000036
:109C7000E780003A63C8A40497C7FF1F9387870152
:109C80009C43DC47B307F94091872302F4006383C8
:109C900009048327C900B307F4409587A302F400A1
:109CA0001C4C89C79C4799C3228582971783FFFF65
:109CB000670083445C44139714008504BA9723908B
:109CC000470171BF1C48139714008504BA9723906D
:109CD000070069BF832789000547B307F4409587CC
:109CE000A302F40083570400638EE7028DC3094783
:109CF0006384E7040D47E395E7FA978701009387AC
:109D000027E61CCC97870100938787E611A89787E1
:109D10000100938767AC1CCC978701009387C7AC81
:109D20005CC8BDBF97870100938707981CCC9787B5
:109D3000010093876798EDB797870100938707E73E
:109D40001CCC97870100938767E7D9BF95E51783F8
:109D5000FFFFE702C3380046184483479400758329
:109D60009D8B6317F70097100000E78060B448C42C
:109D70001783FFFF6700E33882801783FFFFE70246
:109D8000633413893500C16442094111AA89014431
:109D9000F11413590901054A2EC697100000E780F7
:109DA0002026B2456348A400014541011783FFFF07
:109DB0006700833483A7090013171400BA9783D769
:109DC00007006388B7006394970063742A01050451
:109DD000E1B70545D9BF1783FFFFE702C32DAA8965
:109DE0002E89328BB6843A8ABE8A97A00000E7801B
:109DF00020FB71C9268597200000E78020098D4748
:109E000063E7A7007D551783FFFF6700432E83DBC1
:109E1000440097100000E780A0242A8497100000D7
:109E2000E78040259307740031443305850263CDF4
:109E3000A70297100000E780A02297100000E7809B
:109E400020222A8497100000E780C0229307740024
:109E500031443305850263C3A70497100000E780EF
:109E600020209307450029A897100000E780802054
:109E7000330585021307F0179307C017E35FA7FAAE
:109E80002D55E3C277F963040B02D6865286A68568
:109E90004A8597200100E78020BAB5B797100000E7
:109EA000E780401D330585029307C5FFD1BF832797
:109EB00049001385C90083D5270097000000E7807B
:109EC00000EC61F581B769553DBF97C7FF1F23952A
:109ED000A7DC97C7FF1F9387E7DB904381470C46BA
:109EE0003307F500420741836393B70082805446ED
:109EF000139847008507C2962390E600D5B797C709
:109F0000FF1F938727D99C4303C58700828017C50D
:109F1000FF1F035565D882801783FFFFE702231CCC
:109F2000C1671387D7FF630BE502636AA700F117C8
:109F30006300F50201451783FFFF6700831C138749
:109F4000E7FF6302E502FD171D8D13351500E5B728
:109F500097500000E780C0267D15C5BF97500000D0
:109F6000E78040FBD5BF97500000E78060F9EDB770
:109F70001783FFFFE702A3164111AA8401442EC6EE
:109F800097100000E780C008B2456348A40001456F
:109F900041011783FFFF6700C3169C481315140087
:109FA0003E9583570500E385B7FE0504C9BF034806
:109FB0005500814693F7F60F63E5070181473E851B
:109FC0008280584593975600BA9703D727006316A7
:109FD000B70003D70700E304C7FE8506E1BF834649
:109FE000450001479377F70F63E4D700814711A835
:109FF0001C45131657000507B29703D60700E31355
:10A00000B6FE3E8582801783FFFFE702A30B9317FE
:10A010000501C18797CAFF1F938ACAC7635BF0080F
:10A0200083A70A00C0479C4703570400198D4205C7
:10A0300041816368F500014422851783FFFF6700B3
:10A04000A30B12052A94CDBFDC4713944900014AA3
:10A050003E94834744006341FA02014A8347540017
:10A060006349FA028509C20993D9090183A70A0045
:10A070009847E3EBE9FCC1B71C4413195A00A685C5
:10A080003E994A8597000000E780C0EE05E1050A89
:10A09000C9B75C4413195A00A6853E994A859700B2
:10A0A0000000E78020ED19E1050A4DBFE30C09FA35
:10A0B00061B7AA8481495DBF1783FFFFE7022302CE
:10A0C0001C452A8481E79307C5001CC51C44231244
:10A0D00004001CC09307F00F63EDB70093F5F50F74
:10A0E000228597200000E78020E21783FFFF6700AA
:10A0F000430193940501C167C18063F9F500A6850A
:10A10000228597200000E78040E5C5B7C18193F51F
:10A11000F50F228597200000E78000DFA6852285C5
:10A1200097200000E78040E0C9B797C7FF1F9387DB
:10A1300067B6884382801C4599C797C7FF1F23AB2A
:10A14000A7B4014582807D55828097C7FF1F938702
:10A1500067B4984383474500484792073E958280FD
:10A160001783FFFFE702A3F7617100451C183EC685
:10A17000B70780013EC81C183ECA8357440002CE70
:10A1800002D002CC231EF100834784002A8902D228
:10A190002301F1023C083ED402D697000000E7807C
:10A1A00000FB835705002316F10297500000E7805B
:10A1B00060C42307A1025C4003556400F18313F7D8
:10A1C00017008347F10252055181F99BD98FA307EC
:10A1D000F10297100100E780807539CDAA840355FC
:10A1E000050097A00000E78080BC83D704002AD236
:10A1F0006800231CF10083D72400231DF1001C48B4
:10A2000003D647008C4397200000E78000CD8347AA
:10A21000B400CA8617760100130686428117A3058B
:10A22000F4006C00481097200100E780E0805D6139
:10A230001783FFFF6700E3EC2155D5BF1C45B1CF65
:10A2400003C5A700894613576500630BD7028D46E7
:10A25000630ED70285466300D70213074006330515
:10A26000E50203C7B700418B15CB83C7B700BD8B91
:10A270003355F54082801375F5031307803EC5B74B
:10A2800009671375F50313070771D1BF3727090055
:10A290001375F5031307077CD9B70145828017832F
:10A2A000FFFFE702C3E303A98500630C09048347AA
:10A2B000B900AE8493F7070E85C303459900930553
:10A2C00020030D810505B305B5028844610597306B
:10A2D0000100E780E0A935A02E8597000000E78007
:10A2E00020F62A8419CD97000000E780605C832562
:10A2F000C900B307B54063FA87002E94B305A440A4
:10A30000E9F51783FFFF6700C3DF85457DBF17832E
:10A31000FFFFE702C3DC2A8403D50500011132C622
:10A3200036C43AC22EC002CA02CC02CE97A00000A8
:10A33000E780E0A782452ACA22852ECC970000003C
:10A34000E780E0E003570500231EE100975000007E
:10A35000E78040AAA24632469247230FA1003687E3
:10A360004C08B2862285014697000000E780E0A6EF
:10A3700005611783FFFF6700C3D81783FFFFE7025C
:10A3800003D661711C183EC6B70780013EC81C1871
:10A390003ECA3C0800453ED4AA8402CC02CE02D07C
:10A3A00002D202D697000000E78060DA83570500EA
:10A3B00035592316F10297500000E780A0A3230728
:10A3C000A10209C48357440081EB21594A855D618C
:10A3D0001783FFFF6700E3D20355640052055181E4
:10A3E00097100100E780A0542A8965D18347B40003
:10A3F00093F7070E99C71305840197300100E78092
:10A40000609983574400231EF10083478400230191
:10A41000F1025C4003550900D98313F7070883470D
:10A420001102231CA10093F7F707D98FA300F102B3
:10A4300083572900231DF1005C40F18313F71700B7
:10A440008347F102F99BD98FA307F10297A000007F
:10A45000E780E0952AD235D98347940068001397A6
:10A4600057008347B400FD8BD98FA305F4001C4827
:10A4700003D647008C4397200000E78000A6A687FC
:10A48000177701001307C71B740005464C1026857B
:10A4900097000000E78060942A890DD98347B400B3
:10A4A000A685FD8BA305F40097000000E78060DF20
:10A4B00031BF1783FFFFE70283C2832485FE2A840E
:10A4C0004111268597000000E78080D7834734FF3D
:10A4D00093F7070E8DCB2AC6268597000000E780EC
:10A4E00060C809CD834734FFB245FD8BA309F4FE54
:10A4F00091C5228597300100E7808087410117834D
:10A50000FFFF670003C07DD98327C4FF268582979C
:10A5100075F5834734FF93F7070E91C7228597306F
:10A520000100E7802087032584FE97000000E78074
:10A5300000E5E9B71783FFFFE70263B79C414111CC
:10A540002A8903C7070089472E84935667006380D2
:10A55000F6040D466388C6049307F0076304F70208
:10A560002E8597200000E780C0A7AA848149C16B8F
:10A57000130C490097B7FF1F9387C7719C439847F7
:10A5800063E4E90441011783FFFF670003B603D7C3
:10A5900045008547E3F8E7FE2E8597200000E78019
:10A5A000A0A9E1B703D74500E3FEE7FC2E8597207D
:10A5B0000000E78000A3AA84228597200000E7809E
:10A5C00060A4C204C98C5DB7DC470355A900139A87
:10A5D00049003E9A93170501C187635DF0008357D8
:10A5E0000A006397A70263E774038327CA00034D39
:10A5F0005A002DA0A1672167A98F1307F7EFE37415
:10A60000F7FE6397090097000000E780209161FD45
:10A6100085098DB783278A00034D4A00835DA90011
:10A6200003576900216A138BC7003AC6814A33CAAF
:10A630004D01631E5D0197B7FF1F938727669C43FB
:10A64000E1DBA2866286814526858297D1B7A16724
:10A650009387F7EF930C4BFF63F24703B2455A859C
:10A6600097F0FFFFE780A0710DC103278B00104713
:10A6700009CE10436382C4023107D5BFEE856685DB
:10A6800097000000E780008F71F993861A0093FA13
:10A69000F60F130B0B0271BF835644005C43E3E9D2
:10A6A000F6F622853AC697100000E780807DA16704
:10A6B0009387D7042A8A035D4400324763E89700F2
:10A6C0008347D90093E707F8A306F9001C4766857E
:10A6D0002286E2858297C1670844FD17337AFA0023
:10A6E000529508C02312A40125B797B7FF1F93877F
:10A6F000675A9843814715C31447814763FFD500C4
:10A70000939745004C47BE9519C903C7550081472B
:10A710006375E600DC451606B2973E85828003C766
:10A7200045008147E37BE6FE16069C45F5B7178397
:10A73000FFFFE7022399AA892E8A814497BAFF1F57
:10A74000938A4A5583A70A00984763E6E400178373
:10A75000FFFF6700639ADC471394440001493E946D
:10A7600013BB140083474400634BF900014913BB3A
:10A77000140083475400634FF9008504E1B708448F
:10A78000931759005287DA860146A2853E95829931
:10A790000509C9BF4844931759005287DA86054610
:10A7A000A2853E9582990509E9B71783FFFFE70265
:10A7B0000393814517F5FFFF1305054897B7FF1F62
:10A7C000239C074C97000000E780A0F61783FFFF4B
:10A7D0006700239397B7FF1F9387C74B9C4395C38D
:10A7E0001783FFFFE702A38F814517F5FFFF1305CE
:10A7F000A54497000000E780C0F31783FFFF6700C0
:10A80000439082801783FFFFE702C38B37E4040085
:10A810008327841241112315E100AE893289368ADB
:10A820003A8681460147ED45AA8482972AC621C906
:10A830000356A100D28597400100E780C0248327FA
:10A84000C413CE8526858297058905C98327440DC3
:10A850002314210101462C00268582972A8401C9F0
:10A86000B7E7040083A7C712ED4528008297228529
:10A8700041011783FFFF670023884944D5B765541A
:10A88000FDB75C41FD175CC182801783FFFFE702C3
:10A890000385B7E70400FC5F829795473305F5020F
:10A8A00081450D811783FFFF6700A3851783FFFF95
:10A8B000E702E382B7E70400FC5F82979547330520
:10A8C000F5020D811783FFFF6700A3831783FFFF46
:10A8D000E702E380B7E7040083A7870B0355050071
:10A8E00082971783FFFF6700C3811773FFFFE7029B
:10A8F000037F035505003287AE861796FF1F035668
:10A9000086BB97B5FF1F9385A53997000000E780A8
:10A91000A0EF1773FFFF6700C37E1773FFFFE70207
:10A92000037CB7E7040083A7C71782971773FFFF5D
:10A930006700237D1773FFFFE702637AB7E7040020
:10A9400083A7871397B5FF1F9385853582970145A8
:10A950001773FFFF6700E37A1773FFFFE70223789F
:10A96000B7E7040083A7C71F81451795FF1F03554D
:10A9700085B082971773FFFF6700A3781773FFFFF7
:10A98000E702E375B7E7040083A7871397B5FF1FB6
:10A9900093850532829701451773FFFF6700637641
:10A9A0001773FFFFE702A373B7E7040083A7C71F6E
:10A9B00081451795FF1F035505B282971773FFFF57
:10A9C000670023741773FFFFE70263712E8597807A
:10A9D0000000E780E0AF97800000E780E0EC1773AD
:10A9E000FFFF670003721773FFFFE702436F978053
:10A9F0000000E780E0F61773FFFF670083705C4993
:10AA0000E1175CC95CC583572501A1072319F5002F
:10AA100083570501A1072318F5008280F14733050C
:10AA2000F50297B7FF1F9387A72A9C433E95828024
:10AA30008D476315F60803D74600854763F0E7089E
:10AA40001773FFFFE702A369368536842E899710B6
:10AA50000000E780005929C9835744009314050179
:10AA6000C18063E39704228597100000E780605758
:10AA7000FD14231294009307A0026300F5029307CC
:10AA8000B0026307F50293079002631FF500228569
:10AA900097000100E780C08501A80146CA8522858C
:10AAA00097A00000E78060B01773FFFF6700636541
:10AAB000228597100000E780C003FDB7828097B61B
:10AAC000FF1F938626219C42014599CF9843D4428B
:10AAD00017B6FF1F2320E6206396D70097B6FF1F07
:10AAE00023ACE61E1385C7FE82801773FFFFE702C3
:10AAF000035F97000000E780A04B71443305850297
:10AB0000914597900000E78020E911E5655517739E
:10AB1000FFFF6700035F97B7FF1F23A9A71A9700DE
:10AB20000000E780E04833058502914597900000DA
:10AB3000E78080E661DD97B7FF1F23ABA71897007A
:10AB40000000E780E04697B7FF1F239BA7169700FA
:10AB50000000E780E04597B7FF1F2394A71697777B
:10AB60000100938727B317B7FF1F232FF714970709
:10AB70000000938707E917B7FF1F2325F714014546
:10AB800079B71773FFFFE7028355AA8517B5FF1F33
:10AB90001305051397100000E780C05B1773FFFFD4
:10ABA000670023561773FFFFE70263539700000007
:10ABB000E78060FD97100000E780405B97B7FF1FBC
:10ABC000938747119C4391CF1387C7FE19CB83D539
:10ABD000C7FF17B5FF1F1305651097200100E78019
:10ABE00020191773FFFF6700C3511773FFFFE702B8
:10ABF000034F97000000E780C0EC09CD8347850034
:10AC00002A8493F7070499EB0355E50097000000A9
:10AC1000E78080F91773FFFF6700A34E8347C500E5
:10AC20009304450117B9FF1F1309C90A85E3832758
:10AC300009005CC997B7FF1F23AE97088327490017
:10AC4000F1FB97B7FF1F23A99708E9B7FD17230664
:10AC5000F500610597800000E780C0D68307840077
:10AC600063CB07048347840093E707F82304F400C9
:10AC7000B7E704009C5F82974205A947418133757D
:10AC8000F5028347840093F707FCC98F2304F4007F
:10AC90008347D4003E951C402318A40089CF9843D5
:10ACA00019CB8347C4005040814585073305F50221
:10ACB000420541810297832709005CC897B7FF1FAF
:10ACC00023AA97008327490089E797B7FF1F23A589
:10ACD00097008347C4009DDF8355040117B5FF1F0C
:10ACE0001305C5FF97200100E780800825B717737B
:10ACF000FFFFE702C33E97B7FF1F938767239C4779
:10AD000001448583858B85E3AE84B2853A869710AE
:10AD10000000E780804B2A8419C597100000E78067
:10AD2000C041829408CC22851773FFFF6700633D02
:10AD30001773FFFFE702033941112E8932C6AA8932
:10AD400097000000E780C031324713060502CA862B
:10AD5000970500009385C5CC17B5FF1F130545F671
:10AD600097000000E780E0F82A8425C99304C50015
:10AD700097000000E780E0411946AA8526859710D4
:10AD80000000E78080158545268597100000E78044
:10AD90006011177501001305A58D4E9583450500BB
:10ADA000268597100000E78020165C4831468145D3
:10ADB000A1075CC85CC483572401E1172319F40080
:10ADC00083570401E1172318F4001C4C3E8597704B
:10ADD000FFFFE780C033A3042501228541011773DB
:10ADE000FFFF670063311773FFFFE702432F411135
:10ADF000AA842EC632C497100000E7806036004D4A
:10AE0000B2452246834784000CC050C093F7F70335
:10AE100093E707042304F400231804002685971001
:10AE20000000E780803183479400A9462317A400DF
:10AE300013D7370005073307D7029D8B85072306F5
:10AE4000F400A306E40083C70401D8488507230F54
:10AE5000F7FE17B7FF1F1307E7E75843232A04003D
:10AE60009307440129E317B7FF1F2327F7E617B716
:10AE7000FF1F2321F7E617B4FF1F130424E62285E2
:10AE800097200100E78000E11C44858B5D8D19E56A
:10AE90008145228597200100E78080ED41011773ED
:10AEA000FFFF670003261CC317B7FF1F2326F7E227
:10AEB000D9B71773FFFFE702832297050000938538
:10AEC00065B7014597000000E78000B001451773A2
:10AED000FFFF670003231773FFFFE702432097007C
:10AEE0000000E78080B01773FFFF6700832183476E
:10AEF000C500A5E31773FFFFE702631E2A8403550D
:10AF0000E50097000000E78000C821C18347840066
:10AF100093F7F7FB2304F4001C4091C7DC4381C77F
:10AF20004C400145829797000000E78080B917B533
:10AF3000FF1F1305A5DA97200100E780A0E5035560
:10AF4000E40097000000E78020C61773FFFF67004A
:10AF5000431B82801773FFFFE702631897B7FF1F39
:10AF6000938747D797050000938565C817B5FF1FDE
:10AF70001305C5D623A0070023A2070097200100D0
:10AF8000E780E0CE1773FFFF6700A3171C4D91CF3A
:10AF9000DC4381CF1773FFFFE7026314834507008B
:10AFA00082971773FFFF6700C315828097B7FF1F53
:10AFB000938707D59C4303C50700828097B7FF1F7F
:10AFC000938707D49C4303C51700828097B7FF1F60
:10AFD000938707D39C4303C52700828097B7FF1F41
:10AFE000938707D29C4303C54700828097B7FF1F12
:10AFF000938707D19C4303C53700828097B7FF1F13
:10B00000938707D09C4303C55700828097B7FF1FE3
:10B01000938707CF9C4303C56700828097B7FF1FC4
:10B02000938707CE9C4303C57700828097B7FF1FA5
:10B03000938707CD9C4303C58700828097B7FF1F86
:10B04000938707CC9C4303C59700828097B7FF1F67
:10B05000938707CB9C4303C5A700828097B7FF1F48
:10B06000938707CA9C4303C5B70011E11D45828041
:10B0700097B7FF1F9387C7C89C4303C5C70082804B
:10B0800097B7FF1F9387C7C79C4303C5D70082802C
:10B0900097B7FF1F9387C7C69C4303C5E70082800D
:10B0A00097B7FF1F9387C7C59C4303D507018280CD
:10B0B00097B7FF1F9387C7C49C4303C527018280AE
:10B0C00097B7FF1F9387C7C39C4303D5470182806F
:10B0D00097B7FF1F9387C7C29C4303D56701828040
:10B0E00097B7FF1F9387C7C19C4303D58701828011
:10B0F00097B7FF1F9387C7C09C4303C5A7018280F2
:10B1000097B7FF1F9387C7BF9C4303C5B7018280D2
:10B1100097B7FF1F9387C7BE9C4303C5C7018280B3
:10B1200097B7FF1F9387C7BD9C4303C5D701828094
:10B1300097B7FF1F9387C7BC9C438857828097B7F8
:10B14000FF1F9387E7BB9C4303D5C702828097B755
:10B15000FF1F9387E7BA9C4303D5E70219E1130564
:10B16000800C828097B7FF1F938787B99C4303C5E4
:10B170000703828097B7FF1F938787B89C43C85BFC
:10B18000828097B7FF1F938727B78843828097B73E
:10B19000FF1F9387A7B68843828019E17D5582807F
:10B1A000F5DE984265DFFDD917B7FF1F130747D8B3
:10B1B0001847AA877155058B631D072403C507002F
:10B1C0001547E37DA7FC03C737001305F0057D177E
:10B1D0001377F70FE364E5FC03C35700E30003FCB8
:10B1E00083C86700E38C08FA03C7770049457917DD
:10B1F0001377F70FE364E5FA03C7A70011481305B7
:10B20000F7FF1375F50FE36BA8F803CE97000D4811
:10B210001305FEFF1375F50FE362A8F803C8B70026
:10B220006309080065181378F80F1305600DE367CC
:10B2300005F703C5C700794879151375F50FE36F56
:10B24000A8F403C8D7000D457D181378F80FE367FD
:10B2500005F503D80701930E4017511842081358FB
:10B260000801E3ED0EF303C8E7007D181378F80F2B
:10B27000E36605F303C827017D181378F80FE36F21
:10B2800005F103C88700C54E75181378F80FE3E77A
:10B290000EF103D86701856E938EBEE06D184208EB
:10B2A00013580801E3EC0EEF03D847016D1842086C
:10B2B00013580801E3E40EEF03D887017918420818
:10B2C00013580801E36C05ED03C8A7017D18137836
:10B2D000F80FE36505ED03C5B7011D487D1513752E
:10B2E000F50FE36DA8EA03C5D70171487915137509
:10B2F000F50FE365A8EA03D5E7011308E00F7D1514
:10B3000042054181E36CA8E803C507024948791565
:10B310001375F50FE364A8E8C85301C937C83400B2
:10B320005915130858BFE36BA8E603A8870237C571
:10B330003400130555BF5918E36205E717B5FF1F21
:10B34000232EC59A03C6050117B5FF1F232AF59AB8
:10B350000545E375C5E403D82501D04933760603D6
:10B36000E31E06E203C61501E30A06E217B6FF1F55
:10B370002324B69883C5270001466387A50003C62A
:10B380001700F1453306B60283C707039305C002D1
:10B3900072971A071307C70516031A979608469758
:10B3A000B387B70241553E973297420741836362A4
:10B3B000E8061773FFFFE70283D236859780000007
:10B3C000E780A06897000100E78020482A8497A0C2
:10B3D0000000E780805A2A9497F00000E7806026FA
:10B3E0002A9497900000E780A0812A9497F0FFFFAD
:10B3F000E780E06F2A9497400000E78060932A94EA
:10B4000097700000E780A09C22951773FFFF6700EC
:10B4100043CF82801773FFFFE70263CC4111A3077C
:10B42000A10097A00000E780A0C59305F1001705D3
:10B4300000001305E5B597F0FFFFE780802F014579
:10B4400041011773FFFF6700C3CB1773FFFFE702CC
:10B4500083C617B4FF1F1304A4AD032884007959D1
:10B460009368180097B4FF1F23A814AD1378180031
:10B4700063100802BA84BE89368B328A2E89AA8A62
:10B4800097F0FFFFE780E0A77D15269519E5315974
:10B490004A851773FFFF670083C597F0FFFFE780BA
:10B4A00040A67D152695A167E353F5FE97B7FF1FCC
:10B4B0009387C7DE98433E8C814B01CB014597F0C3
:10B4C0000000E7802044933B15004A85DA865686C3
:10B4D000D28597900000E780C04D2A8911CD1C4489
:10B4E000F99B17B7FF1F2329F7A483270C00CDD39F
:10B4F000E3800BFA829769BF268597B7FF1F23ABBE
:10B5000007A297F0FFFFE780809C4146CE8517B5E4
:10B51000FF1F130565AB97300100E780C05697D039
:10B520000000E78040990325040B97D00000E780D6
:10B53000009D054597D00000E78000A405459700D1
:10B540000000E78060EDA9B797B7FF1F9387479E7C
:10B550009C47858BEDC71773FFFFE70243B817B50C
:10B56000FF1F1305A5A497B7FF1F23A3079C97B739
:10B57000FF1F23A1079C97B7FF1F23AF079A9720B0
:10B580000100E780208197500000E780E0F59710E8
:10B590000100E780A04C97100100E780A05297B708
:10B5A000FF1F938767979C4391C7054597800000CD
:10B5B000E780402097A7FF1F9387C77F9C4399C7C9
:10B5C00041657D1597700000E78040A297F000006C
:10B5D000E780E03D97D00000E780808F97B7FF1F9E
:10B5E0009387C7A99C43139717016356070097F0E9
:10B5F0000000E78000AD97B7FF1F23A7079C97B710
:10B60000FF1F23A5079C97B7FF1F23A3079C97B78E
:10B61000FF1F23A1079C97000000E780008C970084
:10B620000000E780007297F0FFFFE780401897F076
:10B630000000E78040D61773FFFF670083AC82806D
:10B6400097B7FF1F9387C78E884382801773FFFFCA
:10B65000E702E3A897800000E7806075978000000C
:10B66000E780C0771773FFFF6700A3A91773FFFF79
:10B67000E70243A52A849304140201112E85B2899E
:10B68000A685214636C63A8997300100E780403DBD
:10B690000DE9B24638082686CE85130594049750E6
:10B6A0000000E780604121462C084A859730010060
:10B6B000E780003B1335150005611773FFFF670036
:10B6C000A3A30145D5BF1773FFFFE70243A193056D
:10B6D000450617A5FF1F1305E56297100100E780D7
:10B6E00020691773FFFF6700C3A11773FFFFE7020D
:10B6F000039F41112EC697F0FFFFE780601BB24504
:10B7000088C141011773FFFF6700A39F1773FFFFF5
:10B71000E702439BAA842E8497800000E780006C98
:10B72000AA898545228597000000E780E07D83C7D0
:10B73000E4011389940899E313890403CE852285D3
:10B7400097000000E780407C21469305190222857E
:10B7500097000000E780607897A7FF1F9387477DD9
:10B760008C43228597100000E780C0822146938594
:10B770008402228597000000E78020761773FFFF80
:10B78000670083971773FFFFE702E392397197F021
:10B790000000E780E0B49305400661E9978000006F
:10B7A000E78000606302051497A7FF1F83C7475710
:10B7B00013B7170097A6FF1F2384E656014499CFBD
:10B7C000C16417A9FF1F1309A9769309400EFD1440
:10B7D00097000000E780C0866342A40A97F0FFFF4D
:10B7E000E780000D4169B7290900096AFD7A2A8BB3
:10B7F00081447D199389F97B130A0A71938A8AC758
:10B8000097000000E780C08363D7A4041304400EB0
:10B81000B387840217A7FF1F130787710324070B41
:10B820003E948357C4016382270B18403307EB40D3
:10B8300063EAE900834744008507B3874703D69747
:10B840006365F70801468145094597F0FFFFE780EA
:10B85000604EAA8B29E597400000E78080838547EA
:10B860006317F50689659385057117A5FF1F1305F5
:10B87000654997100100E780A04F95A0B3073403F6
:10B880000327090BBA9703D7C7016308970003C7BB
:10B890005700A38207002382E700050415BF930524
:10B8A000C500228597000000E78080E65E8522863D
:10B8B00097650100938505DD97F0FFFFE780E05273
:10B8C0005E8597100000E780608A850415BF97A702
:10B8D000FF1F9387E7659C478D83858BC1F72161A7
:10B8E0001773FFFF6700A38001468545094502D015
:10B8F00002D202D402D697F0FFFFE780A043AA84C9
:10B9000079DD97F00000E780E09C1389C4002A8469
:10B9100081454A8597000000E780005F0C40414662
:10B920004A8597000000E780405B832944006385D7
:10B93000090C4E8502D802DA02DC02DE97300100E3
:10B94000E780E0382ACE141005462C0808184ECCA3
:10B9500097500000E780E00A1375F50F51ED83550D
:10B96000840093E525004A8597000000E780E05EAB
:10B9700011460C104A8597000000E78000560146EA
:10B9800097650100938585D0268597F0FFFFE780B6
:10B99000C045268597000000E780407D5C40A1D32C
:10B9A000014685450D4597F0FFFFE780A038AA8442
:10B9B0001DD548401389C40097300100E78020312D
:10B9C0002AC64A8597000000E780404C3246636FE4
:10B9D000C5004C404A8597000000E78000500146B2
:10B9E0008145268597F0FFFFE78020402685970058
:10B9F0000000E780A077E5B583558400ADB71763F5
:10BA0000FFFFE702C36D97A7FF1F938767529C470D
:10BA10001DC193E7870017A5FF1F1305A52E17A7C4
:10BA2000FF1F232BF75097100100E7804032176368
:10BA3000FFFF6700036DDD9B17A7FF1F232EF74E47
:10BA400097300000E780E0647DF117A5FF1F130524
:10BA5000652B97100100E780E033D1BF1763FFFF2C
:10BA6000E70263654169AA892E8AB28A368BBA8B4E
:10BA7000814417ACFF1F130CAC4B930C400E7D1987
:10BA800097F0FFFFE780C05B63C4A40001443DA0C2
:10BA90003384940383270C0B3E948357C40163863D
:10BAA00027055A87D6865286CE851305040397004C
:10BAB0000000E780E0BB01C923800B0022851763EB
:10BAC000FFFF6700C3628347F40185C35A87D686A8
:10BAD0005286CE851305940897000000E78040B990
:10BAE00009C585472380FB00D1BF850451BF83571B
:10BAF00045006380071E1763FFFFE702A35C011187
:10BB00002A8497000000E780C04D09C98547630972
:10BB1000F50605611763FFFF6700035E97E000000D
:10BB2000E780007C7DF5835744004947ED9BE39215
:10BB3000E7FEC145228597000000E7804033AA84D4
:10BB4000228597000000E780204F0357440002CE73
:10BB500091472A89631AF700228597000000E78041
:10BB6000A0513C082ACC3ECE97E00000E7808076CA
:10BB70005C55C5D374084A86A6850545829751BF92
:10BB800003574400D147E3F6E7F8032A0400C169EC
:10BB9000014997AAFF1F938AAA39130B400EFD197A
:10BBA00097F0FFFFE780C049634FA90E2285032A63
:10BBB000040097000000E780C042A1452A89228541
:10BBC00097000000E780A02AAA8422859700000041
:10BBD000E780804A14402A86AA8978082685CA8583
:10BBE00097000000E780C0E7AA8405D503C7F401E9
:10BBF00089476315F7008347C10181DF5546D28528
:10BC00001385640097300100E780E0E701459780E5
:10BC10000000E780C01901C583D7C401A5E797A735
:10BC2000FF1F9387E7309C4793551900858913D7E9
:10BC30003700058B01CF8983858B6399B700014558
:10BC40002EC697000000E780C0DBB2454E85978086
:10BC50000000E780601F0346C1012A849375190024
:10BC6000268597900000E780E03935C126859780CA
:10BC70000000E780E018268511C00145978000008C
:10BC8000E780004C97300000E780A0408547E31232
:10BC9000F5E883C754001307F00FE38CE7E6850748
:10BCA000A382F400BDB5B304690383A70A0BBE9455
:10BCB00083D7C401638B37015546D2851385640051
:10BCC00097300100E780C0D955DD0509D1BD5DD8A9
:10BCD0006DB782801763FFFFE702C33E97800000C5
:10BCE000E780000C05C1C164014417A9FF1F1309B7
:10BCF00029249309400EFD1497F0FFFFE78040349C
:10BD0000634EA40017A5FF1F1305C5FF9710010080
:10BD1000E780E0031763FFFF6700033E330534034A
:10BD20008327090B3E958357C5016388970023122B
:10BD3000050097800000E780A00C050475BF97A759
:10BD4000FF1F9387E71E9C478D83858B8DE31763C9
:10BD5000FFFFE702C33817A5FF1F1305A5FA9710C9
:10BD60000100E78020031763FFFF670083398280AB
:10BD70001763FFFFE702A336970500009385C5A070
:10BD800017A5FF1F130505F897100100E78020EEA7
:10BD90001763FFFF6700E3361763FFFFE7022334F3
:10BDA0008841B7E70400BC5B0505420541818297E5
:10BDB00009C585472300F50005051763FFFF6700E8
:10BDC000433483C7F5FF2E858507A38FF5FE828058
:10BDD00083C7F5FFFD1793F7F70FA38FF5FE99EFD4
:10BDE0001763FFFFE702A32FB7E70400BC571385D3
:10BDF000F5FF82971763FFFF6700A33082801C4125
:10BE0000035745008D8FBA951CC12312B5003E859E
:10BE1000828093D78500A2051441DD8D83574500AC
:10BE20001387E6FF18C189072312F50013D6850092
:10BE30004111238FB6FEA38FC6FE410182801841B7
:10BE40009307F7FF1CC18357450085072312F500B0
:10BE5000A30FB7FE8280835745008D8F2312F50014
:10BE60001C41BE950CC12E858280AA8703D747004E
:10BE700008410D8FAA952392E7008CC38280184158
:10BE800008453305A7408280835745000357650066
:10BE90001D8F1C4108453385A7403305A74082808C
:10BEA0001763FFFFE702A32341112EC62A849700E0
:10BEB0000000E780A0FDB2456373B50001A0835781
:10BEC00044000840BE952312B4003E95410117631B
:10BED000FFFF670003231763FFFFE70243204111C1
:10BEE0002E84B28532C697000000E780A0FB324660
:10BEF000A28597300100E78000B941011763FFFF79
:10BF0000670023201763FFFFE702631D2E8485452A
:10BF100097000000E78000F9230085001763FFFF0A
:10BF20006700231E1763FFFFE702631B41112317FE
:10BF3000B100894597000000E780C0F68347E10023
:10BF40002300F5008347F100A300F50041011763CA
:10BF5000FFFF6700031B1763FFFFE702431893D738
:10BF60008500A2054111DD8D2317B1008945970099
:10BF70000000E78020F38347E1002300F5008347BA
:10BF8000F100A300F50041011763FFFF670063178D
:10BF90001763FFFFE702A3141397850193D7850169
:10BFA000C166938606F0D98F13D78500758FD98F18
:10BFB000A2053707FF00F98D4111DD8D2EC6914591
:10BFC00097000000E78000EE6C00114697300100FA
:10BFD000E78060AB41011763FFFF670083121763BF
:10BFE000FFFFE702C30F1C41854503C4070097000C
:10BFF0000000E78080E622851763FFFF670063107B
:10C000001763FFFFE702A30D1C414111894503C7D8
:10C01000070083C717002307E100A307F10097007B
:10C020000000E78080E30355E10041011763FFFF53
:10C030006700230D1763FFFFE702630A1C414111EC
:10C04000894503C7070083C717002307E100A3073B
:10C05000F10097000000E78040E08357E1004101D4
:10C0600013D58700A2075D8D420541811763FFFF4D
:10C07000670023091763FFFFE70263060C414111C4
:10C080002A841146680097300100E780C09F9145DF
:10C09000228597000000E78040DCB247C1669386A6
:10C0A00006F01397870113D58701598D13D78700A1
:10C0B000758F598DA2073707FF00F98F5D8D4101FC
:10C0C0001763FFFF6700E3031C45BE950CC1828028
:10C0D000AE87944391E6584101EF0CC15CC1828068
:10C0E00003C7570013671700A382E700B687D5B7C9
:10C0F0000CC3EDB7AA87084119CD1841D44398C3A2
:10C100006313D500D8C32A870346570093761600D9
:10C1100081E6232007008280944381CA8C4203A8D1
:10C1200047008CC363930601CCC3799A14C3A3025E
:10C13000C7003687D1BF1C45DC471D8DB777DBB6FE
:10C14000938777DB09853305F502420541818280BB
:10C15000F147B385F50248452E9582808347450017
:10C1600085072302F50082801763FFFFE70223F7AC
:10C170002A8409E41763FFFF6700A3F8834744009C
:10C18000F5DBFD1793F7F70F2302F400E5F71C44E6
:10C1900003D7270005072391E700DC4399C32285D5
:10C1A00082974C4889CD83475400898B99E71C447A
:10C1B00022859C479C439C478297232A0400004089
:10C1C000232004007DB71763FFFFE70243F1835785
:10C1D000250041112EC681EB0144228541011763E0
:10C1E000FFFF670003F2035705008147F146E305AF
:10C1F000F7FEB385D702404585072E94834544005A
:10C2000008C4F5F5B247AA8481E7232A040009A8E7
:10C210001C456C0022859C439C43829748C84DDD99
:10C2200085472312F400B24723200400231804009A
:10C230002319F4005C485CC483D72400FD172391C4
:10C24000F40061BF1763FFFFE70263E997A7FF1FD1
:10C25000938747AD88432326050023240500410525
:10C2600097100100E78000B31763FFFF670063E9E1
:10C270001763FFFFE702A3E617A4FF1F130484AAB6
:10C280001C40411199CF9C472300B5002AC65CC1D0
:10C2900097000000E78040FB1C40DC4399C3324517
:10C2A000829741011763FFFF6700A3E5034745003D
:10C2B00029E3584DAA877D551DCF1763FFFFE7027D
:10C2C00003E21CC3DC4797A6FF1F23ADE6A4F1568B
:10C2D000130507012390D7009705000093850502F9
:10C2E00097100100E780A09801451763FFFF6700E2
:10C2F00043E17D55828082801763FFFFE70223DEE2
:10C3000001116146814528009760FFFFE78020E02A
:10C3100097A7FF1F938707A19C4328009305F00F61
:10C32000DC473EC697000000E780C0F40561176354
:10C33000FFFF670003DD97A7FF1F9387A79E9C431E
:10C34000D847A1679387C702631EF70A397106DED3
:10C3500022DC26DA80004AD84ED652D456D2328514
:10C36000B28497000000E780C0C7AA89268597009D
:10C370000000E78020C92318A4FC26859700000050
:10C38000E78040C82319A4FC268597000000E780B9
:10C3900060C783D744000A8A231AA4FC858393F7D5
:10C3A000F70F230EF4FC8607BD0793F7073F330111
:10C3B000F1408A8A01498347C4FD6367F902CE854B
:10C3C000130584FC232C54FD97000000E78080EACD
:10C3D0005281130104FCF2506254D2544259B259B2
:10C3E000225A925A21618280268597000000E780B8
:10C3F00060C193171900D69705092390A7001379F8
:10C40000F90F55BF828097A7FF1F9387A7919C4381
:10C41000D847A1679387A702631AF70A397106DE26
:10C4200022DC26DA80004AD84ED652D456D2328543
:10C43000B28497000000E780C0BAAA8926859700D9
:10C440000000E78020BCFD572318A4FC2685231993
:10C45000F4FC97000000E780E0BA83D744000A8A22
:10C46000231AA4FC858393F7F70F230EF4FC8607A9
:10C47000BD0793F7073F3301F1408A8A014983479B
:10C48000C4FD6367F902CE85130584FC232C54FD9B
:10C4900097000000E78000DE5281130104FCF25097
:10C4A0006254D2544259B259225A925A216182801E
:10C4B000268597000000E780E0B493171900D6970F
:10C4C00005092390A7001379F90F55BF828097A71C
:10C4D000FF1F938727859C43D847A167890763106F
:10C4E000F70A397106DE22DC26DA80004AD84ED6F9
:10C4F00052D456D23285328997000000E78060AE70
:10C50000AA894A8597000000E780C0AF8357490099
:10C510000A8A2318A4FC858393F7F70F230CF4FCF5
:10C520008607BD0793F7073F3301F1408A8A8144AC
:10C53000834784FD63E7F402CE85130584FC232A38
:10C5400054FD97000000E780E0D25281130104FC03
:10C55000F2506254D2544259B259225A925A21612D
:10C5600082804A8597000000E780C0A99397140055
:10C57000D69785042390A70093F4F40F55BF8280CB
:10C580009797FF1F9387077A9C43D847A1679387A4
:10C59000E704631EF70A397106DE22DC26DA800022
:10C5A0004AD84ED652D456D23285B2849700000073
:10C5B000E78020A3AA89268597000000E78080A451
:10C5C0002318A4FC268597000000E780A0A3231A67
:10C5D000A4FC268597000000E780C0A283D7440012
:10C5E0000A8A2319A4FC858393F7F70F230EF4FC22
:10C5F0008607BD0793F7073F3301F1408A8A014957
:10C600008347C4FD6367F902CE85130584FC232CA0
:10C6100054FD97000000E780E0C55281130104FC3F
:10C62000F2506254D2544259B259225A925A21615C
:10C630008280268597000000E780C09C9317190030
:10C64000D69705092390A7001379F90F55BF82806B
:10C650009797FF1F9387076D9C43D847A1679387E0
:10C66000C704631AF70A397106DE22DC26DA800075
:10C670004AD84ED652D456D23285B28497000000A2
:10C68000E7802096AA89268597000000E78080979A
:10C69000FD572318A4FC2685231AF4FC97000000FC
:10C6A000E780409683D744000A8A2319A4FC858337
:10C6B00093F7F70F230EF4FC8607BD0793F7073FA8
:10C6C0003301F1408A8A01498347C4FD6367F90257
:10C6D000CE85130584FC232C54FD97000000E780D1
:10C6E00060B95281130104FCF2506254D254425991
:10C6F000B259225A925A2161828026859700000001
:10C70000E780409093171900D69705092390A7005A
:10C710001379F90F55BF82809797FF1F9387876022
:10C720009C43D847A167DD076317F7041763FFFF32
:10C73000E702E39A79713285328497000000E7803E
:10C74000408A2AC6228597000000E780A08B23112B
:10C75000A102228597000000E780A088B24523004F
:10C76000A102280897000000E780C0B04561176368
:10C77000FFFF6700039982809797FF1F9387875A6F
:10C780009C43D847A167938787046317F70417630F
:10C79000FFFFE702C394797132853284970000006D
:10C7A000E78020842AC6228597000000E7808085E4
:10C7B0002311A102228597000000E7808082B24504
:10C7C0002300A102280897000000E780A0AA456185
:10C7D0001763FFFF6700E39282809797FF1F93879D
:10C7E00067549C43D847A1679387A7046312F70255
:10C7F0001763FFFFE702A38E011128008145970010
:10C800000000E78020A705611763FFFF6700638FC3
:10C8100082809797FF1F9387E7509C43D847A16773
:10C82000938757026319F7021763FFFFE702238B11
:10C830000111328597F0FFFFE780A07A2308A1005D
:10C840008145280097000000E780C0A205611763BA
:10C85000FFFF6700038B82809797FF1F9387874CAA
:10C860009C43D847A1679387E702631BF7041763CC
:10C87000FFFFE702C38601113285328497F0FFFF84
:10C88000E7804078AA84228597F0FFFFE7808077D1
:10C89000854709E9228597F0FFFFE780807442050C
:10C8A000B337A00028008145231891003ECA9700A5
:10C8B0000000E780209C05611763FFFF6700638429
:10C8C00082809797FF1F9387E7459C43D8479947F6
:10C8D0006313F7081763FFFFE702638079713285FE
:10C8E000328497F0FFFFE780C06F2AC6228597F059
:10C8F000FFFFE78020712310A102228597F0FFFF40
:10C90000E780206E2301A102228597F0FFFFE780D8
:10C91000406DA301A102228597F0FFFFE780606CC4
:10C920002302A102228597F0FFFFE780806B23138B
:10C93000A102228597F0FFFFE780A06AB245231489
:10C94000A102280897000000E780C09245611753B4
:10C95000FFFF6700037B82809797FF1F9387873CC9
:10C960009C43D847A1679387C7036313F7081753FE
:10C97000FFFFE702C37679713285328497F0FFFFBB
:10C98000E78020662AC6228597F0FFFFE780806750
:10C990002310A102228597F0FFFFE780A0662311F4
:10C9A000A102228597F0FFFFE780A0632302A10286
:10C9B000228597F0FFFFE780C062A302A1022285D3
:10C9C00097F0FFFFE780E0612303A102228597F043
:10C9D000FFFFE7800061B245A303A102280897008A
:10C9E0000000E780208945611753FFFF67006371EE
:10C9F00082801753FFFFE702836E01112A8497F0AC
:10CA0000FFFFE780005EAA84228597F0FFFFE780A2
:10CA1000605F228597F0FFFFE780C05E0357440008
:10CA20008D4763F7E700228597F0FFFFE780805D81
:10CA3000228597F0FFFFE780E05C2800A68597003D
:10CA40000000E780208305611753FFFF6700636BD9
:10CA50009797FF1F9387072D9C43D847A167FD0732
:10CA6000631FF7001753FFFFE702636732859700E4
:10CA70000000E78040F81753FFFF6700836882805B
:10CA80009797FF1F9387072A9C43D847A167E5071D
:10CA90006315F7081753FFFFE70263647971328566
:10CAA000328497F0FFFFE780C0532AC6228597F0B3
:10CAB000FFFFE7802055228597F0FFFFE780805435
:10CAC0002310A102228597F0FFFFE780A0535205B3
:10CAD00051812311A10222852302010297F0FFFF59
:10CAE000E7802050A302A102228597F0FFFFE78094
:10CAF000404F2303A102228597F0FFFFE780604E9D
:10CB0000B245A303A102280897F0FFFFE7808076D3
:10CB100045611753FFFF6700C35E82809797FF1F31
:10CB2000938747209C43D847A1679387E703631FF8
:10CB3000F7001753FFFFE702835A32859700000082
:10CB4000E78060EB1753FFFF6700A35B8280979736
:10CB5000FF1F9387271D9C43D847A16793874704EE
:10CB6000631EF7021753FFFFE7026357797132859F
:10CB7000328497F0FFFFE780C0462AC6228597F0EF
:10CB8000FFFFE7802048B245280897F0FFFFE780C5
:10CB9000606E45611753FFFF6700A3568280979729
:10CBA000FF1F938727189C43D847A1679387870265
:10CBB0006310F7041753FFFFE70263527971328560
:10CBC000328497F0FFFFE780C0412AC6228597F0A4
:10CBD000FFFFE7800041B2452300A102280897F03B
:10CBE000FFFFE780206945611753FFFF670063512E
:10CBF00082801753FFFFE702834E011197F0FFFF7A
:10CC0000E780203EAA85280097F0FFFFE780806636
:10CC100005611753FFFF6700C34E9797FF1F938768
:10CC200067109C43D847A167D107631FF7001753CC
:10CC3000FFFFE702C34A328597000000E780A0FBB0
:10CC40001753FFFF6700E34B82809797FF1F93877F
:10CC5000670D9C43D847A167C507631FF7001753AB
:10CC6000FFFFE702C347328597000000E780A0F886
:10CC70001753FFFF6700E34882809797FF1F938752
:10CC8000670A9C43D847A167B907631FF70017538A
:10CC9000FFFFE702C344328597000000E780A0F55C
:10CCA0001753FFFF6700E34582809797FF1F938725
:10CCB00067079C43D847A167AD07631FF700175369
:10CCC000FFFFE702C341328597000000E780A0F232
:10CCD0001753FFFF6700E34282809797FF1F9387F8
:10CCE00067049C43D84789476318F7021753FFFF2F
:10CCF000E702E33E0111328532C897F0FFFFE7807B
:10CD0000402EAA85280097F0FFFFE780A056056116
:10CD10001753FFFF6700E33E82809797FF1F9387BB
:10CD200067009C43D847A1678D076311F704175329
:10CD3000FFFFE702C33A01113285328497F0FFFF0B
:10CD4000E780202A13066100AA844C0022859730D0
:10CD50000000E780C0232800A68597F0FFFFE7804A
:10CD6000605105611753FFFF6700A33982809797D1
:10CD7000FF1F938767FB9C4381CFDC4391CB175305
:10CD8000FFFFE702C33582971753FFFF6700633742
:10CD900082801753FFFFE702833479713C08AE8429
:10CDA0003ED2A165B7070A002A843ED448103C0849
:10CDB000DD053ED636C432C63AC297D0FFFFE780C3
:10CDC000E02F12474810BA8597F0FFFFE780C013A5
:10CDD00032464810B28597F0FFFFE780E014A24684
:10CDE0004810B68597F0FFFFE7800012501001470A
:10CDF0008146A685228597D0FFFFE7808051456157
:10CE00001753FFFF6700E32F1753FFFFE702232DA0
:10CE100001117C000329C501AE843ECAA165B70794
:10CE200007002A843ECC48087C00C5053ECE97D03A
:10CE3000FFFFE780A0288345D900480897F0FFFF4F
:10CE4000E780800C500801478146A685228597D04F
:10CE5000FFFFE780004C05611753FFFF6700632A5F
:10CE60001753FFFFE702A32783C7950093F7F70740
:10CE7000A384F50097000000E78040F91753FFFFF7
:10CE8000670023281753FFFFE702632579713C08E9
:10CE9000AE843ED2A165B70709002A843ED448106B
:10CEA0003C08938545043ED632C636C497D0FFFF72
:10CEB000E780C020A2464810B68597F0FFFFE780C4
:10CEC000A00432464810B28597F0FFFFE780C00506
:10CED000501001478146A685228597D0FFFFE78045
:10CEE000404345611753FFFF6700A3211753FFFF1E
:10CEF000E702E31E83C7950041112A8493F7F707E1
:10CF0000A384F50032852EC697F0FFFFE780800FDF
:10CF100085672AC46370F50297700000E78020E9F6
:10CF20002246B24509ED114781462285970000004F
:10CF3000E78060E641011753FFFF6700831C01474C
:10CF40008346F501DDB71753FFFFE702A317011171
:10CF50003C003ECAB7070A003ECC3C003ECE83C729
:10CF60009500AA89328593F7F707A384F5002E84EC
:10CF700097F0FFFFE78000098567637DF504A165F1
:10CF8000AA8493858504480897D0FFFFE7800013A3
:10CF9000268597700000E78080E12A8929E1914584
:10CFA000480897F0FFFFE78020F6A685480897F02D
:10CFB000FFFFE78060F7CA85480897F0FFFFE7802A
:10CFC000A0F4014781465008A2854E8597D0FFFF07
:10CFD000E780203405611753FFFF6700E3118145A7
:10CFE000480897F0FFFFE78020F20349090275BF68
:10CFF0001753FFFFE702030D79711C103ECAB707F4
:10D000000F003ECC404D1C10AA84AE8948089945BB
:10D0100032C636893ECE97D0FFFFE780200A3246DF
:10D020004808B28597F0FFFFE78000EE630C090225
:10D03000A545480897F0FFFFE780C0E62546CA856A
:10D0400097200100E78020A4500801478146CE8543
:10D05000268597D0FFFFE780C02B45611753FFFF60
:10D06000670083098355C402480897F0FFFFE780F3
:10D07000A0EB0355E402814505C58547854563015D
:10D08000F502C167FD179305F00F630BF5007D15E1
:10D0900097700000E780208E9305150093F5F50F3B
:10D0A000480897F0FFFFE78020E68345040348081F
:10D0B00097F0FFFFE78040E583451403480897F0A9
:10D0C000FFFFE78060E483552403480897F0FFFFE3
:10D0D000E78080E583554403480897F0FFFFE78029
:10D0E000A0E49DB71753FFFFE70263FF83C79500D6
:10D0F0008146014693F7F707A384F50097000000E7
:10D10000E78040EF1753FFFF6700A3FF1753FFFFB0
:10D11000E702E3FC79713E841C103ECA2E89B707F2
:10D120000F00A1653ECCFD051C10AA84480842C032
:10D130003AC23ECE36C432C697D0FFFFE78000F831
:10D1400032464808B28597F0FFFFE780E0DBA24651
:10D150004808B68597F0FFFFE78000DD12474808D2
:10D16000BA8597F0FFFFE78020DC0248630C0802D5
:10D170009145480897F0FFFFE780C0D21146A2858D
:10D1800097200100E7802090500801478146CA851A
:10D19000268597D0FFFFE780C01745611753FFFF33
:10D1A000670023F68945480897F0FFFFE78080CFA6
:10D1B000834704002300F50083471400A300F50013
:10D1C000E1B71753FFFFE702E3EF83C795000111B3
:10D1D0002A8A93F7F707A384F5003285AE8432C616
:10D1E00097F0FFFFE78000E232462A89328597F008
:10D1F000FFFFE78000DF85676373F902AA894A852C
:10D2000097700000E780A0BA2A8419ED1147814683
:10D210004A86A685528597000000E780C0B7056161
:10D220001753FFFF670043ED9387E9FF93F7F70F6D
:10D230000547E366F7FE8347F50195EB8947E380F1
:10D24000F9FE8346F401528501474A86A685970078
:10D250000000E78040B4A167D90748083ECC230A04
:10D26000010002CE97000000E780A0B04DBF639E92
:10D27000E7008947639EF90093071020231FF500FC
:10D2800097700000E780C0B76DBF0947E39BE7FADE
:10D290008D47E398F9FA228597700000E78080DFD8
:10D2A0009797FF1F938747C79C4399E79797FF1F5F
:10D2B000938747B09C4399C703D50400978000002B
:10D2C000E780A0CE231F040022855DBF1753FFFF18
:10D2D000E702E3E001113C003ECAB7070B003ECC79
:10D2E0003C003ECE83C795002A89328593F7F70725
:10D2F000A384F500AE8497F0FFFFE780A0D09317DA
:10D300000501C187635AF006A1652A849385E50269
:10D31000480897D0FFFFE78060DAA285480897F0B9
:10D32000FFFFE78060C09797FF1F9387A7A89C43E4
:10D33000A9EB01449375F40F480897F0FFFFE780CD
:10D34000A0BC9355844093F5F50F480897F0FFFF74
:10D35000E78080BB9355044193F5F50F480897F09B
:10D36000FFFFE78060BA014781465008A6854A85DD
:10D3700097D0FFFFE780E0F905611753FFFF6700D3
:10D3800043D8416585460546A2857D159750000026
:10D39000E78060BD59DD510597000100E780808F6F
:10D3A000130440063344850271B71753FFFFE702A9
:10D3B00003D30111B70706003EC683C79500216459
:10D3C0002A8993F7F707A384F500AE842800930514
:10D3D000A4040AC40AC897D0FFFFE78020CE30001B
:10D3E00001478146A6854A8597D0FFFFE78060F216
:10D3F00097E0FFFFE780801513049404480822CCCF
:10D40000230A010002CE97000000E78080960561A4
:10D410001753FFFF6700E3CE1753FFFFE70283CAEE
:10D42000C1642A8901449799FF1F938969B0130A3F
:10D430008002FD1497E0FFFFE78080C16347A400EE
:10D4400001451753FFFF670023CBB307440303A72E
:10D45000C90ABA9703D707006306970083D7270046
:10D46000638427010504F9B70545E1BF1753FFFFA2
:10D47000E70243C52A8A2E8999C123A00500814964
:10D480008144979AFF1F938A6A8A614B97E0FFFF56
:10D49000E78040C263C7A4004E851753FFFF6700B3
:10D4A000A3C53384640383A70A003E948357040012
:10D4B00099E763040900232089008504C1BF414620
:10D4C000D2851305440097100100E780605975F577
:10D4D000A289E5B71753FFFFE702C3BE39717C0885
:10D4E0003ED4B7070A003ED67C083ED883C79500D5
:10D4F0002A8A328593F7F707A384F5002E8932C66E
:10D5000097F0FFFFE78000B085676373F508324648
:10D51000AA84328597F0FFFFE780A0AC8547AA89EF
:10D5200063E8A706A16593858504281097D0FFFFBF
:10D53000E780C0B8268597700000E78040872A847E
:10D5400029ED9145281097F0FFFFE780E09BA68525
:10D55000281097F0FFFFE780209DCE85281097F0D8
:10D56000FFFFE780609A014781463010CA855285E7
:10D5700097D0FFFFE780E0D9A16793877704481829
:10D580003EDC230A010202DE97F0FFFFE780607EA7
:10D5900021611753FFFF670023B68145281097F0DC
:10D5A000FFFFE7806096A685281097F0FFFFE780D1
:10D5B000A0979797FF1F938727CE9C4381CB228507
:10D5C0006389090097D00000E78040248345040266
:10D5D00071B797D00000E780C022CDBF1753FFFF7F
:10D5E000E70243AE83C795004111AA8993F7F70775
:10D5F000A384F5003285AE84328A97F0FFFFE7807E
:10D6000060A08567637FF5022A8997600000E78044
:10D61000007A2A84914631C58347F501054763871F
:10D62000E70291C70D476366F704AD461DA8930551
:10D63000050303250A00414697100100E780404298
:10D640000DE941011753FFFF670003AB93059508F0
:10D6500003250A00414697100100E780604081469B
:10D6600069F54A86A6854E8597000000E780C0814F
:10D67000C9BF83250A001305940897700000E7804E
:10D68000A02919C1C146F1BF9797FF1F9387C7888B
:10D690009C4399E79787FF1F9387C7719C4399C75E
:10D6A000228597800000E780208A69FD8547A30FC7
:10D6B000F400228597B00000E7806084228597609F
:10D6C0000000E780E0734E8581464A86A68597F084
:10D6D000FFFFE780607BA1679387570448003EC443
:10D6E0002302010002C697F0FFFFE780806891BF28
:10D6F0001753FFFFE702239C83C795004111AA89B6
:10D7000093F7F707A384F50032852E89B28A97F044
:10D71000FFFFE780208F85676374F50EAA8497600A
:10D720000000E780C0682A840DED416B014A978BA9
:10D73000FF1F938BEB7F130C400E7D1B19A8330446
:10D740008A0383A70B0B3E948357C4016383670549
:10D75000050A97E0FFFFE780A08EE342AAFE954608
:10D760000DA08357C501639697029305050303A592
:10D770000A00414697100100E780802E994611E18A
:10D7800081462686CA854E8597F0FFFFE780C06FE9
:10D7900085A883A50A001305040397700000E7809D
:10D7A000A017C14679FD2285231E940097A0000092
:10D7B000E780E074228597600000E78060649797B7
:10D7C000FF1F938767AD9C43A9C3230004022285F2
:10D7D00097D00000E78040F04E8581462686CA85B6
:10D7E00097F0FFFFE780406AA1679387070448002E
:10D7F0003EC42302010002C697F0FFFFE780605796
:10D8000041011753FFFF6700838E89472300F4020D
:10D81000E1B7397106DE22DC4AD8800052D456D2F4
:10D820005AD026DA4ED65ECE2E8A32892A8B97D0EF
:10D83000FFFFE780E07D0605710541998A8A330183
:10D84000A140232224FC231404FC97D0FFFFE7808F
:10D85000207C83479A000605350593F7F7072315C3
:10D86000A4FCA304FA004A85232624FC97E0FFFFCA
:10D87000E780407993170501C1876340F002568124
:10D88000130104FCF2506254D2544259B259225A44
:10D89000925A025BF24B21618280AA844A8597E00A
:10D8A000FFFFE7802076AA894A8597E0FFFFE7809F
:10D8B0006075A1659385C5022A89130544FC97C04C
:10D8C000FFFFE780A07F268597C0FFFFE780E0731A
:10D8D000854511C94A86CE8597C0FFFFE780606DF8
:10D8E000AA8B21E98945130544FC97E0FFFFE780F7
:10D8F000A061A685130544FC97E0FFFFE780C062A6
:10D90000CE85130544FC97E0FFFFE780E061CA8500
:10D91000130544FC97E0FFFFE78000610147814663
:10D92000130644FCD2855A8597D0FFFFE780609E9E
:10D93000B9B78145130544FC97E0FFFFE780C05C61
:10D94000A685130544FC97E0FFFFE780E05DCE85E8
:10D95000130544FC97E0FFFFE780005DCA851305CF
:10D9600044FC97E0FFFFE780205C814497D0FFFFF5
:10D97000E780006AE3D4A4FA83A70B01139714008D
:10D98000BA9783D5070099C5130544FC97E0FFFFBC
:10D99000E78080598504D9BF797106D622D44AD050
:10D9A00000184ECE52CC56CA26D25AC8AE893289F9
:10D9B000AA8A97D0FFFFE780A0650605690541990F
:10D9C0000A8A3301A140232A24FC231C04FC97D09B
:10D9D000FFFFE780E06383C7990006052D0593F7F5
:10D9E000F707231DA4FCA384F9004A85232E24FCF9
:10D9F00097E0FFFFE780006193170501C187634F40
:10DA0000F0005281130104FDB25022549254025985
:10DA1000F249624AD24A424B45618280AA844A85D1
:10DA200097E0FFFFE780005EA1659385A5022A8944
:10DA3000130544FD97C0FFFFE7804068268597C027
:10DA4000FFFFE780805C854509C9CA8597C0FFFF55
:10DA5000E78020592A8B29E18945130544FD97E089
:10DA6000FFFFE780604AA685130544FD97E0FFFFAE
:10DA7000E780804BCA85130544FD97E0FFFFE780F0
:10DA8000A04A01478146130644FDCE85568597D0AE
:10DA9000FFFFE7800088B5B78145130544FD97E097
:10DAA000FFFFE7806046A685130544FD97E0FFFF72
:10DAB000E7808047CA85130544FD97E0FFFFE780B4
:10DAC000A046814497D0FFFFE7808054E3DBA4FAAF
:10DAD00083270B0113971400BA9783D5070099C5C4
:10DAE000130544FD97E0FFFFE78000448504D9BF9C
:10DAF0001743FFFFE702A35E83474500404DD5EF84
:10DB0000FD575DC48346940009476363D70A034603
:10DB1000B400854663EEC6088306E40063CA0608BF
:10DB20005C45F9562390D7009787FF1F83C747208E
:10DB300099E3A304E4009787FF1F9387A7279C43DB
:10DB400081E78947A306F4009787FF1F9387C7746F
:10DB50009C4381E789472306F400970500009385DD
:10DB60004506AA841305040197F00000E780201001
:10DB7000FD57231AF40281471CDC01489787FF1FD9
:10DB800023A4871A9787FF1F9387471A232E04031E
:10DB900004C0804397D0FFFFE780C0516146330641
:10DBA000C502814522859740FFFFE78040568147A7
:10DBB0003E851743FFFF6700C354FD57D5BF17438A
:10DBC000FFFFE702C3512A84035545029760000016
:10DBD000E780E01D19E5231E04001743FFFF6700DF
:10DBE00043528357E401F5DB930504FF1745010019
:10DBF000130585E397E00000E780E014F9BF1743C1
:10DC0000FFFFE702C34D2E89A16541119385E5030E
:10DC10002A8436C432C6BE843AC297C0FFFFE7806A
:10DC2000E04912472285BA8597E0FFFFE780C02DC3
:10DC300032462285B28597E0FFFFE780E02EA246BC
:10DC40002285B68597E0FFFFE780002E6303090277
:10DC50009145228597E0FFFFE780C0241146A68505
:10DC600097100100E78020E241011743FFFF6700A2
:10DC700043498945228597E0FFFFE780A02283C7BB
:10DC800004002300F50083C71400A300F500E9BFDA
:10DC90001743FFFFE702A34483C79500444D0547A0
:10DCA00093F7F707A384F5001C42411183C70700CF
:10DCB0006367F7062E842A89B1C003C7D400630FB7
:10DCC000F7021787FF1F1307E70E184305C3A38644
:10DCD000F40097A00000E780404A83C7D40099E78A
:10DCE00041657D1597400000E780403083D72403CD
:10DCF000918B89C797E00000E780C0134A85A28511
:10DD000097F0FFFFE7808010A167C10748003EC47D
:10DD10002302010002C697F0FFFFE7808005410162
:10DD20001743FFFF6700E33D1743FFFFE702233B75
:10DD300003D745008D47AA8441112E8432892E8550
:10DD400063E3E70297E0FFFFE780C02BAA8523008B
:10DD50000900268597C0FFFFE780A02841011743EF
:10DD6000FFFF6700033A97E0FFFFE780A0292AC67C
:10DD7000228597E0FFFFE780E028B24585472A86A5
:10DD80002300F900268597C0FFFFE7808022F9B7BE
:10DD9000397106DE22DC26DA80004ED652D456D205
:10DDA0004AD85AD05ECEAE89B284AA8A97D0FFFFF5
:10DDB000E780002506051305250241990A8A3301EB
:10DDC000A140232224FC231404FC97D0FFFFE7800A
:10DDD000202383C7990006054D0593F7F707231500
:10DDE000A4FCA384F9002685232624FC97E0FFFFEA
:10DDF000E780402193170501C1876340F0025281FB
:10DE0000130104FCF2506254D2544259B259225ABE
:10DE1000925A025BF24B21618280AA8B03AB040011
:10DE200097C0FFFFE780601E51E583D7440001499A
:10DE30008544F11793B71700A301F4FC834734FC22
:10DE4000A165C9C79385E504130544FC97C0FFFF8E
:10DE5000E780C026A685130544FC97E0FFFFE78016
:10DE6000A00ADE85130544FC97E0FFFFE780C00BA6
:10DE7000834734FC114691E30946DA85130544FCD7
:10DE800097E0FFFFE78060058144630A0900416B6A
:10DE90007D1B97D0FFFFE780A01663CCA40201474B
:10DEA0008146130644FCCE85568597C0FFFFE78068
:10DEB0004046B1B7A685130634FC97000000E78002
:10DEC000E0E6933415002A8986048DBF9385C50446
:10DED000A5BF8327C90013971400BA9783D50700FD
:10DEE00063886501130544FC97E0FFFFE780C003EA
:10DEF000850445B71743FFFFE702E31B79711C1048
:10DF00003EC4B7070F003EC61C103EC883C795002D
:10DF1000AA8A328593F7F707A384F500AE89328485
:10DF200097E0FFFFE780000E93170501C187635A52
:10DF3000F0062A8A228597E0FFFFE780A00C2A8955
:10DF40005285032B040097C0FFFFE780000C39EDDA
:10DF50008357440081440544F11793B71700A30386
:10DF6000F10083457100DA872287CA86528628002D
:10DF700097000000E780E0C8014781463000CE8569
:10DF8000568597C0FFFFE780C038A1679387D70306
:10DF900048083ECC230A810026CE97F0FFFFE78099
:10DFA00040DD45611743FFFF67006314A285130638
:10DFB000710097000000E78060D7AA84094455D11A
:10DFC0003544E30055FB4A8597F0FFFFE7800045A5
:10DFD0000D4441D9014497D0FFFFE7806002634DB3
:10DFE000A400C16B0144FD1B97D0FFFFE7804001F7
:10DFF000634EA4001544B5B7DC4413171400BA9758
:10E0000083D70700638327030504F1B7D844931728
:10E010001400BA9703D70700631B770123902701E9
:10E02000268597A00000E78080DB01441DBF050422
:10E0300065BF1743FFFFE702E30883C7950041115F
:10E040002A8A93F7F707A384F50032852E89328454
:10E0500097E0FFFFE78000FB93170501C18763533B
:10E06000F006AA89228597E0FFFFE780A0F9231137
:10E07000A1004E85832A040097C0FFFFE780E0F8E7
:10E0800039E58357440085440144F11793B71700DD
:10E09000A300F1000348110003572100D6875285E1
:10E0A000CE862686CA8597F0FFFFE7806006A167C7
:10E0B000F10748003EC42302910022C697F0FFFFFB
:10E0C000E78020CB41011743FFFF6700E302A285F1
:10E0D0001306110097000000E78040C52A84894498
:10E0E00055D98357210011678544BA97C207116734
:10E0F000C1831307F7EFE36FF7F89787FF1F938745
:10E10000A7E19C4381CB8545130521009750000072
:10E11000E7802075835521002285814497C0FFFF49
:10E12000E78040E525D923100500228597A000004F
:10E13000E78040CD85B71743FFFFE702C3F783C7EA
:10E14000950041112A8B93F7F707A384F5003285D8
:10E150002E8A328497E0FFFFE780C0EA931705011B
:10E16000C1876351F006AA8A228597E0FFFFE78006
:10E1700060E92A895685832B040097C0FFFFE7805A
:10E18000C0E831E58357440081440544F11793B753
:10E190001700A301F10003483100DE875A854A8742
:10E1A000D6862286D28597F0FFFFE78060F6A167CA
:10E1B000ED0748003EC42302810026C697F0FFFF0A
:10E1C000E78020BB41011743FFFF670043F2A285B0
:10E1D0001306310097000000E78040B5AA84094487
:10E1E0005DD99167CA97C2071167C1831307F7EF1B
:10E1F0000544E362F7FACA8597C0FFFFE78080D73E
:10E20000014451F9814997D0FFFFE78060E063DB6B
:10E21000A900984893971900BA9703D7070005EF0C
:10E220002390270197D0FFFFE78080DE1544E38429
:10E23000A9F6268597A00000E780C0BC9787FF1F3E
:10E24000938787CD9C430144B9D74A8597500000F6
:10E25000E780C05889B785097DB71743FFFFE702FC
:10E2600063E679713E847C083EC82E8AB7071400A5
:10E27000A1653ECAE5057C08AA89080836C442891A
:10E2800032C6BA8AC6843ECC97C0FFFFE78000E35F
:10E29000CA85080897E0FFFFE78000C732460808F4
:10E2A000B28597E0FFFFE78020C8A246630A090411
:10E2B0009D45080897E0FFFFE780C0BE1D468145E9
:10E2C0009740FFFFE780A0E463890A0891450808AA
:10E2D00097E0FFFFE78000BD1146A685970001008B
:10E2E000E780607A100801478146D2854E8597C045
:10E2F000FFFFE780000245611743FFFF6700C3DFB0
:10E30000B685080897E0FFFFE78000C21C400808B8
:10E31000D8439355C701858912075183B205D98D1A
:10E3200097E0FFFFE78040C01C40080883C58700D6
:10E3300097E0FFFFE78040BD1C40080883C5A700A9
:10E3400097E0FFFFE78040BC1C40080883C59700AA
:10E3500097E0FFFFE78040BB85BF8945080897E04D
:10E36000FFFFE78020B483C704002300F50083C7C4
:10E370001400A300F500BDB71743FFFFE70283D4E5
:10E3800083C795004111AA8993F7F707A384F50085
:10E390003285AE84328497E0FFFFE780A0C69317F2
:10E3A0000501C187635DF0042A89032A040097C030
:10E3B000FFFFE78080C519E9835744000548F1173E
:10E3C00093B71700A307F100814631A81306F100A7
:10E3D000A28597000000E78060951DC51C459DC77C
:10E3E00083D6470001480347F10093078500D28890
:10E3F0004A86A6854E8597000000E78040E64101E9
:10E400001743FFFF670043CF09487DBF1D486DBF1D
:10E410001743FFFFE70203CB65715C083EC4B707F3
:10E420007B013EC65C083EC883C795002A8A3285B8
:10E4300093F7F707A384F500AE8997E0FFFFE78025
:10E4400040BA8357E100E1C78945280097C0FFFF24
:10E45000E780C0C68145280097E0FFFFE780C0AA9B
:10E4600097C0FFFFE780A0CC9787FF1F9387C7E285
:10E470009C431784FF1F0344A48BAA843334800079
:10E4800099C3136424009787FF1F9387A7929C4327
:10E4900099C3136444009787FF1F9387E7A79C43A2
:10E4A00099C31364840083D504002800014997E0D0
:10E4B000FFFFE78060A783D52400280097E0FFFFD7
:10E4C000E78080A683D54400280097E0FFFFE7801F
:10E4D000A0A597D0FFFFE780A0AE93150501C181ED
:10E4E000280097E0FFFFE78020A4A285280097E09E
:10E4F000FFFFE78060A39C446360F9020147814607
:10E500003000CE85528597C0FFFFE78080E05961DB
:10E510001743FFFF670043BEDC4413144900280083
:10E520003E9497E0FFFFE7806096834744000347EF
:10E53000540089070607BA978607E36AF5FC8355F6
:10E5400024002800814A97E0FFFFE780E09D834593
:10E550004400280097E0FFFFE780009B83455400BC
:10E56000280097E0FFFFE780209A8347440063C9B3
:10E57000FA00814A8347540063C1FA020509A5BF26
:10E580001C4413975A002800BA9783D50700850AC0
:10E5900097E0FFFFE7804099C9BF032BC400939722
:10E5A0005A0028003E9B83552B00850A97E0FFFF09
:10E5B000E780809783550B00280097E0FFFFE780F6
:10E5C000A0964DBF1743FFFFE70263B15C4993E795
:10E5D00017005CC997A00000E78020B61743FFFF33
:10E5E000670023B21743FFFFE70263AF2E84814524
:10E5F00097F0FFFFE780C0E705C583570500FD17CB
:10E600002310F50009C4835725002310F400970058
:10E610000000E78060FB01451743FFFF670063AE22
:10E6200031457DD823100400C5BF1743FFFFE70223
:10E6300063A983C7950041112A8A93F7F707A3843A
:10E64000F50032852E89328497E0FFFFE780809BBA
:10E6500093170501C1876356F006AA89C145228533
:10E6600097E0FFFFE780A0802A8B4E85832A040075
:10E6700097C0FFFFE780609931E983574400231179
:10E6800001000544F11793B71700A300F10081447E
:10E690000348110003572100D6875285CE86228673
:10E6A000CA8597F0FFFFE780A0A6A16793871702AE
:10E6B00048003EC42302810026C697E0FFFFE780A2
:10E6C000406B41011743FFFF670003A313061100CE
:10E6D000A28597F0FFFFE7806065AA8409E5231112
:10E6E0000100094475B7930521005A859700000081
:10E6F000E78080EF835721002A84D9DB9787FF1FAB
:10E70000938787819C4381CB8545130521009750D2
:10E710000000E7800015835521002685314497C00D
:10E72000FFFFE78020852DD52310050026859790D3
:10E730000000E780206D0144A1BF1743FFFFE702FF
:10E74000039A41112E896C00AA8402C697F0FFFF3C
:10E75000E78000D20DC10357050005072310E5002F
:10E7600097000000E78040E681473E85410117435E
:10E77000FFFF670003993247954765DBCA85268509
:10E7800097300000E780400DC147E34005FE32446A
:10E79000854741462310F40083570900A6851305D9
:10E7A00044002311F40097000100E780C02D22856A
:10E7B00045BF1743FFFFE702E39083C79500411170
:10E7C000AA8A93F7F707A384F5003285AE893284CD
:10E7D00097E0FFFFE780008393170501C187635629
:10E7E000F0062A8AC145228597D0FFFFE78020687E
:10E7F000AA845285032B040097C0FFFFE780E080C6
:10E8000031E983574400231101008544F11793B780
:10E810001700A300F1000144034811000357210031
:10E82000DA875685D2862686CE8597F0FFFFE78069
:10E83000208EA1679387070248003EC423029100FF
:10E8400022C697E0FFFFE780C05241011743FFFF58
:10E850006700838AA2851306110097F0FFFFE78007
:10E86000E04C2A8409E523110100894475B7268507
:10E870009305210097000000E78060ECAA8449FD21
:10E8800083552100228597B0FFFFE780A06E49F5F0
:10E89000014997C0FFFFE780A077635DA900184892
:10E8A00093171900BA9703D707000DEF03572100FC
:10E8B0002390E70097C0FFFFE7808075630625037C
:10E8C0009777FF1F938747659C4399C7035521009E
:10E8D00097500000E78080F0228597900000E78045
:10E8E00060521DBF050975B795443DB705C1930733
:10E8F000F00F630FF500C547630CF5009307F5FFB4
:10E9000005453315F500420541818280014582802D
:10E9100041657D158280B9E91733FFFFE702237C4B
:10E9200003450603328497000000E78060FC9305EE
:10E93000803EB305B502C205C18181CD0357E40213
:10E94000854763F8E7001305040197E00000E780BE
:10E9500020428357E40241677D176385E700FD1776
:10E960002317F4021733FFFF6700A3798280173360
:10E97000FFFFE7024374004283C79500444D0349FB
:10E98000140093F7F707A384F500834704002209D6
:10E9900011673369F900A167B347F90041112A8B68
:10E9A000AE8A63ECE70E834724001307C00EB91745
:10E9B00093F7F70F6373F71003473400C14763EE13
:10E9C000E70E834744001307E00793C70708637106
:10E9D000F70C8349840083477400A209B3E9F90066
:10E9E000856763F7F90A034A6400834754004E853C
:10E9F000220A336AFA0097500000E780403B61C169
:10EA000023962403834B3400137AFA00239A3403A9
:10EA1000238874032399440393890401631C090028
:10EA200023A60402239804024E8597E00000E780A5
:10EA300060363DA0034924004A8597000000E78026
:10EA400020EB2397A402834744004E85A388F40259
:10EA5000E38D0BFCE30B09FC97E00000E780202F1F
:10EA600097900000E780007381460146D6855A855D
:10EA700097E0FFFFE7800058A167938797033EC4A4
:10EA800023020100480002C697E0FFFFE780602EE6
:10EA900041011733FFFF670083658544A286268600
:10EAA000D6855A8597E0FFFFE780C054A16793871A
:10EAB00097033EC423029100F1B7BD44C5B791440A
:10EAC000F1BF1733FFFFE702E35F01111C08404D60
:10EAD0003EC2B7070F003EC41C083EC62A89AE8955
:10EAE00097C0FFFFE780A0DA585C1C5C6346B70E56
:10EAF0006394E50063E2A70E3385A740B3B7A70090
:10EB0000B305B7401306803E81469D8D97000100F6
:10EB1000E78080B793140501C180A1659385C50383
:10EB2000480097B0FFFFE78060598145480097D0C3
:10EB3000FFFFE780603D83550404480097D0FFFF46
:10EB4000E780803E83552404480097D0FFFFE7808C
:10EB5000A03D814589CCC167FD179305F00F6388FF
:10EB6000F400268597500000E780E0E0AA85480081
:10EB700097D0FFFFE780403903554404814501CD1C
:10EB8000C167FD179305F00F6307F500975000006C
:10EB9000E78060DEAA85480097D0FFFFE780C03697
:10EBA00083456404480097D0FFFFE780E035834544
:10EBB0007404480097D0FFFFE780003550000147FC
:10EBC0008146CE854A8597B0FFFFE7808074056156
:10EBD0001733FFFF67004352814481B71733FFFFAC
:10EBE000E702E34F83C7950093F7F707A384F50087
:10EBF00097000000E78020ED1733FFFF67006350A8
:10EC00001733FFFFE702034C83C795004111404DC6
:10EC100093F7F707A384F5002A8A3285B284AE8978
:10EC200097D0FFFFE780003E2A8B268597D0FFFF15
:10EC3000E780403D2A89268597D0FFFFE780603A2C
:10EC400093170B0163CA0702E177CA97C207C18312
:10EC5000116763E3E70293070910C207C183130733
:10EC6000B00F637BF70093170901C187AA8A634A33
:10EC7000F000C54763FE570141011733FFFF6700EE
:10EC8000A34797B0FFFFE780C028E31725FFD5B75C
:10EC900063080B0263060902814463890A02B7070D
:10ECA0007F0023106405231124057CC0568597003E
:10ECB0000000E780E0C39304803EB304950239A0CE
:10ECC000B7077F00232004047CC08144035524043B
:10ECD00097E00000E780A0A3A1C497C0FFFFE780F2
:10ECE00000BB269593D7F44133379500AE97BA977A
:10ECF00008DC5CDCCE85528597000000E780A0DC54
:10ED000099E023220404A1679387B70348003EC417
:10ED10002302010002C697E0FFFFE7808005A9BF3C
:10ED2000814701481CDC232E0403E9B71733FFFF9A
:10ED3000E702E33A97C0FFFFE780C037E1473305BA
:10ED4000F502914597500000E78000C5E55711C5D1
:10ED50009777FF1F23ACA7FC81473E851733FFFF42
:10ED60006700233A85471777FF1F2303F7FC82804C
:10ED70001733FFFFE702A3369777FF1F9387C7FA82
:10ED800080433DC0835704046390A706835724043F
:10ED9000639CB7043689B28497C0FFFFE78020AF39
:10EDA0005C5C63C3B7046395B7001C5C63EEA702A9
:10EDB0008347640463F3F400A6872303F4048347C2
:10EDC000740463F39700A687A303F40483574404F1
:10EDD00041677D176385E70085072312F4043C44EF
:10EDE00081C7CA85268582971733FFFF6700633185
:10EDF0009777FF1F938747F39C43014599C303C54A
:10EE0000870082801733FFFFE702632D0111B707E8
:10EE100007003EC683C79500584D0AC493F7F7070D
:10EE20000AC8A384F5002A89AE8411CB1C4283C78B
:10EE300007002304F70097900000E7800034216466
:10EE400093055402280097B0FFFFE7802027970022
:10EE50000000E78020FAAA85280097D0FFFFE7800E
:10EE6000A00A300001478146A6854A8597B0FFFF7A
:10EE7000E780204A13044402480822CC230A0100F8
:10EE800002CE97E0FFFFE780C0EE05611733FFFF7A
:10EE9000670023271733FFFFE702632401117C007B
:10EEA0003ECAB70707003ECC7C003ECE83C7950024
:10EEB0002E84AA8493F7F707A384F500A1659385B0
:10EEC0005502480897B0FFFFE780401F97000000F9
:10EED000E78040F2AA85480897D0FFFFE780C0028C
:10EEE000500801478146A285268597B0FFFFE7803D
:10EEF000404205611733FFFF6700A3209777FF1F8C
:10EF0000938787E29C43094599C303C59700828094
:10EF10009777FF1F938747E19C43094599C303C532
:10EF2000D70082809777FF1F938707E09C430145B6
:10EF300099C303C5A70082801733FFFFE702831838
:10EF40000111B70708003EC683C79500404D0AC4AB
:10EF500093F7F7070AC8A384F5002A89AE8429C469
:10EF60001442854703C7060063E0E70A834794001D
:10EF7000094681496380C702B307F740A304E40050
:10EF8000B339F00083C716002305F4009790000002
:10EF9000E780A01E03572403058B19C76386090069
:10EFA00097D00000E78000E92164930584022800DF
:10EFB00097B0FFFFE780801097000000E78040F4E3
:10EFC000AA85280097D0FFFFE78000F49700000093
:10EFD000E78080F5AA85280097D0FFFFE780C0F280
:10EFE000014781463000A6854A8597B0FFFFE7803C
:10EFF000403213047402480822CC230A010002CED6
:10F0000097E0FFFFE780E0D605611733FFFF670059
:10F01000A30E1733FFFFE702830C01117C003ECAE9
:10F02000B70708003ECC7C003ECE83C795002E84F7
:10F03000AA8493F7F707A384F500A1659385850259
:10F04000480897B0FFFFE780600797000000E7805F
:10F0500020EBAA85480897D0FFFFE780E0EA9700F9
:10F060000000E78060ECAA85480897D0FFFFE780A2
:10F07000A0E9500801478146A285268597B0FFFF89
:10F08000E780202905611733FFFF67008307977723
:10F09000FF1F938767C99C43014599C303C5B70008
:10F0A00082801733FFFFE70283030111B7070700D0
:10F0B0003EC683C79500404D0AC493F7F7070AC8B8
:10F0C000A384F5002A89AE8405C81C42054783C77E
:10F0D00007006368F7060347B400630FF700A30552
:10F0E000F40097900000E78040098347B400B9CF4F
:10F0F00097D0FFFFE78040BE21649305B40028004D
:10F1000097B0FFFFE78080FB97000000E78060F882
:10F11000AA85280097D0FFFFE78000DF01478146DE
:10F120003000A6854A8597B0FFFFE780801E29043E
:10F13000480822CC230A010002CE97E0FFFFE780B7
:10F1400040C305611733FFFF6700A3FB97D0FFFFA4
:10F15000E78020BF55B71733FFFFE70243F80111DF
:10F160007C003ECAB70707003ECC7C003ECE83C77A
:10F1700095002E84AA8493F7F707A384F500A16570
:10F18000AD05480897B0FFFFE78040F39700000007
:10F19000E78020F0AA85480897D0FFFFE780C0D617
:10F1A000500801478146A285268597B0FFFFE7807A
:10F1B000401605611733FFFF6700A3F49777FF1F21
:10F1C000938787B69C43094599C303C5C7008280CE
:10F1D0001733FFFFE702A3F001117C00AE843ECAA3
:10F1E000A165B70707002A843ECCD1057C004808FA
:10F1F0003ECE97B0FFFFE78060EC97000000E7800D
:10F2000020FCAA85480897D0FFFFE780E0CF500890
:10F2100001478146A685228597B0FFFFE780600FF2
:10F2200005611733FFFF6700C3ED1733FFFFE702E8
:10F2300003EB83C7950093F7F707A384F5009700C6
:10F240000000E78020F91733FFFF670083EB1733D7
:10F25000FFFFE70223E783C795000329C50141119A
:10F2600093F7F707A384F5001C4283C9070085477D
:10F2700063E637079777FF1F938707029C432E8427
:10F28000AA8485CF97000000E78080F38947630652
:10F29000F502630409028347C9006380370323062C
:10F2A000390197900000E78040ED83572903898B4F
:10F2B00089C797D00000E780E0B72685A285970030
:10F2C0000000E78020F1A167CD0748003EC423027B
:10F2D000010002C697E0FFFFE780A0A941011733B4
:10F2E000FFFF670063E19777FF1F9387E7A39C43C6
:10F2F0001D4599C303C5E70082801733FFFFE7026E
:10F3000003DE0111B70707003EC683C79500584DBD
:10F310000AC493F7F7070AC8A384F5002A89AE84C4
:10F3200015C71C4283C7070093968701E18663C413
:10F33000060685466381D7068346E7006388F600A4
:10F340002307F70097900000E78020E321649305EE
:10F35000E400280097B0FFFFE78040D69700000048
:10F36000E780A0F8AA85280097D0FFFFE780C0B902
:10F37000014781463000A6854A8597B0FFFFE780A8
:10F3800040F93504480822CC230A010002CE97E058
:10F39000FFFFE780009E05611733FFFF670063D61C
:10F3A0001733FFFFE702A3D301117C003ECAB70762
:10F3B00007003ECC7C003ECE83C795002E84AA84F5
:10F3C00093F7F707A384F500A165B905480897B03E
:10F3D000FFFFE780A0CE97000000E78000F1AA853C
:10F3E000480897D0FFFFE78020B2500801478146C8
:10F3F000A285268597B0FFFFE780A0F1056117334E
:10F40000FFFF670003D01733FFFFE702A3CBAA84F7
:10F4100001441779FF1F13096991E14997C0FFFF64
:10F42000E78040C96344A400014519A833053403AB
:10F43000832709003E9583572500639797001105A0
:10F440001733FFFF670043CB0504C9BF032E8500B8
:10F45000630A0E121773FF1F130303AC0323030089
:10F460006315030029436390061203234E016315BD
:10F4700003001D43639907101733FFFFE702A3C37F
:10F48000C689428A3E89BA8AB684328BAE8B2A8478
:10F49000B5E103554E0019E501431A851733FFFF07
:10F4A0006700E3C4A167A98F116763FBE7009700BA
:10F4B0000000E78080F5814597F0FFFFE780C012EC
:10F4C0000844B70700E05841F98F18455CC1B707F9
:10F4D000001FF98F1CC55C4991C7610597E00000CA
:10F4E000E780408BE38A09FA228597900000E78045
:10F4F00060C65DB7328597C00000E78040430D438A
:10F5000049DD1C44116703D54700A167A98F63FB40
:10F51000E70097000000E78040EF814597F0FFFF8C
:10F52000E780800C0323840093164B01D18283472C
:10F53000B300035663008588FD8BA305F300FD77B8
:10F540007D8E558EFD76FD16B204F18E8327430124
:10F55000C58E231273012313D30023045301230503
:10F560002301A3044301BDDF228597B0FFFFE7809D
:10F5700020CDAA850844B5D1610597D00000E78069
:10F58000207F8DB71D431A8582801733FFFFE70266
:10F5900063B30569AA84AE89328A0144FD5A7D1994
:10F5A00097C0FFFFE780C0A56347A400014517335C
:10F5B000FFFF670063B4D84493171400BA9703D7CA
:10F5C0000700631F37032390570163070A0026854E
:10F5D00097900000E780A0809C449DC383D767007C
:10F5E000B3F72701639E3701D2880148814701475D
:10F5F000814601468145268597000000E78040E569
:10F60000050479BF1733FFFFE702C3AB79711C1004
:10F610003EC4B7070F003EC61C103EC883C7950006
:10F62000AA8A328593F7F707A384F5002E893284DE
:10F6300097D0FFFFE780009D93170501C187635AAC
:10F64000F006AA89228597D0FFFFE780A09B2A8A2F
:10F650004E85032B040097B0FFFFE780009B39ED38
:10F660008357440081440544F11793B71700A3035F
:10F67000F10083457100DA872287D2864E86280002
:10F6800097E0FFFFE780E057014781463000CA85D9
:10F69000568597B0FFFFE780C0C7A1679387F70340
:10F6A00048083ECC230A810026CE97D0FFFFE78092
:10F6B000406C45611733FFFF670003A4A285130662
:10F6C000710097E0FFFFE7806066AA84094455D186
:10F6D000528597E0FFFFE78060D40D4459D9054675
:10F6E000D285268597000000E78060EA2A8451B71A
:10F6F0001733FFFFE702A39E835507000346270049
:10F7000041112A842E8532C62EC497E0FFFFE78080
:10F71000E0D001C93246A245228597000000E7806B
:10F7200000E741011733FFFF6700A39D1733FFFF79
:10F73000E702639883C795004111AA8A93F7F707F8
:10F74000A384F5003285AE89328497D0FFFFE7802D
:10F75000608B93170501C1876357F00AC1452A8A58
:10F76000228597C0FFFFE78080702A8D228597D081
:10F77000FFFFE78020892A89228597D0FFFFE78055
:10F780004086930705F893F7F70F1307E007AA8B56
:10F79000637BF706228597D0FFFFE78080842A8C61
:10F7A000228597D0FFFFE780C083AA8C5285032B68
:10F7B000040097B0FFFFE780408539E98357440094
:10F7C000231101008144F11793B71700A300F10042
:10F7D0000544034711008356210093878400568512
:10F7E000DA8822885286CE8597F0FFFFE78020A72F
:10F7F000A167E90748003EC42302810026C697D0CE
:10F80000FFFFE780005741011733FFFF6700238E9A
:10F8100013061100A28597E0FFFFE7802051AA841C
:10F8200009E52311010009446DB7930521006A859C
:10F8300097F0FFFFE780A0F02A8441FD8355210067
:10F840009356C9001316490185486688E2875E878A
:10F85000858A5182268597000000E78060BF2A8450
:10F860008DBF1733FFFFE702038583C79500411162
:10F870002A8B93F7F707A384F5003285AE8932848B
:10F8800097C0FFFFE780007893170501C187635297
:10F89000F00A2A8A228597C0FFFFE780A076AA8A0D
:10F8A000228597C0FFFFE780E0752A89228597C0EF
:10F8B000FFFFE7800073930705F893F7F70F13072F
:10F8C000E0072A8C6377F706228597C0FFFFE78061
:10F8D0004071AA8C228597C0FFFFE78080702A8D37
:10F8E0005285832B040097A0FFFFE780007239E563
:10F8F0008357440085440144F11793B71700A301CF
:10F90000F10003473100930784005A85DE8826887A
:10F91000D6865286CE8597F0FFFFE78040948D47CC
:10F9200048003EC42302910022C697D0FFFFE78023
:10F93000404441011723FFFF6700637BA285130644
:10F94000310097E0FFFFE780603E2A84894455D963
:10F950009356C9001316490185486A88E68762876D
:10F96000858A5182D68597000000E78060AEAA8420
:10F9700049BF1723FFFFE702E3742A89814401444A
:10F98000617A916A176BFF1F130B0B5997B0FFFF3A
:10F99000E780006863C7A40022851723FFFF670084
:10F9A000A3758327090093991400CE9703D5070008
:10F9B00033074501420741836364570305C10327A9
:10F9C0000B0019C785453E8597400000E78060E938
:10F9D000832709000504CE972390070085047DB78F
:10F9E00097000000E78060A2832709000504CE97F6
:10F9F0002390070065D5814597F0FFFFE780C0BEE3
:10FA0000F1BF1723FFFFE702E36B83C795004111A6
:10FA10002A8A93F7F707A384F50032852E8932846A
:10FA200097C0FFFFE780005E93170501C187635A07
:10FA3000F004AA89832A040097A0FFFFE780E05C16
:10FA400031E58357440085440144F11793B717000B
:10FA5000A301F10003483100D68752850147CE86C5
:10FA60002686CA8597D0FFFFE780806AA167F507E1
:10FA700048003EC42302910022C697D0FFFFE780D2
:10FA8000402F41011723FFFF67000367A28513067C
:10FA9000310097E0FFFFE78060292A8489445DD91F
:10FAA0009767FF1F938747479C4381CF044997B0CF
:10FAB000FFFFE780E055AA85268597400000E78094
:10FAC00040DA1305040197000000E780C0EA2285B0
:10FAD00097800000E78000338144ADBF1723FFFF0C
:10FAE000E702635D83C795004111AA8A93F7F70780
:10FAF000A384F5003285AE8932842311010097C0BA
:10FB0000FFFFE780205093170501C1876354F0067B
:10FB10002A8AC145228597C0FFFFE7804035AA8B1E
:10FB20005285032B040097A0FFFFE780004E21E9D8
:10FB30008357440085440144F11793B71700A3008D
:10FB4000F1000348110003572100DA875685D28659
:10FB50002686CE8597D0FFFFE780805BA1679387DD
:10FB6000270248003EC42302910022C697D0FFFF1F
:10FB7000E780202041011723FFFF67004357A2853C
:10FB80001306110097E0FFFFE780401A2A8489449A
:10FB90004DD99767FF1F9387273898433E8901CF38
:10FBA000044997B0FFFFE780A046AA8526859740C5
:10FBB0000000E78000CB1305040197000000E780F8
:10FBC00080DB97B0FFFFE780A04495443DD99305C3
:10FBD00021005E8597F0FFFFE78060B6AA8435F1CB
:10FBE0001C480357210022852390E70097800000DE
:10FBF000E780402183270900A9D7035521009740BA
:10FC00000000E780A0BD35BF1723FFFFE702A34A2E
:10FC100083C795004111AA8A93F7F707A384F500DB
:10FC20003285AE89328497C0FFFFE780A03D9317ED
:10FC30000501C1876351F0062A8A228597C0FFFF1C
:10FC4000E780403C2A895285032B040097A0FFFFE0
:10FC5000E780A03B31E58357440085440144F11718
:10FC600093B71700A301F10003483100DA875685E6
:10FC70004A87D2862686CE8597D0FFFFE780404907
:10FC8000A167F90748003EC42302910022C697D01D
:10FC9000FFFFE780000E41011723FFFF67002345A8
:10FCA000A2851306310097E0FFFFE78020082A8431
:10FCB00089445DD99167CA97C2071167C183130749
:10FCC000F7EF8544E362F7FA9767FF1F9387C7242E
:10FCD0009843BE8B01CF044997B0FFFFE7804033C4
:10FCE000AA85268597400000E780A0B71305040188
:10FCF00097000000E78020C897B0FFFFE780403101
:10FD000095443DD11C48228581442390270197804A
:10FD10000000E780200F83A70B00B9D74A859740E2
:10FD20000000E780A0AB89B71723FFFFE702233B62
:10FD30002A844105B28497000000E780C0C311C542
:10FD4000228597800000E780E00B81460146A6856A
:10FD5000228597800000E780C04E1C4C89C7DC4795
:10FD600099C3228582971723FFFF6700833997671E
:10FD7000FF1F938767FB9C43014599C313850701C8
:10FD800082809767FF1F938727FA88438280172313
:10FD9000FFFFE702C3349317C600DD8DC205411192
:10FDA000C1812A8432C697C0FFFFE780E017324640
:10FDB000228511829375F60F97C0FFFFE780C0146C
:10FDC00041011723FFFF6700C3331723FFFFE7023B
:10FDD000632F79713C083ED2B7070C003ED43C0833
:10FDE0003ED683C79500AE842A8993F7F707A3848C
:10FDF000F500A16593853504481097A0FFFFE780C3
:10FE0000E02BC165FD150144176AFF1F130A4A1252
:10FE1000930A400EAE892E8B2EC697B0FFFFE78067
:10FE200020224205931704014181C183B24563E951
:10FE3000A702C167FD176387F500481097C0FFFF51
:10FE4000E780800E501001478146A6854A8597A01D
:10FE5000FFFFE780004C45611723FFFF6700C329C0
:10FE60003307540383270A0BBA9703D6C701630AE3
:10FE70003601638A3501481097000000E78060F181
:10FE8000DA85050451BFB285EDBF1723FFFFE702F6
:10FE9000832279717C083EC8B70711003ECA7C08EE
:10FEA0003ECC83C79500AA89328593F7F707A384D0
:10FEB000F5002E8997C0FFFFE780C014856763783F
:10FEC000F504A165AA848905080897A0FFFFE780CB
:10FED000E01E268597400000E78060ED1334150092
:10FEE0000A04A285080897C0FFFFE780E001A68505
:10FEF000080897C0FFFFE780200325CC0147814613
:10FF00001008CA854E8597A0FFFFE78080404561B5
:10FF10001723FFFF6700A31DB30754030327CA0A73
:10FF2000BA9703D70700631C970003D627006380A6
:10FF30006505080897000000E780A0E5DE85050458
:10FF40002EC697B0FFFFE780A0104205931704016B
:10FF50004181C183B245E3E1A7FCC167FD17E38F8F
:10FF6000F5F8080897C0FFFFE78000FC41BFB285A5
:10FF7000F9B7C165FD150144176AFF1F130A4AFB53
:10FF8000930A80022E8BAE8B65BF1723FFFFE7021B
:10FF9000031518418347170083460700A207D58F32
:10FFA000D207D1832390F50083472700034717002A
:10FFB0008D45A207D98F91832310F60097C0FFFFCC
:10FFC000E780A0E91723FFFF6700A3131723FFFFB4
:10FFD000E702430FC16401441769FF1F130949F584
:10FFE00093098002FD1497B0FFFFE7806006634726
:10FFF000A40001451723FFFF6700031033053403F6
:020000040001F9
:100000008327C90A3E9583570500E38597FE0504BB
:10001000D9BF1723FFFFE702E30A2A8AAE89B28419
:10002000B68A97400000E78080D819E591473E8561
:100030001723FFFF6700430C2A894E8597C00000F5
:10004000E780E08E2A84638E0A048D476DD10357C2
:100050000500C547E31D47FD0347F9018546AD4748
:10006000E317D7FC8347450081CF4146A6855D0550
:1000700097F00000E780C09E814755D9AD4745BF46
:10008000130965012302E500CA8526859710000043
:10009000E780606231C1A547E38B0AF823020400C0
:1000A00079B705C183570500E39247F94146A68514
:1000B000190597F00000E780A09A81472DD999474C
:1000C000BDB74E8597000000E78080F02A849547F1
:1000D00039DD130955004DBF4146A6852310440163
:1000E000231134011305190097F00000E780A0994F
:1000F000228597800000E780A0EA81470DBF172383
:10010000FFFFE702C3FD79717C003ECCB7070A0010
:100110003ECE7C003ED083C79500B2842E8493F7F8
:10012000F707A384F5001306A1002A892C00268571
:1001300097000000E780A0E5A16528088D0597A03D
:10014000FFFFE780A0F790408355A1000355810091
:10015000854697000000E78000ECAA84AA8528085D
:1001600097C0FFFFE78040DA0356A1008355810066
:10017000280897000000E780C0C130080147814689
:10018000A2854A8597A0FFFFE780A0188547481001
:100190003ED42302910202D697D0FFFFE78060BDD4
:1001A00045611723FFFF6700C3F51723FFFFE70231
:1001B00003F379717C003ECCB7070A003ECE7C0089
:1001C0003ED083C79500B2842E8493F7F707A384AB
:1001D000F5001306A1002A892C002685970000004F
:1001E000E780E0DAA16528088D0597A0FFFFE7808A
:1001F000E0EC90408355A1000355810081469700B3
:100200000000E78040E1AA84AA85280897C0FFFF84
:10021000E78080CF0356A10083558100280897000E
:100220000000E78000B7300801478146A2854A8573
:1002300097A0FFFFE780E00D48102302910202D44F
:1002400002D697D0FFFFE780C0B245611723FFFFBA
:10025000670023EB1723FFFFE70263E89700000026
:10026000E78060DB1723FFFF6700A3E99767FF1FA5
:100270009387C7AB884382801723FFFFE70223E6FB
:10028000835725004111AE842A842307B10017F556
:10029000FFFF130525466C002316F10097A0FFFF12
:1002A000E780204991C4228597800000E780E0D64E
:1002B000FD572310F4001306200281451305540056
:1002C0009720FFFFE780A0E441011723FFFF6700AD
:1002D00043E31723FFFFE702E3DE79717C003ECCA6
:1002E000B7070A003ECE7C003ED083C79500AA899E
:1002F000AE8493F7F7073285A384F5001306A100B7
:100300002C0097000000E78080C80355810011444D
:1003100097400000E780A0A915C50355A10001443E
:1003200097B00000E780A06011CD03570500835708
:10033000810045446318F700854597000000E78079
:10034000E0F30144216993053900280897A0FFFFD5
:10035000E780C0D6A285280897C0FFFFE780C0BA13
:100360000356A10083558100280897000000E7800C
:1003700040A2300801478146A6854E8597A0FFFF21
:10038000E78020F948104AD42302810202D697D090
:10039000FFFFE780009E45611723FFFF6700C3D57D
:1003A0001723FFFFE70203D29767FF1F9387C797C3
:1003B0002A8488432E8915C5035745038357C401F2
:1003C0006311F7022326050223180502410597D081
:1003D0000000E780209C6306090097800000E7800A
:1003E00060DB81449769FF1F938989B4130A8002F7
:1003F00097B0FFFFE780C0C563C4A4049767FF1FE1
:100400009387479B9C4399C70355C40197200000DD
:10041000E780C0BD63070900228597800000E78060
:10042000C0A01306400E814522859720FFFFE7807C
:1004300000CEFD57231EF4001723FFFF6700C3CB38
:100440003385440383A7C90A3E95035705008357A4
:10045000C4016317F700CA8597000000E78000E237
:10046000850479B71723FFFFE702C3C583C795004B
:100470004111AA8993F7F707A384F5003285AE846A
:1004800097C0FFFFE78000B885676378F5042A8985
:1004900097400000E780A091014401CD83D704007C
:1004A000314463882701854597000000E78080EF8D
:1004B00001444E85A2864A86A68597D0FFFFE78035
:1004C000A09CA1679387170448003EC423028100C3
:1004D00002C697D0FFFFE780C08941011723FFFFC5
:1004E000670083C11723FFFFE702C3BD9767FF1FA4
:1004F00093878783804329C4014597C00000E78024
:10050000002181470148C1641CDC232E0403232001
:1005100004041769FF1F1309A9A101449309400EA0
:10052000FD1497B0FFFFE780A0B1634FA4008145A1
:1005300017F5FFFF1305857F97A0FFFFE780601F7A
:100540001723FFFF670043BB330534038327090BE1
:100550003E958357C5016387970085459700000046
:10056000E78040E4050475BF9357050113D7870062
:10057000A380F50093170501C183A1832380E500C3
:100580002381F500A381A50082801723FFFFE702E6
:1005900003B52300050083C71500A300F50083C73A
:1005A00025002301F50083C73500A301F50083C7AB
:1005B00045002302F50083C75500A302F50083C759
:1005C000650093059500A30305002303F5002304AC
:1005D0000500328597000000E78040F91723FFFFF0
:1005E000670023B21723FFFFE702C3AD4111E954AF
:1005F0000DCD85CD93F9C5FF2E842A89AA84338A2F
:10060000A900B7EA040063189A020D88854411CC4A
:10061000B7E704009C5F82972AC622866C003305E8
:10062000390197E00000E780004626854101172345
:10063000FFFF670063AC83A78A0391048297931737
:100640000501C183A183A38EF4FE93570501238F77
:10065000F4FEA183238EA4FEA38FF4FE6DB763E6A0
:10066000D5021723FFFFE70283A7B2874111368621
:10067000BE8536C697E00000E780E040B246410103
:1006800036851723FFFF6700C3A781463685828022
:10069000838705001387F5003D05FD8793F77708ED
:1006A000834607007D158606B58FA300F500630716
:1006B000B7007D17834717009D83DDB7828017231E
:1006C000FFFFE702C3A1B7E7040083A7070932874A
:1006D0002A863A858297133515001723FFFF670096
:1006E00043A215C181478DC11723FFFFE702239F56
:1006F000414697E00000E780003985473E85172393
:10070000FFFF670003A081473E8582801DCD172330
:10071000FFFFE702C39C414681452A849720FFFFE3
:10072000E780E09E41468145130504039720FFFFC3
:10073000E780E09D0147C1672322040438C87CC8D4
:1007400005451723FFFF6700C39B01458280814752
:100750003DCDB5CD1723FFFFE7026398B2842E8904
:100760001306800581452A849720FFFFE780209AA1
:10077000CA8524C4268597000000E780C0F641465C
:10078000814522859720FFFFE78060983044A2854D
:10079000228597000000E780C0F293040401A2853F
:1007A000268597000000E780E0EEA6851305040289
:1007B00097000000E78000EE228597000000E780A8
:1007C00020F585473E851723FFFF670083933E850D
:1007D00082801723FFFFE702E38E4111E9540DCD1C
:1007E00085CD93F9C5FF2E842A89AA84338AA9006E
:1007F000B7EA0400639844030D88814411CCB7E73D
:1008000004009C5F82972AC622866C00330539015A
:1008100097E00000E7802027268541011723FFFF8E
:100820006700838D83A78A0391048297931705013C
:10083000C183A183A38EF4FE93570501238FF4FE99
:10084000A183238EA4FEA38FF4FE6DB765CD17237D
:10085000FFFFE7022387B28411E605451723FFFF58
:10086000670083892A842E890145EDD93C48784860
:10087000B3E6E700E5D69386F7FFB3B7F6007D173A
:10088000032A4404BA9734C87CC863050A06C149E0
:1008900013050A03B38949412295637D3601B28667
:1008A0002E86A68597000000E780A0DB7C40BE94E2
:1008B00064C065B7CE862E86CE8597000000E7809F
:1008C00040DAC114D2944E9923220404A2879306DD
:1008D000040103C7070003C607038507318FA38FF1
:1008E000E7FEE398F6FE3044A285228597000000DB
:1008F000E78020DD2699C1493306994063EC9900D1
:10090000A9DCA686A6851305040397000000E780EE
:1009100040D579BF8147B306F4003307F60003479B
:10092000070083C5060085072D8F2380E600E3942A
:1009300037FF3044A285228597000000E78060D809
:10094000C1145DBF014582800DC11713FFFFE7028F
:1009500003791306800581459710FFFFE780207B10
:1009600005451713FFFF6700C37901458280814762
:1009700049C5C1C51713FFFFE7026376FC41414635
:100980002E84AA846399C70413860501A287814631
:10099000C14503C7070003C507038507298F330532
:1009A000D600034505008506298FA38FE7FEE39255
:1009B000B6FE3044A285268597000000E78060D00F
:1009C000228597000000E78060F885473E85171371
:1009D000FFFF67000373138507031D8E8145229572
:1009E0009710FFFFE780A0727C40130700F8130602
:1009F0000402A2972388E70251BF3E858280171325
:100A0000FFFFE702C36D6D712E84B284AA8590103A
:100A10002800368997000000E780A0D309EDD5575C
:100A200025A050400C40280097000000E78040E2DD
:100A30007DD5FD142104F5F42C004A8597000000B3
:100A4000E78020F3814761DD3E8551611713FFFF89
:100A50006700236B1713FFFFE702636841112EC481
:100A600032C62C00054697000000E78080F941015E
:100A70001713FFFF6700E3681713FFFFE702236602
:100A800001112A842EC602C802CA02CC02CE97E007
:100A90000000E780C023B2462A86A2850808970096
:100AA0000000E78060FB1375F50F05611713FFFF6A
:100AB000670023651713FFFFE70263627971B2874E
:100AC0002A8421462308B10013051101BE853AC4CA
:100AD00036C697E00000E78000FBB246930591011F
:100AE000368597000000E78060A8228514103546FF
:100AF0000C0897000000E78020F62A84224701E9CD
:100B000021460C103A8597E00000E780C0F7228567
:100B100045611713FFFF6700C35E1713FFFFE7026E
:100B2000035C7171AE84AA850A8532849700000047
:100B3000E78060BB11C90A86A68522859700000060
:100B4000E78020B8814711E1C5473E854D61171305
:100B5000FFFF6700035B1713FFFFE70243551D719B
:100B60002A8AB289BE8435468547130511012E8C29
:100B7000B68A3A8BC28C468D2308F10097E00000BC
:100B8000E78060F010100C085285231F01009700C9
:100B90000000E780C0F82A843DEDA1476313FD08FB
:100BA0009307900591E0E5473546E285130511016D
:100BB00013990A012308F1001359090197E0000075
:100BC000E78060EC1357890093978A00D98F9008CB
:100BD0000C085285231FF10097000000E78020F4E5
:100BE0002A8415E9A1E49387FA0091831379F90027
:100BF0003EC6631309004149668B8144C14B854D54
:100C0000B247639F970C6A868C0033855C0197E03E
:100C10000000E78040E7228525611713FFFF67008A
:100C2000C34C93079004C9F0A547BDBF8347010596
:100C30000947C14B2308F10083471105A58FA3087D
:100C4000F10093872400814463E1FB040147140809
:100C50003386E6008C08B386E400BA95DA9683C63C
:100C6000060083C505000507AD8E2300D600E3907E
:100C7000E7FE4147639CE70490080C085285970003
:100C80000000E780C0E925D181A0B3069B00BA87A8
:100C90001008B305F60090083E9603C5060003460B
:100CA000060085078506298E2380C500E39277FF1D
:100CB000998F90080C085285BE9497000000E78039
:100CC00000E68947014749D12A84B1B790083E968A
:100CD000034606001408BE962380C600850759BF48
:100CE000B24785046387971481471808B306F70055
:100CF00098083E973386F90003470700034606002D
:100D00008507318F2380E600E39177FF90080C0878
:100D1000528597000000E78080E05DF53546E2856A
:100D2000130511012308B10197E00000E780A0D569
:100D3000139704014183939784002183D98F10185E
:100D40000C085285231FF10097000000E78020DD8A
:100D500025FD814710183387F9003E9603470700A9
:100D600003460600B306FB008507318F2380E600AB
:100D7000E39277FF65A81808B306F70098083E9736
:100D80003386F90003470700034606008507318FC5
:100D90002380E600E3E127FFCA87639E7709900876
:100DA0000C08528597000000E78060D711FD81474D
:100DB0009800B306F700900818103E973E96034738
:100DC0000700034606008507318F2380E600E39184
:100DD00077FF3546E285130511012308B10197E03D
:100DE0000000E78040CA1397040141839397840071
:100DF0002183D98F10180C085285231FF10097000A
:100E00000000E780C0D1E31105EC8147101833875B
:100E1000F9003E960347070003460600B306FB00B1
:100E20008507318F2380E600E3E227FFC109410BEC
:100E3000C1BB814785B79408BE9683C606001808D3
:100E40003E972300D700850789BF638006321713BA
:100E5000FFFFE702C32559712A84BE89B28B8547FB
:100E60003546130511022E8B468C4289BA8A368A82
:100E70002300F10297E00000E780E0C010180C109A
:100E800022852317010297000000E78040C96318FC
:100E90000512A147631FFC069307900563930900A1
:100EA000E5473546DA851305110293140A0123003C
:100EB000F102C18097E00000E780E0BC93178A0050
:100EC00013D78400D98F90080C1022852317F102C4
:100ED00097000000E780A0C47DE1639209049307B6
:100EE000FA00BD88918391E0C144C207C183DE8CC2
:100EF000814A3EC6414DB24763E2FA0E6286B3852F
:100F00004B01881097E00000E78080B54DC93D5542
:100F10007DA093079004E39609F8A54759B7834746
:100F200001050947C14C2300F10283471105B3C7EE
:100F3000F900A300F10293872900814963E1FC04D1
:100F4000814618103306D7008C083387D900B69530
:100F500056970347070083C5050085062D8F23009C
:100F6000E600E390D7FE41476390E70690080C1037
:100F7000228597000000E78080BA35D189A0B3862A
:100F80003A01BA871010B305F60090083E9603C5E3
:100F900006000346060085078506298E2380C500C6
:100FA000E39297FF3387EC4090080C102285BA99A2
:100FB00097000000E780A0B68947014741D16561ED
:100FC0001713FFFF6700631290083E960346060062
:100FD0001410BE962380C600850779B7B247850AEC
:100FE00093990A01939D8A0093D909016391570F40
:100FF00085473546DA85130511022300F10293D99E
:10100000890097E00000E78000A8B3ED3D01900063
:101010000C1022852317B10397000000E78020B051
:1010200059FD8147A68963EA970626860C084A85FA
:1010300097E00000E78020A581471810B306F7006D
:10104000100898083E973E9603470700034606009F
:101050008507318F2380E600E3E197FE639FA905B2
:1010600090080C10228597000000E78040AB21F922
:1010700081479810B306F700900818183E973E96DF
:1010800003470700034606008507318F2380E600EB
:10109000E391A7FF4109C10CB9BD18089000B30640
:1010A000F7003E963387FC0003470700034606001F
:1010B0008507318F2380E600B5B798084E97034720
:1010C00007001C10CE972380E700850941BF8547A4
:1010D0003546DA85130511022300F10293D9890000
:1010E00097E00000E780209AB3ED3D0190000C10DE
:1010F00022852317B10397000000E78040A2E31088
:1011000005EC814718089000B306F7003E96338738
:10111000FC0003470700034606008507318F238044
:10112000E600E391A7FF41460C084A8597E00000DE
:10113000E780609581471810B306F70010089808FB
:101140003E973E9603470700034606008507318F0A
:101150002380E600E391A7FF90080C1022859700FA
:101160000000E780C09B1DD599BD7D558280171377
:10117000FFFFE702C3F601112A842E859305510073
:10118000328902C002C202C402C69304740097F0FE
:10119000FFFFE780A03D1D46A6851305910097E05F
:1011A0000000E780408E10088A854A85970000007D
:1011B000E780E09619ED93071400180883C607002E
:1011C0000346070085070507B18EA38FD7FEE39777
:1011D000F4FE05611713FFFF6700A3F21713FFFF6B
:1011E000E70243EE2E848C414111AA8983871500C2
:1011F0003289914463D30700A1449757FF1F938717
:10120000A7099C43A1C7C1CA8D472310F10083C71A
:1012100025004A852301F10083C73500A301F100B1
:1012200083C745002302F10083C75500A302F100E4
:1012300083C7650093059100A30301002303F10018
:101240002304010097F0FFFFE78040320C404A86FC
:101250000A8597F0FFFFE780803303280400835658
:101260004400A6881D0881470147E51642868A8505
:101270004E8597000000E780408E2A8919E5A685F3
:10128000228597B0FFFFE780E0C14A85410117132F
:10129000FFFF670063E64A860A8597F0FFFFE78055
:1012A000002F6DB71713FFFFE702C3E12E848C41B7
:1012B0004111AA89838715003289914463D30700BD
:1012C000A1449757FF1F938727FD9C43A1C7C1C621
:1012D0008D472310F10083C725004A852301F100C3
:1012E00083C73500A301F10083C745002302F10045
:1012F00083C75500A302F10083C7650093059100E1
:10130000A30301002303F1002304010097F0FFFF72
:10131000E780C0250C404A860A8597F0FFFFE780EA
:10132000002783564400032804008A85858EC20660
:101330001D08C1822312D400A68881470147E51603
:1013400042864E8597000000E78060B04101171388
:10135000FFFF670063DA4A860A8597F0FFFFE780A0
:1013600000234DBF1713FFFFE70263D7B335B0006B
:10137000011185052A891315F60133651501230826
:10138000B1009305110136843AC632C03EC442C250
:1013900097F0FFFFE780801DA2471248425593D681
:1013A0008700230BF1009305910193578800A30A4E
:1013B000D100A30BF100230C010197F0FFFFE780A0
:1013C000E01A3247024603280400B337E000835690
:1013D00044009207914411C2A1444A85A6884286DE
:1013E0000C0897F0FFFFE78040772A8919E5A6856A
:1013F000228597B0FFFFE780E0AA4A8505611713B1
:10140000FFFF670003D01713FFFFE702A3CB011113
:101410003EC68647B335B0008505AA891315F60187
:101420005D8D2308B1009305110136843A89B28499
:1014300042C446C297F0FFFFE7804013224892481B
:10144000164593578800A30AF1009305910193D79D
:101450008800230B0101A30BF100230C110197F06D
:10146000FFFFE780A0103247104083564400B33797
:10147000E000920703280900914891C0A1480C0898
:101480004E8597000000E780809CAA8401E983557F
:1014900044004A8597B0FFFFE780C0A0268505611C
:1014A0001713FFFF670043C5AA959307F00F1707AF
:1014B00001001307E75A6317B50013C5F7FF13754B
:1014C000F50F828005058346F5FFB58FBA9783C770
:1014D0000700D5B70357450014419307F00F1706CF
:1014E00001001306E657369742074183139506011C
:1014F0004181631BE500AD8FB29703C5070013055B
:1015000015F3133515008280850603C5F6FFA98FF4
:10151000B29783C70700D9BF1713FFFFE70223BCA9
:10152000B28736842E86BA86AA853E85BA8497F01D
:10153000FFFFE7806052634F0500228597D00000CF
:10154000E780E0782A86A686A285268597F0FFFFA9
:10155000E78080501713FFFF6700A3BA1713FFFF40
:10156000E70243B65D712A8BAE8A170501001305A9
:10157000A54C2C00B284368ABA893E8997F0FFFFC9
:10158000E780C04F2A845DE134104146DA852800A7
:1015900097F0FFFFE780404C2A8449E98547A30381
:1015A000F100A6C2930771002408BEC4A686854731
:1015B0000D462C18281002DC02DED6C0BEC697F0FD
:1015C000FFFFE78000442A8435E183477102A68645
:1015D0000D4693F7F7072300FA00C1473EDE2C18AB
:1015E0008947281026DCA303F10097F0FFFFE7806E
:1015F00040412A8405ED4146A6854E8597D00000DE
:10160000E78060488D47A6860D462C182810A30356
:10161000F10097F0FFFFE780C03E2A8401E94146D0
:10162000A6854A8597D00000E780E0452285616164
:101630001713FFFF670043AC1713FFFFE70223AA4E
:1016400097F700009387C7A0984383C74700797135
:101650002A89AE84170501001305853E0C083AC49B
:101660002306F10097F0FFFFE78040412A8405ED53
:1016700014104146CA85080897F0FFFFE780C03D77
:101680002A8415E1140815462C00081097F0FFFF76
:10169000E780803C2A8401E921462C08268597D0E2
:1016A0000000E780403E228545611713FFFF670079
:1016B00043A51713FFFFE70283A297F70000938764
:1016C00027999C477971AA842E8417050100130578
:1016D000A5370C083EC697F0FFFFE780203A0DE9DA
:1016E00014104146A685080897F0FFFFE780C03632
:1016F00005E1140811466C00081097F0FFFFE78021
:10170000A03519E58347F10193F7F7032300F400AF
:1017100045611713FFFF6700C39E1713FFFFE70222
:10172000039C3688A14881470147E54697F0FFFFB3
:10173000E780A0421713FFFF6700A39C1713FFFF6A
:10174000E702E3993688A14881470147E54697F0CB
:10175000FFFFE780C06F1713FFFF6700839A17131F
:10176000FFFFE702C39701112A842E850C0832C6B9
:1017700097F0FFFFE780803009ED324797060100C0
:101780009386062B1008C145228597000000E7804C
:10179000E0D805611713FFFF6700A3961713FFFF3B
:1017A000E702E3934111C1472EC032C48A8509463E
:1017B0003EC23EC697F0FFFFE780A0244101171309
:1017C000FFFF670003941713FFFFE70243914111E6
:1017D000AE8613061009AA850A8502C002C202C499
:1017E00002C697F0FFFFE780202741011713FFFF94
:1017F000670023911713FFFFE702638E3287970676
:1018000001009386E6242E869305000297000000CF
:10181000E780C0D01713FFFF6700A38E1713FFFFE9
:10182000E702E38B7971C1472ACC2ED032D42C0841
:101830000D4628003ECE3ED23ED602C402C602C8A5
:1018400002CA97F0FFFFE780C01B45611713FFFF37
:101850006700238B1713FFFFE70263880111AA8437
:101860002E84170501001305251F8A8597F0FFFFB9
:10187000E780C02015E514084146A6850A8597F043
:10188000FFFFE780601D09ED8347E1010347F10198
:10189000A207D98FCA07C9836177D98F2310F400B3
:1018A00005611713FFFF6700C38515CD1713FFFFF1
:1018B000E702E3829747FF1F9387C74B9043974503
:1018C000FF1F9385654B1745FF1F1305A54697D04E
:1018D0000000E78000C51745FF1F1305A545171336
:1018E000FFFF670003821745FF1F1305A544828091
:1018F0008DCD1703FFFFE702837E9747FF1F938776
:101900006747944301112E840A869745FF1F9385EC
:10191000A54697D00000E78040C60A85029401459D
:1019200005611703FFFF6700C37D7D5582801703A4
:10193000FFFFE702C37A97D00000E78080D1974786
:10194000FF1F23A9A74217F5FFFF1305E5C997B0AD
:101950000000E780C0741703FFFF6700837A174712
:10196000FF1F130767439317150008433E95FD5764
:101970002310F50082801703FFFFE70243762A84D5
:10198000084009E51703FFFF6700A3771C41584093
:101990001CC06313E5005CC083475500232005008D
:1019A000F99BA302F50097A0FFFFE780207CC9BF49
:1019B0001703FFFFE70203719747FF1F9387C73F96
:1019C00098432A8411CB8347350093F7070289C7D0
:1019D00003550500894502971305440197B000009F
:1019E000E780403B835504000355E4009730000036
:1019F000E780A00C485819C597A0FFFFE780007743
:101A0000232A04021305840397000000E780E0F610
:101A10008144B1499790FFFFE780C06D63CBA4027A
:101A2000834734002320040493F727FCA301F40028
:101A300000489790FFFFE780E06C13161500814582
:101A400022859700FFFFE780806C1703FFFF670088
:101A5000A36AB38734030329040385043E994A85A6
:101A600097000000E78060F12304090065B7834711
:101A7000350093F7070299E3014582808357E5001B
:101A8000E39CB7FEC167FD176316F600054582802B
:101A9000054599A81703FFFFE70263649317060142
:101AA000C187B2842A8401496359F0028357050033
:101AB0009DCB01456367F600034584003E953325C1
:101AC000A6001375F50F0DA01C4813171900BA973F
:101AD00083D70700E38E97FA05099790FFFFE78009
:101AE0006062E343A9FE01451703FFFF67006361DE
:101AF0001703FFFFE702035DAE89AA849790FFFFFB
:101B0000E78000562A8497D0FFFFE780A02EAA86A0
:101B100001471306840197050000938585E4174566
:101B2000FF1F1305A5279790FFFFE780801C2A89D8
:101B300025C98C441304C50022859E0593F505082C
:101B400097A0FFFFE780403CCC4083877400E18191
:101B500063DD070493E50508228597A0FFFFE78072
:101B6000A03A0D4693854400228597A0FFFFE780A9
:101B7000C03683D50400228597A0FFFFE780E03DB3
:101B800083D52400228597A0FFFFE780003D03D680
:101B9000490083A50900228597A0FFFFE780E03375
:101BA0004A851703FFFF6700235593F5F5076DB7C7
:101BB0001703FFFFE702A35201112A84328532C6C0
:101BC00097A0FFFFE780E0279780FFFFE780603462
:101BD000835704001747FF1F130787353246231B1F
:101BE000F100930700F8A30DF1001C471843231AD6
:101BF000A1008983858BB307F740B28548083ECEA4
:101C0000231C0100230D010097000000E78080EEF7
:101C100005611703FFFF6700C34E1703FFFFE702CD
:101C2000634A004101453DC49304C40026853289BE
:101C3000AE8997A0FFFFE780C02495452A8A2685B4
:101C4000035B040197A0FFFFE7802021268597A072
:101C5000FFFFE780603E8D45AA8A268597A0FFFF9B
:101C6000E780A01F268597A0FFFFE780E03C5C4847
:101C7000420A135A0A01D2975CC4231864018147AF
:101C800063983A0146054D81330625419337160086
:101C900013F5F70F1703FFFF670003461703FFFF56
:101CA000E702634189692A8BAE8B328AB68A814406
:101CB0000144314CFD199790FFFFE780A04363CDAD
:101CC000A4009790FFFFE780E045018D33B5AA009F
:101CD0001703FFFF6700A3413389840383270B00A9
:101CE0003E9963170A008347890085043E94E1B753
:101CF00003560A00DE854A8533F6C90097000000C6
:101D0000E780E0F16DD10545E1B71703FFFFE7027A
:101D1000033D01112A847C000355E5003ECAB70744
:101D200007003ECC7C003ECE97200000E7802008D4
:101D30002A898545480897A0FFFFE7802039994503
:101D4000480897A0FFFFE780E015AA844A859720FE
:101D50000000E780A0082380A4009747FF1F938717
:101D6000271D9C434166130606F09396870113D7FF
:101D70008701558F93D68700F18E558FA207B7063E
:101D8000FF00F58FD98F11462C00138514003EC437
:101D900097D00000E78020CF5008A3820400894537
:101DA000228597000000E780E0E019C9AA851305A5
:101DB000840397A0FFFFE780E0313C4085073CC0EB
:101DC00005611703FFFF6700C3331703FFFFE70237
:101DD00003319790FFFFE780E0342A840504979051
:101DE000FFFFE78020333305A402F1479145330517
:101DF000F50297200000E78020BA11E5655517032A
:101E0000FFFF670003309747FF1F23AFA7F89790A6
:101E1000FFFFE78020312A8405049790FFFFE780C9
:101E2000602F3305A4028945060597200000E7804E
:101E3000A0B669D59747FF1F23A0A7F69790FFFF8D
:101E4000E780402E2A8405049790FFFFE780802CCE
:101E50003304A4029747FF1F239287F49790FFFF54
:101E6000E780402C2A849790FFFFE780A02A930701
:101E700014003385A7029747FF1F2392A7F2970705
:101E80000100938727811747FF1F232DF7F0014596
:101E9000BDB71703FFFFE702E322AA842E8901449E
:101EA0009749FF1F9389C908130A80069790FFFF7F
:101EB000E78040266347A40001451703FFFF670042
:101EC000A3233305440383A709024A86A6853E95CA
:101ED00097000000E780E0B919E10504C1BF05459E
:101EE000E9BF1703FFFFE702031DAA8A2E8BB28BFF
:101EF000368C3A8A814401448149974CFF1F938C68
:101F00002C03130D80069790FFFFE780A02063C984
:101F1000A40011E085494E851703FFFF6700231DCC
:101F20003389A40383A70C025E86D6853E994A8531
:101F300097000000E780E0B31DC19790FFFFE780A6
:101F4000601E0544636D4501D2866286DA851305FD
:101F5000090397000000E780A0D411C185498504DA
:101F60005DB71703FFFFE702E315C16441112A893A
:101F700001449749FF1F9389A9FB130A8006FD14AA
:101F800036C632C42EC29790FFFFE780A018924554
:101F90002246B2466348A400014541011703FFFFF2
:101FA000670083153305440383A709023E9509C6DC
:101FB00083473500C18B9DC791C68347350093F792
:101FC00007028DC3630699008357E500639C2701D0
:101FD0000357050001CB63E7E50083478500BA9707
:101FE000E3CDF5FA050469BF1703FFFFE702830D90
:101FF000C1642A8901449749FF1F938969F3130A31
:102000008006FD149790FFFFE780C0106346A40090
:102010001703FFFF6700430E3305440383A709023C
:102020003E958357E500638A9700630499006396A1
:10203000270197000000E780E0970504E1B7170348
:10204000FFFFE702C30689692A8AAE8A328BB68B04
:102050008144174CFF1F130CACED930C8006314DDF
:10206000FD199790FFFFE780E00A63C6A4001703FD
:10207000FFFF670083073389940383270C0283558E
:10208000CA015A863E994A8597000000E780609E03
:1020900031C1814D15A03384AD038327090303D6D5
:1020A0000B00D68533F6C9003E94228597000000C8
:1020B000E780E0B609E9850D9790FFFFE780800390
:1020C000E3CBADFC01A8228597000000E780E08A01
:1020D00023040400850471B71703FFFFE702A3FD83
:1020E0004169AA8A014A174BFF1F130B6BE47D1944
:1020F000C14B054C9790FFFFE780C0016346AA00E3
:102100001703FFFF6700A3FE93098006B3073A0396
:1021100083290B02BE9983D7E900638E270163846C
:102120002A01639A570103A4890301E84E859700A9
:102130000000E780C0BD050A75BF8357040163999D
:1021400077099304C400268597A0FFFFE78060D33A
:1021500085452A8D2685835C040197A0FFFFE780D3
:10216000C0CF268597A0FFFFE780A0E762056185C5
:10217000635905048D45268597A0FFFFE780E0CDD4
:102180008945268597A0FFFFE78020CD89452685D4
:1021900097A0FFFFE78060CC8545268597A0FFFFCD
:1021A000E780E0CC83470500094793F7F707639A78
:1021B000E7009945268597A0FFFFE78040CBA30263
:1021C00085014848337D2D01231894016A9548C440
:1021D0000040A1BF1703FFFFE70263F037E40400EC
:1021E0008327041D82979747FF1F83C767C1171571
:1021F000FF1F1305A533A300F5008327441C829716
:102200008327841C81461306F00F81450145829780
:102210001703FFFF6700E3EE1747FF1F130747AEE3
:1022200018439745FF1F83C5A5BD9747FF1F938799
:10223000A7BB83468703034697036397D500974759
:10224000FF1F238FC7BA828083C587010347A70377
:102250006317B6009747FF1F2384E7BA828003C63F
:1022600087016317C7009747FF1F238BD7B882806A
:1022700083C68701130750026319D70093076002D2
:102280001747FF1F230EF7B6828083C68701130608
:1022900060026315D60093077002DDB783C787011C
:1022A00055BF9747FF1F938727B4D44B0947638DCA
:1022B000E6081703FFFFE70283E21749FF1F130930
:1022C000E9AF3E8483470900918B9DCFB7E40400BA
:1022D00083A7041D829783A7441C1745FF1F13057E
:1022E00065AE829783A7841C81461746FF1F03466D
:1022F00066AF81450145829721C583470900ED9B63
:102300001747FF1F230CF7AA8347040093F7F70F23
:1023100085CB91471747FF1F2322F7AE9700000098
:10232000E78080EB97000000E78040EFB7E704000C
:10233000BC4F414691451745FF1F034565AB82974A
:102340001703FFFF6700E3DB82801703FFFFE7024D
:1023500003D98D4741116306F504C5476308F502AB
:1023600085476310F5029747FF1F238DA7A8B7E79E
:102370000400BC4B930500101745FF1F034545A7FC
:10238000829741011703FFFF6700A3D785471747CF
:10239000FF1F2309F7A6B7E70400BC4B93050020F5
:1023A000E1BF9747FF1F938727A4D44B1147638D45
:1023B000E600B7E7040083A7071D8297B7E704008C
:1023C000BC4B930500044DBF05491747FF1F23274A
:1023D00027A383C7070032C62E8493F7F70FD5D300
:1023E000B7E4040083A7041D7D141374F40F8297CF
:1023F000E37689FCB245994703C61500E3F0C7FCB4
:10240000FC4409061745FF1F130505A08297BC4829
:10241000930500081745FF1F0345859D829779BFE7
:102420001703FFFFE702A3CB1747FF1F1307C79B45
:102430004047184B1C409746FF1F23ADF69A631682
:10244000E4001747FF1F2329F79A130584FE97908E
:10245000FFFFE78000AA035564FF9780FFFFE78036
:10246000807297A0FFFFE78060D01703FFFF67002F
:1024700043C91703FFFFE70283C69747FF1F9387F0
:10248000A796D84BDC4789C797000000E78080F902
:1024900085471747FF1F2323F7969747FF1F93870B
:1024A00027869C43930500021745FF1F034545946B
:1024B00083C787031747FF1F2304F794B7E7040078
:1024C000BC4B82971703FFFF6700A3C39747FF1F0B
:1024D00023AEA79082801703FFFFE702A3BE37E475
:1024E00004007C4CA1451745FF1F0345659082976A
:1024F0007C48A1451745FF1F0345858F9744FF1F63
:102500009384848E8297DC4489EB97000000E780F7
:1025100080D91703FFFF670023BE03D567FF9780AD
:10252000FFFFE7804066AA896DD1D84891476310C4
:10253000F7027C4C91451745FF1F0345658B829739
:102540007C4891451745FF1F0345858A829703A95B
:10255000490103D409018947B7E904001747FF1F60
:10256000232EF78883A7091D21044204829783C77D
:1025700084011715FF1F130565FB61191717FF1F4E
:10258000A306F7FA83A7491C418082979747FF1F4C
:10259000238A078683A7C91C814609469375F40FD1
:1025A0004A85829711E99747FF1F83C7E79589C737
:1025B0009700FF1FE7800064B7E70400BC4F214687
:1025C000A1451745FF1F0345A582829799B71703B9
:1025D000FFFFE702C3B093F7052001112E8481CFDE
:1025E00097000000E78020E91345042005611703E8
:1025F000FFFF670003B193F70510A9CF9734FF1FC2
:102600009384847EDC4897000000E78020C1173760
:10261000FF1F1307E76E184383C78401034787032F
:102620006318F700DC4489C797000000E78080DF6B
:1026300085471737FF1F2323F77CB7E70400BC4B00
:10264000930500021735FF1F0345857A82971345CE
:10265000041069BF93F70508BDC79737FF1F83C7ED
:10266000B77AE91719469735FF1F9385057A130541
:10267000D10093F4F70F1739FF1F0349E97897C08A
:102680000000E780404093970401C1831737FF1F84
:1026900013070778231DF100231CF1009737FF1F54
:1026A000938787743ACE3ACAD8432306010009CBF0
:1026B000DC439315890154080D46E1856800829733
:1026C0001345040825B793F72500A5C39737FF1FC7
:1026D00093878771D84B89476306F7029737FF1FA7
:1026E00083C7C76D13F7270011EF918B99CFB7E719
:1026F0000400BC4F1306000A89451735FF1F034528
:10270000256F829713452400D5B59737FF1F938710
:10271000275F9C4383C787031737FF1F2302F76E8A
:1027200097000000E78060DBF1BF93F7050281CBE3
:1027300097000000E78060DA1345040245BD93F777
:10274000850081CB97000000E780E0D2134584002C
:1027500071BD93F7150081CB97000000E780A0B40E
:102760001345140061B593F7450081CB9700000035
:10277000E78060B31345440095BD93F7050495C306
:102780009737FF1F83C7476691CB97000000E7800C
:10279000A0A491471737FF1F2322F76613450404AF
:1027A000B1B593F705010145E38207E49737FF1FB1
:1027B00093878763D84B91476310F7049737FF1FC0
:1027C0009387C75F9C4313D727008583D98F858B59
:1027D00091E7B7E7040083A7071D8297B7E70400D6
:1027E000FC4F91451735FF1F03458560829785474C
:1027F0001737FF1F2324F76013450401C5BB973724
:10280000FF1F2383A77082801703FFFFE702238D3A
:102810009737FF1F23A0075E9737FF1F23AE075C84
:1028200085471734FF1F1304A44D1737FF1F2327B5
:10283000F75C1C4083C787031737FF1F2302F75C31
:102840009790FFFFE780409329C59717FF1F23A3A9
:10285000A7CE1C40170500001305A5D783C7870323
:102860001737FF1F230EF7581717FF1FA300F7CCCA
:102870009737FF1FA38A0756B7E7040083A7070807
:1028800082979737FF1F2385A7561703FFFF67001F
:102890004387B7C7898E938767ED1717FF1F232BD1
:1028A000F7C845BF1737FF1F03470754795555E74A
:1028B0009737FF1F9387475303C7170005079736BE
:1028C000FF1FA383E65203C717008D463377D70255
:1028D0009736FF1FA38AE65083C617001737FF1FDE
:1028E00013070742184393F6F60FA9EE83478703B1
:1028F0001737FF1F2306F75085471737FF1F23059C
:10290000F74E9737FF1F9387674B9C430145998B81
:10291000A9E717F3FEFFE702837C37E404007C4855
:10292000C1451735FF1F0345A54C82973C48854597
:102930001735FF1F0345C54B8297014517F3FEFF6F
:102940006700237C83C7170085466395F60083479D
:10295000970379BF8347A70361BF82809737FF1F23
:1029600083C78748A1CF17F3FEFFE702437737E419
:1029700004009737FF1F238907467C488545173594
:10298000FF1F0345E54682977C4C91451735FF1F95
:102990000345054682977C4891451735FF1F03453F
:1029A000254582973C48C1451735FF1F03454544DF
:1029B0008297014517F3FEFF6700A3747955828063
:1029C00017F3FEFFE702A3712A84035565FF978082
:1029D000FFFFE780401B9737FF1F9387E740D847EB
:1029E000BE841DEF9790FFFFE78080779C482320EF
:1029F00004009DEB9737FF1F23A087409737FF1FE9
:102A000023AA873EB7E70400BC4B89451735FF1F53
:102A10000345053E8297014517F3FEFF6700636E8D
:102A2000630A8700184375BF80C39737FF1F23A52C
:102A3000873CC9BF7955CDB717F3FEFFE702236A7C
:102A40009737FF1F9387874C88432326050023244D
:102A50000500510597A00000E780C03317F3FEFF83
:102A60006700236A17F3FEFFE70263671734FF1F4F
:102A70001304C4491C40411199CF9C472302B5005F
:102A80002AC61CC197000000E78040FB1C409C4BFD
:102A900099C332458297410117F3FEFF67006366D1
:102AA00017F3FEFFE702A3634111444D32853284E0
:102AB0002EC69790FFFFE780C0522AC422859790C8
:102AC000FFFFE780205403A84400630C0800B245D0
:102AD000835744001840224683D54500AA862685A0
:102AE0000298410117F3FEFF6700A36117F3FEFF91
:102AF000E702E35E404D1DC808C0970500009385BE
:102B000065031305440197A00000E780401697373E
:102B1000FF1F9387A73F9C43014589E79737FF1F16
:102B200023A6873E17F3FEFF6700A35D7D55DDBF3B
:102B300017F3FEFFE702A35A011168009305F00F97
:102B400002C602C802CA02CC02CE97000000E7808B
:102B5000A0F1056117F3FEFF6700A35A9737FF1F27
:102B60009387C73A9C43D847A1679D076319F7022B
:102B700017F3FEFFE702A356011132859790FFFF7E
:102B8000E7802046230AA1008145680097000000E5
:102B9000E78080ED056117F3FEFF670083568280B2
:102BA0009737FF1F938787369C43D847A167938742
:102BB00077036319F70217F3FEFFE702435201118F
:102BC00032859790FFFFE780C041230AA10081452D
:102BD000680097000000E78020E9056117F3FEFF19
:102BE0006700235282809737FF1F938727329C43C9
:102BF000D84795476316F70417F3FEFFE702234E05
